:10000000F01F0010256F0000236F0000236F000019
:10001000236F0000236F0000236F0000000000002A
:10002000000000000000000000000000236F00003E
:10003000236F000000000000236F0000AD350000BA
:10004000AD330000AD330000AD330000AD33000030
:10005000AD330000AD330000AD330000AD33000020
:10006000AD330000AD330000AD330000AD33000010
:10007000AD330000216F0000216F0000C1000000BF
:100080004936000061360000613800007938000010
:10009000216F0000C1390000216F0000216F0000B6
:1000A000216F0000216F0000216F0000216F000010
:1000B000216F0000216F0000216F0000216F000000
:1000C000594A10B5136801331360584B584A1B68DE
:1000D000DBB2302B00D176E018D8182B5AD005D8D7
:1000E000082B37D0102B46D0082351E0202B00D10D
:1000F0007AE0282BF8D14F4B4F491868096888429D
:1001000052D21968481C18604C4B48E0482B00D16B
:100110006AE00AD8382B60D0402BE5D1484B1968EB
:10012000042301295DD11360DEE7502B66D0582BE4
:10013000DAD14448444B1B680168DBB24C1C0460B4
:10014000424843540221424BFF3119608023F13968
:10015000DB0530E00021374B19601968481C186036
:10016000364B5B5C3849DBB20B60282313600122FD
:10017000374B1A6010BD0021324B19602D490B68B6
:10018000581C08602D49CB5C2F49DBB20B6028233B
:100190001360EFE727490B68581C086027495B5C30
:1001A0002949DBB20B609FE7254B19688023DB05EB
:1001B000002902D02021196096E702202449FF304F
:1001C00008601021F7E780231021DB051960082360
:1001D000136081221E4B5200CBE782211C4B490049
:1001E000E9E78021C905DDE780231021DB051960DF
:1001F000082313600422164BFF32BAE71149124B51
:100200001B680868DBB2441C0C60104C23540C4B78
:100210001B680868013B0421834202D98023DB0567
:10022000C9E7116060E7C0462806001004000040DE
:1002300018000040240600101C060010F4050010F1
:100240000806001020060010080000400C060010F0
:100250000406001002231B4A70B511681A4D0B43A7
:1002600013602023194A040011680B431360184BD4
:100270001A682A401A600122186810431860154B4A
:1002800019682940196019680A431A606C22124BD8
:1002900012491A60124B186806F016FF114B1860CD
:1002A000114B1860022C02D1A022104B1A60802240
:1002B0000F4B12021A6080234022DB0501201A60D6
:1002C00070BDC04604800440F8FCFFFF80800440FD
:1002D000304004403440044018000040400D03000A
:1002E000B804001014000040100000400C00004052
:1002F00000E100E00000000000000000FFFFFFFF41
:10030000202303490A681A42FCD0024B1860704748
:10031000148000400080004070B504000D002900EA
:10032000200003F03FF9024B1B68002BF7D170BD92
:10033000D405001010B503F067F910BD10B500200A
:1003400002F054F902F020F910BD00007FB505005D
:1003500000200C0002F0F0FA002801D003F006FFA4
:10036000002323602B60174B1E78002E28D121001C
:10037000280002F00FFB300002F0DEFA002807D060
:1003800003F0F4FE2660210028002E6002F002FB3C
:100390000D4B1B78002B13D00C4B2A6818680C49A6
:1003A000824203D120680D68A84209D01A602368F0
:1003B00001A80B60074903F033FD01A803F0D0FD4D
:1003C0007FBDC04684020010940200107C02001021
:1003D000800200104073000070B504000D00FFF7AC
:1003E000B5FF094A1368002B09D0013B1360032BAA
:1003F00006DD064B1B682360054B1B682B6070BD38
:1004000000232B602360FAE790020010880200109E
:100410008C0200100023034A1360034A1360034A4E
:10042000136070478C0200109002001088020010C8
:10043000002310B50B60036002F0ACFA10BD0000A1
:1004400010B5012403F058FE0C4B0020196803F08E
:100450007DFA002003F06AFA002003F047FA084B07
:1004600020001C60074B196889B203F035F92000A1
:1004700003F022F9200003F0FFF810BDC0040010C3
:10048000F0050010BC04001037B50C240321012036
:1004900003F088F8684601A9FFF79EFF009D002D34
:1004A00002D1013C002CF1D1FFF7CAFF002005F07A
:1004B00047FE28003EBD10B5002003F027FA0120BA
:1004C00003F0EAF803F01EFE10BD000070B50D0049
:1004D0000400FFF7B5FFF8230121064ADB00D150E5
:1004E0002000290005F0B6FAFFF7E5FF05F00EF948
:1004F00070BDC046D806001070B504000D00FFF7AF
:100500009FFF0822074B29001C60074B20001D603D
:10051000064B1A6005F09EFAFFF77CFFFFF7CBFF52
:1005200070BDC046880200108C02001090020010BE
:1005300010B50400FFF784FF200005F0C3F90400A4
:10054000FFF7B9FF200010BD10B50020FFF7F0FF46
:1005500010BD37B504000025FFF7F6FFA54203DB09
:10056000FFF7F2FF00983EBD0321062003F01AF8C2
:10057000684601A9FFF730FF009B002BF0D1013541
:10058000ECE7000010B502000249034803F03DFC0F
:1005900010BDC0464E73000057730000F0B5354BD8
:1005A00085B01B6800900193002805D0019B002BAB
:1005B00002D0002002F028FC01F0B1FF002002F080
:1005C00015F801F0E1FF2C4C0322236802210133CE
:1005D00023602A482A4B02F00DF92368FA26013BD2
:1005E000236002F009F8FFF7AFFF2648FFF7CAFFC4
:1005F00096230024244D9B002B60B60003F0B6FA2E
:10060000002807D002F094FD00242B680134A34297
:10061000F4DC1AE0009B002B27D01C4F3100386817
:1006200006F052FD6423584302F0D6FF02F042FE6A
:100630003100386806F048FD02F0CEFF03A902A899
:10064000FFF7CAFE029B002BDFD0009B002B05D0DA
:10065000019B002B02D0012002F0D6FBFFF774FFB4
:100660000B4803F0D2FB05B0F0BD0A2002F0CCFF2E
:10067000E4E7C04640000010380000105F7300003F
:10068000589800006E73000050020010B80400106B
:10069000747300001A4B73B504001A49186806F009
:1006A00013FD194B194A1A490090200003F0B8FBBA
:1006B00002F056FA002812D002F070FAFA218900EE
:1006C000060006F001FD0500200003F0F7FB114BCA
:1006D0002A006B4310499B19201803F0A1FB20004E
:1006E00003F0ECFB0D4B0E4A1B682018002B02D0C8
:1006F0000C4A00DB0C4A0D4903F092FB73BDC04667
:10070000B804001040420F00857300004E730000D3
:100710008973000018FCFFFF96730000B4040010FA
:100720007F73000082730000F3980000A173000043
:1007300070B50D0006001400002001F057FF01F015
:1007400023FF310028000022054B02F053F8092254
:100750000121044B200002F04DF801F04DFF70BD67
:10076000589800004098000007B5144A1449012029
:10077000FFF7DEFF642002F047FF72B60021114B45
:10078000114A196001231360116013601168194246
:10079000FCD00E4A6846136080230D4A5B02116844
:1007A0000B43136080230B4A11680B4313603923FA
:1007B00001A90093084B984707BDC046A9730000E4
:1007C000B873000070800440748004407880044056
:1007D0008080044038820440F11FFF1F00B5084BA1
:1007E000084A89B01B7868461278074903F018FB5D
:1007F00069460120054AFFF79BFF09B000BDC046CE
:1008000035000010A7040010CB730000D97300005E
:10081000F0B52C4C2C4D237885B001932F78002611
:10082000FFF7DCFFFFF790FE02A803A9FFF7D4FD56
:100830000298002815D0C0B201F0FAFF492805D867
:100840003F281ED830282CD0392835D001F088FE1A
:10085000FFF7C4FF029E002E03D0C82002F0D4FE92
:100860000026032104200136FFF756FD1E2EDBD1A2
:10087000019B2F70237001F073FEFFF765FE05B03A
:10088000F0BD40380928E1D806F06CFB05F2E0E045
:10089000E0E0F7E0E0102B783E2BD7D801332B7047
:1008A000D4E72B78002BD1D0013BF8E72378062B37
:1008B000CCD801332370C9E72378002BC6D0013B85
:1008C000F8E7C04635000010A704001070B50D0011
:1008D000040001F024FE2A0021000120FFF728FF78
:1008E000012005F02DFC70BD10B590B06846FFF7F3
:1008F000D1FE002001F07AFE01F046FE0122084CF4
:1009000011002300684601F075FF23000922012130
:10091000044801F06FFF01F06FFE10B010BDC0463B
:1009200040980000ED73000000B52B228DB0002828
:1009300000D1023268460D4903F072FA04A803F0B0
:10094000A5FC6946012004AAFFF7F2FE032000215E
:10095000FFF7E2FC0220FFF7EBFD0028EED00021BC
:100960000A20FFF7D9FC0DB000BDC0460774000097
:10097000F8B5040016000D00002703F087FC2100E5
:10098000E7741431681C03F0A1FA380001F02EFE60
:1009900001F0FAFD3A00042120000A4B01F02AFF81
:1009A000094C092223000421280001F023FFBE4244
:1009B00005D0230009227821044801F01BFF01F033
:1009C0001BFEF8BD5898000040980000477A0000D0
:1009D00030B58DB0134902A803F078FA2E24002216
:1009E00002A904A8FFF7C4FF0025FFF7ADFDFF34FF
:1009F000002202A904A8FFF7BBFF0321002002F098
:100A0000D1FD684601A901950095FFF7E5FC009B23
:100A1000002B02D1013C002CEAD1FFF795FD0DB06F
:100A200030BDC04618D80000F0B5002491B02000B9
:100A30009626039401F0DAFDFFF786FD02232700D6
:100A400000940193760001F09FFD009B002B00D0E5
:100A5000ABE008AD280003F019FC009BEB742B748D
:100A60006B73AB72EB712B71002C01D1012F05D18F
:100A70000022042128008F4B01F0BCFE8D4D002286
:100A80002B001E218C4801F0B5FE012C01D1012F55
:100A900007D11D202B0002AD00222521401901F0B5
:100AA000A9FE844D00222B003321834801F0A2FED1
:100AB000022C6FD1012F6DD0232002AD00224D21D9
:100AC0007C4B401901F096FE7A4D00222B005921F3
:100AD0007A4801F08FFE042C01D1012F07D1262086
:100AE0002B0002AD00225F21401901F083FE714D01
:100AF00000222B006C21714801F07CFE052C01D1F5
:100B0000012F07D129202B0002AD002272214019AC
:100B100001F070FE09220421694B0DA801F06AFE64
:100B200001F06AFD039B002B07D0143B012B41D839
:100B3000052C3FD0962002F067FD03210800FFF747
:100B4000EBFB002001F0F8FE0023050004A903A838
:100B500004930393FFF740FC039B002B00D199E023
:100B600006AE05AD3100280007AA03F0C3FB0090D4
:100B7000002828D1280003F0A3FC070003981238AE
:100B8000052800D97EE006F0F7F9217D56237D186F
:100B90001E0058E72B0000223A210AA801F02AFE85
:100BA000032C89D1012F8FD186E700220421414BEC
:100BB0004448B3E7FFF7C8FCBFE7601C062106F016
:100BC00069FB00270C009626760067E0601DF5E7BC
:100BD000601E042804D806F0CFF90D141D26470026
:100BE0002B88013300242B80280003F069FC0523A7
:100BF000070016E00C21A87806F062FA0131A9700E
:100C0000F2E701372900380003F08CFC05230224A9
:100C100001932BE030780130182106F03BFB0423D0
:100C20003170019322E0707801303C2106F032FBF4
:100C300003237170F5E7601E042804D806F09CF9C0
:100C4000060C0E1114002B88013BCBE7A8780C2171
:100C50000A3006F01FFBD1E7013FD3E730781730A9
:100C6000DAE770783B30E0E70023B3700721380003
:100C700006F010FB0A000791052C05D13100280071
:100C800003F090FB01279EE731002800019B03F051
:100C900049FBF7E7002D01D101235F40039B842B23
:100CA00005D0182B03D0731E002E00D070E711B0B2
:100CB000F0BDC04658980000107400006074000039
:100CC0004098000012740000114B10B59A6D032A71
:100CD0001AD11C00BB3460782278A178000210433E
:100CE0000904E27808430B49120602438A420BD1F9
:100CF000BA3318780F23034000090F2B03D00F28B5
:100D000000D00A33180010BD01204042FBE7C04666
:100D1000D8060010AFACEAFF3E230F2230B51349CE
:100D2000FF33CC5C0133CB5C1340013BDBB2002CC6
:100D300016D0062B17D80720020062438A18D21853
:100D400015009C352D78062B07D1013C4443091929
:100D50009C3108780002284330BD9D321078F9E7B5
:100D600001204042F8E70220FBE7C046D806001009
:100D7000030003480B2B02D8024A9B009858704787
:100D8000F39800006C7C0000CB10C05C0723194076
:100D90000841063B184070470300103B70B5040043
:100DA0000D000020B72B13D9FA2C11D80F2C10DC12
:100DB000144B1B5D144A9B0029009858FFF7E4FF71
:100DC00000281CD1032C09D129001048FFF7DCFFB3
:100DD00070BD0F4B1B19C83B1B78EBE7042C02D1ED
:100DE00029000C48F2E7252DF2D10F2C02DC0A4B2A
:100DF000185DEDE709480419C83C2078E8E70120B0
:100E0000E6E7C046E8830000080000109683000073
:100E1000F8830000A0830000A5830000B5830000D4
:100E2000002370B505000C001600037099421DDB0D
:100E30002A2925DC032905D11B4B1B78DB0707D5A5
:100E4000083405E0042912D1174B1B78DB0715D4B1
:100E5000164BA2002800D15803F038F8012C18D006
:100E6000002E03D02800124906F044FA70BD07296D
:100E7000EED1104B9B6D082BEAD1E1E70C24E7E79C
:100E8000C83C322CF2D80C4BA400E15803F01EF8F9
:100E9000E6E7084B9B6D042BE2D1280003F00EF827
:100EA000281805F0B5FFDBE7690200102C8400006C
:100EB00020740000D8060010D884000010B500226D
:100EC000FFF7AEFF10BD70B500250400080011004B
:100ED000AA420EDB28225A4352185200115F4B1CC3
:100EE00007D0A94207DA02235B42591AFFF7E6FF4F
:100EF0000125280070BD06F009F8F9E770B5060075
:100F00000D00140005F050FF002806D0042D04DC6D
:100F1000022C02D00122141BE4B22A00310023006B
:100F20000148FFF7D0FF70BD9C7C0000F7B50500BD
:100F30000F00019205F058FF060001000022280072
:100F4000FFF76EFF33000D3B012B0AD8280002F09B
:100F5000B5FF3900019A2818FFF7D0FF04002000E0
:100F6000FEBD284B1A78012314001C401A4213D0EE
:100F7000F31E012BEAD8300039000830FFF70CFFD0
:100F80000028E3D0280002F099FF002329183A0036
:100F90001D48FFF798FFE1E7072E28D11B4B9B6DFB
:100FA000082B00D1083630003900FFF7F5FE061E89
:100FB000E8D11749280006F09DF9280002F07EFFCD
:100FC0003900019A2818FFF799FF041EC7D139008C
:100FD0001048FFF7D9FE041EC1D0280002F06EFFB2
:100FE000330029183A000848FFF76DFFB7E7F31EF2
:100FF000012BD8D839000848FFF7C6FE0028D2D008
:10100000ADE7C0466902001014830000D806001046
:101010002274000082830000878300001FB50D4BFF
:101020001B78002B0AD1FFF777FE0100431C05DB7C
:10103000431C05D10848023105F024FD05B000BD70
:10104000684605F063FF6B461B78002BF6D0012144
:101050006846F1E7790200102474000010B505F02D
:1010600085F800280BD0002001F0C0FA01F08CFABE
:10107000FFF7D4FF01F0A8FA012001F0B7FA10BD84
:10108000F0B51E4B85B01B78002B05D105F086FE10
:10109000041E03D0FFF7C2FF05B0F0BDFFF714FE3A
:1010A000051E08DB05F0EAFC2800FFF761FE0221BF
:1010B00005F0E8FCF0E72100684603F00BFB104F59
:1010C0000E223900684606F0F1F80E4D0E4E0F4C18
:1010D000002803D12B78726D93420BD00E22694603
:1010E000380002F0A8FE736D2200694601202B70C3
:1010F00005F0E4FD200005F0E1FCCDE779020010E9
:101100006A02001078020010D80600105802001081
:1011100010B505F02BF800280BD0002001F066FA7E
:1011200001F032FAFFF7ACFF01F04EFA012001F0B6
:101130005DFA10BD10B5FFF7EBFF10BD1121044A99
:10114000DC3213788B43034909780B4313707047E3
:10115000D806001069020010024B1878C006C00FB4
:101160007047C0466902001070B5FFF7F5FF012512
:10117000041E0D4E05D00D4B53331D7000233370EC
:1011800070BD33782B42F9D005F02EFE03380128CC
:1011900006D8074B210078201D70FFF797F9EDE77F
:1011A0000B22024B9A65E9E769020010D80600108D
:1011B00084020010F0B5050087B0002901D0012499
:1011C00012E005F0FDFD041EF9D1344E3278382DC1
:1011D0000DD110231A4053425A4112013270FFF7C9
:1011E000ADFF01222E4B1A70200007B0F0BD012781
:1011F000782D07D13B0093433370FFF79FFF284BB7
:101200001F70F1E73A4053000193FFF7A5FF002854
:1012100000D00197280005F0A9FD070005F0A0FD0A
:101220006B4639001A79002812D002A8FFF77EFE1B
:101230000028C4D005F0B2FD00280DD0FFF794FFC0
:101240000122174B002128001A70FFF73FF9CBE766
:1012500002A8FFF753FEEBE70620FFF769F9002825
:1012600004D102A805F0ECFC01F0C6F92A20FFF732
:101270005FF9041E07D0FFF777FF00212800FFF772
:101280003BF90024B0E7074805F0DAFC01F0B4F9B7
:101290003470FFF753FFFFF757F9A5E76902001015
:1012A000840200102D74000010B5002802D1FFF751
:1012B0005BFA10BD002001F099F901F065F90122F7
:1012C0000A4C012123005242094801F093FA2300FD
:1012D00007220121074801F08DFA01F08DF97820ED
:1012E000FFF737F98428E4D1E1E7C04648980000C9
:1012F000327400004474000070B504000D0001F069
:101300000EF9262C13DC0020102C27DD20001138CC
:10131000152814D805F030FE1D132D6D373F4E13E0
:101320003113131313131313264213131345442CB1
:1013300054D006DC372C58D00120382C56D0002051
:101340000CE0452CFBD1E120000103F045F8012021
:1013500048E02A4B1B68002B01D1012070BDFFF72C
:1013600037FBFAE7254B1B68002BF6D0FFF75CFB39
:10137000F3E70120FFF712F9EFE70120204B1B688C
:10138000C01A01F041FD0120FFF7AEFAFFF7DCF8CB
:10139000FFF77AF8E1E7FFF73BFADEE704F0D6FE65
:1013A000DBE70022174B1A70174B05321A7001F059
:1013B000D7F8D2E704F0DAFE144B002806D01968FB
:1013C0000322022900DD00221A60C6E71A68511CB8
:1013D000062A01D01960C0E71860BEE70C4802F089
:1013E000FBFF0020FFF7A0FAB7E7002004F0B8FEEB
:1013F000B3E72800FFF758FFAFE7C046B40400107A
:1014000040000010A704001035000010C8000010B4
:10141000F0F1FFFFF8B5012706000C00002001F0F5
:10142000E5F801F0B1F80B4D7F422B003A000121A5
:10143000094801F0DFF92B003A0030002A2101F0C1
:10144000D9F92B0007220121200001F0D3F901F086
:10145000D3F8F8BD489800005B740000030010B595
:1014600003480449002B00D09968FFF7D3FF10BD53
:10147000F398000062740000F0B5002787B001F017
:101480004EF82A4D2A492800FFF7C4FF3C00FFF719
:101490005BF80C260321062002F084F8684601A9B7
:1014A000FEF79AFF0098002804D10137772FF1DD6D
:1014B00007B0F0BDC0B201F0BBF90200462808D069
:1014C000002C0AD00023E356834206D10020205688
:1014D000EEE7002CFAD10027DCE7352A01D0412ABB
:1014E00021D114481449FFF795FFFFF72DF800208C
:1014F000DEE7934206D124182000FFF7AFFFFFF785
:1015000023F8E8E70131300048432356002BF0DC94
:10151000F1D00A4902A802F083FC28000849FFF72D
:1015200079FF0024EBE70021064CECE7F39800007C
:1015300062740000817400006E7400008374000007
:101540008A740000A4850000020010B50F240E323A
:101550000B78234003700B7801311B094370023074
:101560009042F5D110BD000010B50722024B01F0EA
:10157000E9F8013010BDC04648980000F0B50A25D2
:1015800089B004AE0C0001003000FFF7DDFF737876
:101590005D433378ED18B378002B00D0643D737B46
:1015A000002B05D021002D20FFF7DEFF013024188D
:1015B000307B21003030C0B2FFF7D6FF6B1E0B2707
:1015C0002418022B11D837000195F87A2100303009
:1015D000C0B2FFF7C9FF019B2418013B0193013FF3
:1015E000002BF2D10B277F1B1D0003230193019BCE
:1015F000F35C002B11D021002E20FFF7B5FF02383D
:101600002418F05D21003030C0B2FFF7ADFF019B20
:10161000013F24189F42F4DA04E0019B0133019357
:101620009F42E4DA002D18D02A000D4902A802F0EA
:10163000F7FB21009E20FFF797FFB37801380419CC
:10164000002B03D021002D20FFF78EFF2100072261
:10165000044B02A801F0CEF80400200009B0F0BD50
:10166000D67300004898000010B5084B08481B7856
:10167000012B03D00748022B00D1074809227D2106
:10168000064B01F0B7F800F0B7FF10BD00000010E6
:101690009774000095740000817400004898000061
:1016A000F0B543688DB0040086680020019300F017
:1016B0009DFF00F069FF0023E3564A4D002B00D147
:1016C00088E02A78012A0BD0022A00D17FE032007C
:1016D000022B00D0019A444904A802F0A1FB05E0C6
:1016E0003300019A414904A802F09AFB0122404FBD
:1016F00001213B00524204A801F07CF82A78012520
:10170000931E591E8B41DBB202930023E356023B2A
:1017100059424B41DBB203931523E356552B11D1AC
:10172000002A0FD0029B039A93420BD129003B0061
:1017300007222D2001F006F8411920002030FFF784
:101740001DFF0500274B2A4F1B78002B0BD0029B57
:10175000039A2A20934200D1653029003B000722DA
:1017600000F0F0FF2D18200029000C30FFF706FFD5
:101770001523E3560500552B13D11A4B1B78002B6C
:101780000FD0029B039A93420BD001003B0007222B
:101790002B2000F0D7FF291820002030FFF7EEFEA5
:1017A000050000230F4AE3561278002B05D0022AC9
:1017B00015D0002A01D1022B11D03B000722E91CD1
:1017C000300001F017F8FFF74FFF0DB0F0BD320009
:1017D000019B87E7019904A802F078FB86E7019E48
:1017E000EBE7C04600000010A274000099740000EE
:1017F0004898000070B5050000200C0000F0F6FECF
:1018000000F0C2FE0122084E28003300012152429E
:1018100000F0F0FF330007220121200000F0EAFF72
:10182000FFF722FF70BDC04648980000064B074AEC
:101830001B6810B5990088580549002B00D105494F
:10184000FFF7D8FF10BDC046040000103480000030
:10185000A9740000BC74000010B5084B1B78012B64
:1018600004D0022B07D00649064801E00649074884
:10187000FFF7C0FF10BD06490648F9E70000001059
:101880001E7500002E750000D1740000E474000085
:10189000F77400000A75000010B5002802D0FFF7A9
:1018A000FFFE10BDFFF7C2FFFBE7000010B505F01B
:1018B0008FFA002808D036230720044AFF33D35C70
:1018C000043B58439C30801810BDC046D806001019
:1018D00010B5040005F082FA002803D00021712021
:1018E000FEF7F4FD07222100064802F0A4FA05F0F5
:1018F0006FFA002805D0FFF7D9FF0722002102F078
:10190000BBFA10BD82070010F0B53F4E87B004004F
:101910000D000722310002A802F08DFA05F058FAF6
:10192000002806D0FFF7C2FF0722010004A802F03A
:1019300082FA27000C373800FFF7CAFF002D60D06D
:10194000324B1D78023D6B1E9D410023E356EDB2E4
:10195000023B5A425341DBB201931523E356552B08
:1019600015D1019B9D4212D120002030FFF7B0FF1E
:1019700000217820FEF7AAFD00217120FEF7A6FDC8
:1019800014200021FEF7A2FD3800FFF7A1FF00217F
:101990007820FEF79BFD71200021FEF797FD019B4B
:1019A00017209D4200D105380021FEF78FFD152339
:1019B000E356552B12D1019B9D420FD020002030C1
:1019C000FFF786FF00217820FEF780FD00217120BF
:1019D000FEF77CFD00211520FEF778FD072202A905
:1019E000300002F028FA05F0F3F9002805D0FFF7DF
:1019F0005DFF072204A902F01EFA00217120FEF704
:101A000065FD712007B0F0BD8207001000000010D6
:101A100030B58BB000F083FD3A4D2868FFF73CFFEE
:101A200044E004000321062001F0BCFD684601A942
:101A3000FEF7D2FC0098002804D10134772CF1DDA8
:101A40000BB030BDC0B200F0F3FE020042280FD14F
:101A50002D4A1378023B591E8B415B001370FFF730
:101A6000FBFEFEF771FD2868FFF716FF0024D9E79B
:101A7000432805D1244A1378013B591E8B41EDE7D9
:101A8000462807D128680028CBD01F4B1978FFF7CC
:101A90003BFFD5E734280ED11C4A002113680133DF
:101AA000012B06DC13602960FFF7C0FEFEF74CFD3A
:101AB000DCE71160F7E7352801D0412807D1144849
:101AC0001449FFF797FEFEF73FFD0020B8E70F4BE4
:101AD00011491B689B005B580121595618000029C9
:101AE0000BDC0DD000230D4902A82B6002F098F901
:101AF0000B4902A8FFF77EFED8E714339142EBD1E1
:101B000028608BE754020010000000100400001051
:101B100081740000457500003C8000005C75000089
:101B2000F3980000F0B58DB002F046FB012004F000
:101B300017FBF82700211820FEF7C8FC00248E4E62
:101B4000FF00FEF7B8FC00238C4DEB51200002F0A3
:101B500055FB002C73D00121002001F023FD200053
:101B600002F046FB03A90300019002A8002B69D0F4
:101B7000FEF75EFC01230193002C13D002F03DFB25
:101B8000029B182B02D0019B002BDAD000207C4B4B
:101B9000187000F02BFD00F045FD7A48FEF7F2FCCE
:101BA0000123EB6602F072FA029E182E0ED1002C71
:101BB00000D183E0039BD8B200F03AFE0121FFF789
:101BC0009BFBE851002801D00023039305F0E6F8C1
:101BD00004430CD1029B182B09D1694B1B78DB07FE
:101BE00005D5FFF715FF002800D188E00290039982
:101BF0000298FFF7DFFA002807D0FFF7B5FAFEF7E3
:101C00001FFC0399029803F025FF00225E4B1A7017
:101C1000EB59934201D0FEF797FC94352B685C4258
:101C20005C41002B6ED100F063FC584B1A78002AFF
:101C300003D000221A70FEF787FC4F4E81E7032184
:101C400006208AE7FEF7F4FB029B002B94D1002CC0
:101C500000D07BE74E4B1B68002B00D076E72B00B3
:101C600098331B68002B1DD14A4B0024F61800D472
:101C70006CE7494B1B78002B0BD0484802F070F9F9
:101C8000642001F0C1FC464802F06AF9642001F0CA
:101C9000BBFC00F02DFC2B00002294330224364EB6
:101CA0001A6053E73F4A13681133136003F0E6FDEF
:101CB000029B01330293102BF8DDD5E7FFF74CFAB6
:101CC000002883D02E4B300021001C70FEF7FEFB55
:101CD000FFF7D2FB0394061E00D177E72100FFF740
:101CE0000BFB002800D071E7F0B200F0BDFD0390BF
:101CF000482E00D16AE701222B4B1A7066E7782341
:101D0000029374E700F060FF002000F06FFC0025F4
:101D100000F03AFC05F054F8A84204D105F020F890
:101D2000431E9841050001263000684004F066FE1D
:101D300004F01CFA002806D0FFF7A2F900F044FCDA
:101D4000300000F053FC002D0DD005F04DF804AD2F
:101D5000010001222800FFF763F82B78002B02D046
:101D6000280004F078FF05F02BF8002801D104F0DA
:101D7000EFFD00F041FC58E720BF0200D80600103C
:101D8000690200107E7500007902001084020010C4
:101D9000D40500100CFEFFFF940200106A750000CD
:101DA0007475000034060010F40E001073B54A4C30
:101DB0004A4B22684A4D9A4202D1256001F0C4F88C
:101DC0002368AB4201D100232360072602F0B8F854
:101DD00000F072FD0021434801F03AFA012500218C
:101DE000414801F035FA00F047FE00F0EBFF002219
:101DF0003E4C100023680B21B343236023682B4320
:101E0000236001F0B7F92000394C102101F020FACD
:101E100023680022B3432360236828002360042141
:101E200001F0A8F90021200001F012FA01F08CF96C
:101E30009620000201F000FE01232E4D5B4200209F
:101E40002B60FEF751FD002350242B600120FEF78C
:101E500001FA00F0B7FF02F079F92B68002B05D1E9
:101E60006420043C01F0D0FB142CEFD10020FEF7DD
:101E70003BFD2821204802F0BDFB142001F0C4FBEB
:101E80001D48282102F0B6FB1C4801F0BEFF1920B6
:101E900001F0BAFB01F06AFE002819D00020FEF71D
:101EA0007DFB0821164801F0D3F902F002FC03F093
:101EB00065FB0F230193DB18124A13491348009363
:101EC000134B03F075FB134803F0A6FBFFF72AFE44
:101ED000013C002CDBD1E4E708000010BE153E37C2
:101EE000E45BE173984004409C400440744004402B
:101EF00094400440B4040010DE0300008875000024
:101F000010400440CD080000D9030000216A000001
:101F100034060010F0050010F7B5031E019137D00C
:101F20000278303A504242419B181A78782A13D1ED
:101F30001026012501331A7800242D2A01D10133FE
:101F4000013400221878002809D1002C00D0524218
:101F5000019B01201A601BE00A260025EBE7070021
:101F6000303FF9B2092903D87243BA180133E9E7BF
:101F700020210843002D07D00700613F052F03D81B
:101F8000120157380243F1E7024801F03EFF0020FA
:101F9000FEBDC046A08600000378202B00D070470D
:101FA0000130F9E703003038C2B2092A08D92020ED
:101FB00018430300613B5738052B01D901204042EB
:101FC000704770B50E00FFF7E7FF0025040020788A
:101FD000002802D13560200070BDFFF7E3FF002824
:101FE000F8DB2D0105430134F1E7000010B500F0E6
:101FF000D5FD0100014801F008FF10BDAE860000CC
:1020000000B589B0684602F041F96946024801F01E
:10201000FCFE09B000BDC046ED860000F7B50E001D
:1020200001A91500FFF778FF002814D0019F0B4984
:10203000380005F02FF90C006421200005F02AF982
:1020400020003170642105F03FF804492870380001
:1020500005F03AF8FEBD01204042FBE710270000E2
:1020600013B50C006B4660689A1DD91DFFF7D6FFAB
:102070006B4698805A1C991CA068FFF7CFFF6B46EF
:102080006A4618709288044B9A4203D9694601A89F
:1020900002F088F913BDC0466B0700000B0007B5BE
:1020A000586801A9FFF738FF3C20019B584302F014
:1020B00093F907BD07235843074B9C30C018831D75
:1020C0000138834201D1012070471A78013B002A70
:1020D000F7D00020F8E7C046D80600107FB51948B1
:1020E00001F093FE00240326651C34421DD120001C
:1020F000FFF7E0FF002814D02800FFF7DBFF0028DF
:102100000FD0A01CFFF7D6FF00280AD0E01CFFF775
:10211000D1FF002805D00434FF2CE5DD01F03AFFA3
:102120007FBD2100084801F070FE2100684602F0E2
:10213000D1FA684601F01EFF044801F066FE2C004B
:10214000EAE7C0464E730000BA86000017D80000C8
:1021500070B50D00FFF720FF060004000D350E36A8
:1021600020780134FFF71EFF002807DB2870013DAF
:10217000B442F5D12000FFF70FFF70BD0020FCE74F
:1021800070B53F4C86B02368002B07D13D4801F065
:102190003CFE03F0F3F9012323602DE00868012BD6
:1021A0000FD10822384901F098FE002802D1236897
:1021B0000133F1E7354801F028FE03F0DFF9344937
:1021C0003FE00378412B19D132490230FFF7C0FFBD
:1021D0000028F2D00378422BEFD12F490230FFF7CD
:1021E000B7FF0028E9D00378432BE6D12B49023012
:1021F000FFF7AEFF0028E0D006B070BD532B02D130
:1022000027490230F4E74D2B20D126490230FFF751
:102210009FFF0028D1D003784E2BCED12249023027
:10222000FFF796FF0028C8D00378472BC5D10230AE
:1022300001A9FFF7C6FE019B002BBEDB154A1B4917
:1022400053651B4801F0E1FD0023A5E701A9FFF755
:10225000B8FE2023057806009D43AED1300002A9C8
:10226000FFF776FF019B0600E918FF2902DC02A8B0
:1022700002F046FA002EA0D00135042DEED1BBE7C6
:10228000CC050010C38600004E730000D986000004
:10229000F2860000D8060010E6060010F4060010D2
:1022A0001E0700100207001010070010E58600004E
:1022B000E886000037B54C682378002B00D137BD85
:1022C0002000FFF769FE01A9FFF77BFE019B0400D8
:1022D000002BF4D0D8B2FF2B13DD00F0C5FA019B20
:1022E00005001812C0B200F0BFFA01900198002852
:1022F00002D02900FEF7EAF823785A1E9341E41829
:10230000DAE700F0B1FA00250190EFE70123064A71
:1023100010B511784B401370044900D104490548A9
:1023200001F073FD10BDC0469502001085750000D8
:10233000F9860000FD8600000123064A10B51178D9
:102340004B401370044900D10449054801F05DFD7C
:1023500010BDC0469402001085750000F98600008B
:102360000C8700000B0007B5586801A9FFF7D4FDE2
:10237000019B002B0CDC012301939623019A9B0007
:102380005343054A01990548136001F03EFD07BD1E
:102390001E2BF2DD1E23EFE7500200101C87000009
:1023A00010B50C4A1378013BDBB21370002B0AD036
:1023B000012B05D10849094A094801F026FD10BD45
:1023C0000849094AF8E7094801F01FFDFEF7CCF972
:1023D000F5E7C0463400001044870000F398000081
:1023E0004887000040870000767600006C87000078
:1023F00070B50400002C00D170BD642500210220BE
:10240000013D00F0D9FE002DF8D1013CF2E70000BB
:10241000F0B580250F4B6D001A6804262A431A6018
:1024200008220D4F0D491C683C401C6044B2002C32
:102430000CDA0C6834430C601C68013A2C434000F1
:10244000D2B21C60C0B2002AEDD1F0BD0C68B4431A
:10245000F1E7C046FC3F0150FFFEFFFFFC3F00508C
:102460000121044A10B513688B431360FFF7D0FFB6
:1024700010BDC046FC3F0250F0B583B072B60123D8
:10248000843001270600194D0193B0202B683400D9
:10249000BB432B60019B843C1843FFF7B9FF2B68BB
:1024A0000020BB432B60FFF7B3FF2B681020BB431A
:1024B0002B60FFF7ADFF2B68E020BB432B60FFF7DD
:1024C000A7FF2B683B432B6020780134FFF7A0FF68
:1024D000B442F6D1019B84342600002B02D162B6AF
:1024E00003B0F0BD00230193CFE7C046FC3F02508C
:1024F00010B5AC20FFF7B4FFAE20FFF7B1FFA52069
:10250000FFF7AEFF10BD70B50D000400012200F012
:1025100031FE29000122200000F078FE70BD10B5C8
:10252000AF20FFF79DFFA420FFF79AFF10BD10B565
:10253000AE20FFF795FF10BD10B50400F820FFF79F
:102540008FFF2000FFF78CFF10BD10B50400812025
:10255000FFF786FF3F202040FFF782FF10BD0000FD
:10256000202010B5064B1B781843FFF779FF0A208F
:10257000FFF73EFF034B1878FFF7E7FF10BDC0469B
:1025800035000010A7040010842210B5064B074840
:1025900019785200002903D0054901F04CFC10BD08
:1025A00001F06AFCFBE7C046A80400109E0300107F
:1025B0009602001010B584220021024801F05CFC54
:1025C00010BDC0469E03001010B5582204490548AE
:1025D00001F031FCB0220021034801F04DFC10BD98
:1025E0009E03001096020010EE020010014B1870BE
:1025F0007047C046A8040010002310B5074AD35600
:10260000002B07D0013B59B21B0601D4117010BD3D
:10261000002313700248FFF72FFFF8E7A60400100D
:102620009E03001010B508210120FFF76CFF022166
:102630000020FFF768FF00210220FFF764FF06215A
:102640000220FFF760FF03210800FFF75CFF032172
:102650000022080000F0DAFD00220621022000F02E
:10266000D5FD01220621022000F0D0FDFFF78CFFEE
:10267000FFF7C2FFA220FFF7F3FEA020FFF7F0FE56
:10268000C020FFF7EDFE0020FFF756FF0A20FFF7FE
:10269000AFFE4020FFF7E4FE2C20FFF7E1FE3220E2
:1026A000FFF7A6FE2E20FFF7DBFE3220FFF7A0FE8D
:1026B0002F20FFF7D5FE0A20FFF79AFEFFF750FF05
:1026C000FFF72DFF10BD0000030083280DD80F2950
:1026D0000BD88420CA085043C01807231940793307
:1026E0000B41024A115C0B43135470479E030010C8
:1026F000F0B5072580265B1885B0DBB2104F02903D
:1027000003920193019B994201D305B0F0BD84224D
:10271000CB085343029A30009B180A002A4010410C
:10272000039AC0B29446DA199C44634502DB013136
:10273000C9B2E7E714780133044314700132F4E7B7
:102740009E030010F0B587B005921E00DB7883422F
:1027500003D23778380007B0F0BDB4787268244BE4
:10276000041B00209A4216D103231F005C43A418C7
:10277000E318CDB20393EB19DBB20493002301936A
:10278000049BAB42E6D0082302930023009327E08A
:102790000233D21801301378A042F9DB5778941C29
:1027A000E6E7029B082B07D1039B9C42D2D02378FB
:1027B00001340193002302930122019B134206D0AE
:1027C000059B009A28009918C9B2FFF77DFF019B6D
:1027D0005B100193009B01330093029B0133029332
:1027E0007378009A9342DCDC0135EDB2C8E7C0464D
:1027F00087870000F7B505001F000C00160001F0E8
:102800005DFB2B180193019B9D4201D0832C01D9C4
:102810002000FEBD3B00210028783200FFF792FF28
:10282000024B01351B68C0182418ECE73800001073
:1028300000210122042330B50A4C0D5D854203D1ED
:1028400018011043C0B230BD013B002B04D101324E
:102850000433092A00DD002201312829EDD10020AE
:10286000F1E7C0466A9800003C2310B504098000D7
:102870001840011F00D52831621E0020032A06D807
:10288000242904DC0423024A1B1B5218D05C10BD0F
:102890006A98000070B505000024054B2900E05C33
:1028A000044B0134C01800F0D3FC0A2CF5D170BDE4
:1028B0006098000000400440F7B50E4E3468002CCC
:1028C00016D11020FFF7E6FF0B4D2B786F7818001C
:1028D000002239000193013400F04CFC0122390040
:1028E000019800F093FC02350A2CEED101233360ED
:1028F000F7BDC046AC0400109A980000F8B500255A
:102900000B4C2678677801223900300000F032FC49
:10291000013500223900300000F078FC02340A2D25
:10292000EFD10020FFF7B6FF0022024B1A60F8BD7E
:102930009A980000AC04001070B50500FFF7BCFFCA
:10294000002D09D001220721022000F013FC802174
:102950000F4A13688B4313600B21002000F02CFCFE
:102960000124002805D00B21002000F025FC444262
:102970004441002D09D000220721022000F0FAFB7B
:102980008023034A11680B431360200070BDC046CA
:10299000FC3F02500023F0B58BB006900120099354
:1029A0000791FFF7C9FF0400031E01D0182301247B
:1029B000089300232C4E0193377875780122290063
:1029C000380000F0D7FB00222900380000F01EFC80
:1029D000264B0293019B04330593022C1CD0029BCF
:1029E0009B790393029B0398DB791900049300F011
:1029F000E3FB00282AD101991D4AA3008A5C08A99B
:102A00005A500134019B01330193029B019A023B0E
:102A10000293059B9342E0D100222900380000F088
:102A2000A9FB01222900380000F0F0FB114B02360F
:102A3000B342C1D1002C06D00124069B089A1A602B
:102A4000079B099A1A6020000BB0F0BD0499039807
:102A500000F0B2FB0028CED00499039800F0ACFB44
:102A60000028C8D0CEE7C0469A980000929800008F
:102A70006A980000AE980000012210B510000B21EA
:102A800000F078FB00220B21012000F0BFFB0122A7
:102A90000221032000F06EFB00220221032000F03F
:102AA000B5FB10BD37B51021244A0500136801207D
:102AB0008B4313608023224A9B011168214C0B43F6
:102AC00013600B21002200F055FB00220B21012096
:102AD00000F09CFB9F211C4B1A688A431A601A68FD
:102AE0001A491A601A4B186804F0EEFA03028020A3
:102AF000184320602A000320022100F087FB0A20EF
:102B0000002D00D0012000F07FFDFF2223689343B9
:102B1000236022680F4B13430F4A2360136801930D
:102B2000019B002BFADA23680C4A13402360FFF75D
:102B3000A3FF01980004800D3EBDC04638820440CA
:102B40008080044000C001409840044000093D00DE
:102B5000B8040010800000012CC00140FFFFFFF806
:102B600010B50D4C2068002814DA00202060FFF713
:102B700099FF0A280BDC0120FFF794FFE02341387E
:102B8000FF385B00984202D8C03BFF3B2360FFF751
:102B900073FF206810BDC0463C00001010B5FFF761
:102BA000DFFF002801D1002010BD0020FFF77AFFD1
:102BB0000120FFF777FF011EF5D0024804F084FAE8
:102BC000F2E7C0462D47130010B5FFF7C9FF0028F4
:102BD00009D0FFF7E3FF00210300034AC00F9A4228
:102BE0004841024B186010BD34080000B0040010CA
:102BF0000222074B10B51A60064BA0321960064B33
:102C00001A70013258709A7000F0F0FD10BDC04685
:102C10001C06001008060010F40500100022064BE8
:102C2000023110B51960054B1A60054BA2321A70BB
:102C3000587000F0DBFD10BD1C06001008060010E7
:102C4000F405001070B505000E00032431002800C3
:102C5000FFF7CEFF0223FF33984202D0013C002C45
:102C6000F4D170BD70B505000E00032431002800BA
:102C7000FFF7D4FF0223FF33984202D0013C002C1F
:102C8000F4D170BD0A4B10B51B68002B0ED0094C57
:102C9000A31CA270140A5C70140C120EDA709C70E3
:102CA000FFF7E0FF831EFF3B5A425341180010BD5F
:102CB000B4040010F405001070B50E4C2468002C0C
:102CC00015D00D4C160AA270E670160C120E627129
:102CD000A371A21D26711C0A54701C0C1B0E94704B
:102CE000D370FFF7BFFF841EFF3C63425C412000AE
:102CF00070BDC046B4040010F4050010064B10B5BA
:102D00001B68002B05D0FFF79DFF831EFF3B5A4237
:102D10005341180010BDC046B4040010064B10B556
:102D20001868002807D007210220FFF78BFF023820
:102D3000FF384342584110BDB40400100E4B70B52B
:102D400004001868002813D0A11E062911D80725F1
:102D50006D1A072D04D009482A00091801F06BF8F4
:102D60002900E0B2FFF77EFF0238FF3843425841A6
:102D700070BD01204042FBE7B4040010F6050010CE
:102D8000012110B50800FFF75DFF0223FF339842D1
:102D90000FD10120084B1860084B1C78230706D080
:102DA0000323074A234001009370FFF75BFF2000D5
:102DB00010BD01246442FAE7B40400100C060010B0
:102DC000F405001010B5FFF7DBFF01210220FFF72B
:102DD00039FF0223FF3398420FD1084B1B787F2B1A
:102DE00006D9842207210220054B5204FFF764FF15
:102DF00004210920034AFFF745FF10BD0C0600100F
:102E0000020114008080808010B5002848D0802105
:102E1000254A13688B431360012324490A681A4228
:102E2000FCD00322224B1A6001230021214A1360A7
:102E30001160136011681942FCD01F4A1F491360CA
:102E400080230C685B0223430B60002804D180239D
:102E500015490C6823430B60194B196881421ED039
:102E60001860431E9841174B40421840164B11689A
:102E7000C01804F09FF8FA21144B89001860040070
:102E800004F022F91E23C8214343114A2000136095
:102E9000490104F019F90F4B186001F03BF810BD1F
:102EA000034B1860C0E7C046388204400C800440E1
:102EB0007080044074800440788004408080044026
:102EC0004000001000512502001BB700B80400109C
:102ED000C0040010BC04001010B500F03DF9134A06
:102EE000002113681B0B1B031360114A13681B0B93
:102EF0001B0313600F4A13681B0B1B0313600E4A5E
:102F000013681B0B1B03136001220C4B19600C4B45
:102F10001A6019601A6019681142FCD02322094B0B
:102F200000201A60FFF770FF10BDC04600800050FF
:102F30000080015000800250008003504080044017
:102F40004480044008800440014B024A1A60FEE7B6
:102F50000CED00E00400FA0570B500250B490C48A3
:102F600000F053FF0B4E300000F04FFF0A4CE268B8
:102F7000216833000948013500F047FF14340C2D57
:102F8000F5D1074800F041FF70BDC0464E73000008
:102F9000AE980000F19800002C9A0000C098000044
:102FA000CB980000F0B500253D4F04003B68280099
:102FB0008BB0AB425ED03B4B02941B6802A99B686E
:102FC000013098473B68002B02D1374800F01DFFC5
:102FD0000BB0F0BD01342378202BFBD0002B2FD079
:102FE000431C0193800002ABC450FF2D06D1019B0E
:102FF0001800022B45D1002526E01C002278002A6B
:1030000005D0631C202AF8D1002222701C00019BED
:10301000012B2ED10C26234D244B2B602B680298BC
:10302000196800F06AFF2B68002821D01433013E94
:103030002B60002EF2D131003000FFF78DFFC4E786
:103040000028BFD002281AD11949039800F055FF73
:1030500000280BD1134C17482368D96800F0D5FE1F
:1030600023681548196900F0D0FEABE7022006E09E
:103070001D7901982378002BE2D00828ABD1854236
:10308000E8D2084CC0B2236802A99B68984722681E
:103090000A4B92689A4295D00322094B1A7091E725
:1030A000CC050010C4040010F49800002C9A000015
:1030B00083730000ED980000ED860000A12300005E
:1030C0003400001070B50400154D0D281BD00CD82D
:1030D00008280CD00A2816D02100124800F095FECE
:1030E0002B685A1C2A601C7018E07F28F4D10E4B04
:1030F0002A689A4212D921000A4800F086FE2B68FD
:10310000013B2B600AE000232A680848137000F096
:103110007CFE054C2000FFF745FF2C6070BDC046CB
:10312000C805001000990000C8040010F1980000C4
:1031300010B500F01BFD002800D110BD00F0F4FC1C
:10314000FFF7C0FFF5E70000014B024A1A60704725
:10315000C8050010C80400104023044A11680B433E
:1031600013600122024B1A707047C04680800440F1
:10317000D00500100E4B70B51B7804000E00150032
:10318000002B01D1FFF7E8FF631E022B0AD8094B81
:103190002004C01801230268B340012D04D1134359
:1031A000036070BD0348F5E79A430260F9E7C04643
:1031B000D0050010008000500F4B70B51B78050043
:1031C0000C00002B01D1FFF7C7FF0020032D0BD807
:1031D0002800012303F0D0FE02090B0D074AA3408B
:1031E00010681840431E984170BD054AF7E7054A2C
:1031F000F5E7054AF3E7C046D0050010FC3F005054
:10320000FC3F0150FC3F0250FC3F03500E4B70B599
:103210001B7804000E001500002B01D1FFF79CFF66
:10322000631E022B0AD8094B2004C0180123026830
:10323000B340012D04D11343036070BD0348F5E78B
:103240009A430260F9E7C046D0050010FC3F0050E9
:10325000084B70B51B7804000D00002B01D1FFF75F
:103260007BFF182223689343236021680D43256068
:1032700070BDC046D00500103F224021044B1A60AB
:10328000044B3E3A1A60044A13688B43136070473C
:1032900024800440D8800440388204404021044AFD
:1032A00010B513688B431360FFF7E6FF10BDC046EF
:1032B0003882044009490A4A0B681A4080235B009F
:1032C00013430B600421074A13688B431360064BBA
:1032D0001A68064B1A6030BF7047C0460080034032
:1032E000FFF7FFFF10ED00E0388204403482044015
:1032F00010B500F041FAFFF701FB00210948FFF784
:10330000A7FF00210848FFF7A3FF00210748FFF7A8
:103310009FFF00210648FFF79BFF00210548FFF7AC
:1033200097FF10BD0840044000400440AC400440FA
:10333000144004401C40044010B50120FCF78AFFF3
:1033400010BD00008022124B10B5DA679218DA67C0
:103350008022D200DA6780225201DA6780221201CD
:10336000DA6780229200DA6700230121094A494284
:103370001360094A1160094A1360094A1360094A37
:1033800001331360084A1360FFF7D6FF10BDC04633
:1033900004E100E0048204400882044004C00040CC
:1033A0003CC0004000C0004000400140064A10B54B
:1033B000136801331360054B1868FFF725FDFFF70D
:1033C000C1FFC046C04610BDD80500104000001027
:1033D000F0B585B00C00019072B6FFF789FF554B30
:1033E000554D1A68554B1A60019B5A1E93413F2256
:1033F0005B429343524A9B18524A13600423524A39
:1034000011680B43136000232B60A3071AD04F4AA7
:103410004F4913680B40136029684E4BA20700D434
:1034200082E0EC2252010A432A6080221A6092183C
:103430001A608022D2001A60802252011A60802213
:1034400012011A60019B002B53D00024424B434FC2
:10345000434E3C601C60434B21001C60424B3000DB
:103460001C60FFF7F5FE220009212000FFF782FE15
:10347000220009212000FFF7C9FE80213B4A3C4879
:1034800013680B4313600722336876399343336024
:103490003368053A13433360019B584303F08AFDB8
:1034A0000322344B34491860344B1C60344B1A608F
:1034B000344B1A680A4080211A601A680A431A605D
:1034C0008023244A21499B0013600A681A430A603A
:1034D0002A68022113432B6001232B4A13602B4AD5
:1034E00011602B4A13601460136011681942FCD0FC
:1034F0003B6001220021274B52421A60264A136882
:103500000393264B196062B630BFC0460399126818
:10351000914207D101221A60214B1868FFF774FC11
:10352000FFF710FF05B0F0BD802212010A432A60A8
:1035300085E7C04638820440048204403482044057
:10354000FF1800003082044010ED00E000820440CB
:103550007FE2FFFF00E100E00400014004C0004002
:1035600064400440044001400480014080800440E5
:10357000841E000018C000400FF0FFFF08C000408C
:1035800014C000403CC0004078800440708004407B
:103590007480044008820440D8050010D40500104F
:1035A0004000001010B5FFF713FF10BD074B1A685D
:1035B000013203D106490A6801320A601A680132F1
:1035C0001A60044A1368013313607047E80500105D
:1035D000E4050010E005001080235B0498420AD245
:1035E0000023054A01381360044A1060044A13603E
:1035F0000722044B1A607047E805001014E000E051
:1036000018E000E010E000E00B4A1368002800D149
:103610000130C143994209D2591C081811689942D6
:1036200000D2704711688842FCD8F7E71168C91AC0
:103630008142FBD3F5E7C046E8050010014B18684E
:103640007047C046E80500100122034B1A60034A88
:10365000136801331360704700C00040EC05001090
:103660000122034B1A60034A136801331360704749
:1036700000000140F0050010002803D10122044B96
:103680001A6070470128FCD1024B1860F9E7C04668
:1036900004C0004004000140002802D1044B18601F
:1036A00070470128FCD10022024B1A60F8E7C0469F
:1036B00004C0004004000140002805D1044A022350
:1036C00011680B43136070470128FCD1014AF6E7EB
:1036D00004C000400400014010B5002900D1144985
:1036E000002810D18023134A146823431360032257
:1036F000114B1860114B1960114B1A608022114B4D
:1037000052021A6010BD0128FCD18023094A5B00D7
:1037100010680343136000220B4B1A600B4B0332FB
:1037200019600B4B1A608022064B9202E9E7C046F3
:10373000FFFF000080800440EC05001018C000402E
:1037400014C0004000E100E0F00500101800014046
:1037500014000140802210210820064BD205116080
:10376000186080235B011068084202D0013B002BE7
:10377000F9D17047180000408022164B120210B594
:10378000DA676C22144B15481A60154B1968014012
:1037900019601A6804211A60124B1A6802401A60F4
:1037A0001A6800201A600122FFF7E4FC01220421BC
:1037B0000020FFF72BFD012205210020FFF7DAFC96
:1037C000012205210020FFF721FD0022064B1A608F
:1037D00010BDC04604E100E018000040F8FCFFFF07
:1037E000304004403440044004800440F8B50023D5
:1037F000164A174C202123601360164A136080225A
:10380000D2051160144A2168012907D0934203D1DF
:10381000FFF7A0FF0020F8BD0133F4E79342F7D093
:1038200000250E4F3E68013E2368FF2B01D920681A
:10383000F1E73B68B34204D03E68FFF7FFFE0A3071
:103840000500FFF7FBFEA842EED1E1E720060010DD
:103850000406001024060010FF0F000028060010C8
:103860000122034B1A60034A136801331360704747
:10387000004001403406001070B50124164B174A71
:103880001C6013681B191360154B1A68002A13D0AB
:103890001A68144D013A1A601E68002E0DD02100DE
:1038A00020002A68FFF7B2FC2B680221E31A2B6084
:1038B00020002A68FFF7AAFC70BD1B6821002B605E
:1038C00020002A68FFF7A2FC022120002A68FFF7E7
:1038D0009DFC054B1E60EFE700800140380600109C
:1038E0002C0600103006001004800140002803D18F
:1038F0000122044B1A6070470128FCD1024B18606A
:10390000F9E7C0460440014004800140002802D18C
:10391000044B186070470128FCD10022024B1A604A
:10392000F8E7C0460440014004800140002805D16A
:10393000044A022311680B43136070470128FCD12D
:10394000014AF6E7044001400480014010B5002818
:1039500011D18023124A9B00146823431360032271
:10396000104B1860104B1960104B1A608022104BDE
:10397000D2021A6010BD0128FCD18023084ADB0066
:1039800010680343136000220A4B1A600A4B03328B
:1039900019600A4B1A608022054B1203E9E7C04602
:1039A000808004403406001018400140144001405B
:1039B00000E100E03806001018800140148001404A
:1039C0000E22174B10B51B681340062B12D1154B56
:1039D00090321B68134205D0134ADBB25360134B7D
:1039E0001B6810BDDB07FCD5104B1868C0B200F097
:1039F000ACF8F6E7042BF7D00C2B05D10A4AF433C8
:103A000051680B435360ECE7022BEAD1054B1A686F
:103A1000054B920602D500229A60E2E70122FBE7FD
:103A200008800040148000403C06001000800040E8
:103A3000004870473C060010F7B58022002107259A
:103A40002A4B2B4C9203070001912000DA67902249
:103A500000F012FA019B274EA360274B1A68AA4375
:103A60001A600122196811431960244B1968A9438F
:103A70001960196811431960802321495B010868A6
:103A800003430B601F4B1A60823232601E4A126879
:103A900019681E4B1868504303F08CFA390000096E
:103AA00003F088FA10221A4B1A491A60030A0B60B5
:103AB0000323194FC0B2386060203360174B1D607C
:103AC000174B1A6801921A680240602AFBD15F3ACC
:103AD0001868104207D122708022124B92031A609C
:103AE00005230B60F7BD38680190F1E704E100E0C1
:103AF0003C0600100C800040A4400440A840044054
:103B0000808004409880044078800440B80400100D
:103B10002880004004800040008000400880004071
:103B20001480004000E100E010B5FFF781FF0200C3
:103B3000837BC318D87B937B0133DBB293735BB277
:103B4000002B01DA0023937310BD10B50400FFF7BA
:103B50006FFF437BC318DC73437B0133DBB24373DA
:103B60005BB2002B01DA0023437310BD10B5FFF7E1
:103B70005FFF0300807B5B7BC01A431E9841C0B28D
:103B800010BD70B504001D0000202E5C2318002E0F
:103B900009D1121AD518EC1A002C07DCD343DB1715
:103BA0001A40101870BD26540130EEE71970013329
:103BB000F1E7F8B5541E0F001E00050023000100B8
:103BC000092E16D90A21300003F0F4F9220003006F
:103BD00039002800FFF7EDFF04002D1830000A21FE
:103BE00003F06EFA30312970601CF8BD0F70013B94
:103BF0000131002BFADC0020824200DD20002D186C
:103C0000002A00DC0122541EE8E7F7B50E00D917A0
:103C10005F18040001934F40551E092F17D90A2140
:103C2000380003F0C7F9019A0300002A00DA434282
:103C30002A0020003100FFF7E8FF050024183800B3
:103C40000A2103F03DFA3031681C2170FEBD019B52
:103C5000002B00DA951E23006119CA1A002A0CDC19
:103C6000E843019AC017054064196B1C002AE6DA84
:103C70002D221D0022700134E1E71E700133ECE7B4
:103C8000F7B51E00089B1400013A1F090500130038
:103C9000002F11D033000097FFF7F2FF2D180F23EC
:103CA000089F1F40FAB2092F12D830322A70013013
:103CB000FEBD0170013B0130002BFADC0020844284
:103CC00000DD10002D18201E00DC01200138E6E781
:103CD000002E01D03732E9E75732E7E7F0B50500AB
:103CE0000F001C0085B0002801D0002303700026BF
:103CF0001378002B00D16DE0B74204D80023013DBA
:103D00002B70013E32E0252B04D001322B7001369E
:103D10000135EDE75178252902D129700232F6E705
:103D2000931C0393302902D02021531C0393039B3F
:103D30001B782D3B5A425341039AD3180022039318
:103D4000039B1B7818003038092812D99019B84203
:103D500001D9BA1BD2B2692B1FD013D8632B35D02F
:103D6000642B1AD0582B2DD001267642300005B096
:103D7000F0BD0A2042439A18039B303A0133D2B275
:103D80000393DDE7752B11D0782B14D0732BEBD177
:103D9000280008CCFFF7F5FE03E0280008CCFFF769
:103DA00034FF039A2D1801323618A1E7280008CCF9
:103DB000FFF7FFFEF5E708CC009300232800FFF78C
:103DC0005FFFEEE708CC00930123F7E708CC012062
:103DD0002B70E6E7B74200D890E72B70C6E710B526
:103DE00013000A006421FFF779FF10BD00B59BB0F6
:103DF0000A00010001A8FFF7F2FF632800DDFEE7DB
:103E000001A800F0ADF81BB000BD0FB407B504A9C0
:103E100001C90191FFF7EAFF03B008BC04B01847DD
:103E20000EB403B503AA02CA0192FFF7D8FF02B08D
:103E300008BC03B0184770B506000E4303253400D4
:103E400003002C402E420FD1AA420DD90B59035129
:103E50000434131B032BF9D80324131F9B080133CD
:103E60009B00C9182240C3180024A24200D170BD93
:103E70000D5D1D550134F8E770B5830704D00300CC
:103E80009A189A4217D170BD0300032AF8D90C047E
:103E90000B0623430B430C0223430400861808C47B
:103EA000351B032DFBD80324131F9B0801339B00F4
:103EB000C3182240E4E719700133E2E70300002051
:103EC0001A5C002A00D170470130F9E70023CA5C70
:103ED000C2540133002AFAD1704770B500230400A0
:103EE0009A4201D1002007E0E55CCE5CA81BB542F8
:103EF00002D10133002DF3D170BD0200002310B5B3
:103F0000D05CCC5CA04201D0001B02E00133002851
:103F1000F6D110BDFA21094B10B51868890003F0DD
:103F2000D3F8FFF759FB96200002FFF785FD01202B
:103F3000FCF790F9FEF746FF10BDC046B80400102C
:103F400010B5FEF7C9FFFFF707F9FFF7A7F9FEF76E
:103F500069FBFEF719FBFFF7DDFFFFF7F5F810BD72
:103F600010B504002078002800D110BD0134FCF702
:103F7000C7F9F7E770B50500441E0D35A54200D11D
:103F800070BD29780248FFF740FF013DF6E7C046C3
:103F90008774000070B51748FFF737FF164D2800EB
:103FA000FFF7E8FF154C42212000FFF72EFF1448D1
:103FB000FFF7E0FF43212000FFF727FF1148FFF73D
:103FC000D9FF1148FFF721FF1048FFF7D3FF104832
:103FD000FFF71BFF0F48FFF7CDFF4E212000FFF733
:103FE00014FF0D48FFF7C6FF696D0C48FFF70DFF82
:103FF00070BDC0461C9B0000D8060010229B00002C
:10400000E6060010F4060010299B00001E070010B1
:104010002F9B00000207001010070010359B0000C6
:104020000A23021153430F2210401818704770B52D
:104030000A21050003F048F80A210401280003F0D2
:1040400029F92000084370BDC12210B55200022199
:104050000E20FEF717FE0122014B5A7110BDC0461B
:10406000CE06001010B5084C6379002B01D1FFF784
:10407000EBFFA2792379520001211A430C23080097
:104080001A43FEF7FFFD10BDCE06001010B5074C19
:104090002379002B08D16379002B01D1FFF7D4FFDE
:1040A00001232371FFF7DEFF10BDC046CE060010CE
:1040B00010B5054B1A79002A05D000221A711A7220
:1040C000DA70FFF7CFFF10BDCE06001010B501214A
:1040D0000220FEF713FE064B040018787F231840D9
:1040E000FFF79EFF034B5870DC71200010BDC046E7
:1040F0000C060010CE0600100122014B9A7070478A
:10410000CE0600100022024B9A701A727047C04609
:10411000CE06001010B5FFF7D9FF094B09499A7870
:10412000002A03D01A7A012A02D801321A7202E058
:104130000868054A10600022DA700A6010BDC046A7
:10414000CE060010E0050010DC05001010B5FEF7EB
:1041500017FE0C2203001340104203D0024A1178CC
:104160000B43137010BDC046CE06001010B5FFF70C
:10417000EDFF044C23785B0701D5FFF7CBFF00234D
:10418000237010BDCE06001010B50020FEF7D4FB42
:10419000002801D0FFF7EAFF10BD0000002310B592
:1041A000044CE371FFF7F0FFE379002B01D1FFF737
:1041B0008DFF10BDCE06001010B50921084803F090
:1041C0006FF8FA22074BD2001A80FFF7E7FF0022B0
:1041D000054B1A60FA22054B92001A6010BDC046CA
:1041E000CE060010CC060010E0050010DC05001023
:1041F00010B5FFF7C9FF002010BD704710B5FFF7DD
:1042000057FF10BD70B51D4C0D0061782378A27862
:1042100009021943E378120411431B06184A0B43A1
:1042200013401A0A237062701A0C1B0EE370637934
:104230002179A2701B02134A0B43134023711B0AFE
:1042400006006371A079FFF7EBFE0F4B1B881B186C
:1042500033806079FFF7E4FEB070E078FFF7E0FEAE
:10426000F070A078FFF7DCFE28706078FFF7D8FECA
:1042700068702078FFF7D4FEA87070BD0C0600109F
:104280007F7F3F3F071F0000CC060010F0B58DB0C8
:104290000400FEF743FD002805D120001249FFF776
:1042A000BFFD0DB0F0BD0AAE0BAD29003000FFF729
:1042B000A9FF33880793F378B77808932B7809938D
:1042C0000A4B6E781879AD7800F0D2F8099B04900B
:1042D0000193089B20000093079A3B000449039533
:1042E0000296FFF79DFDDCE7419B00000C060010E5
:1042F000469B000070B505000E001400FEF70EFD91
:1043000000280AD028003100FFF77CFF201E03D0D0
:104310000020034B1B79236070BD01204042FBE766
:104320000C060010F7B504880E000500642120007B
:104330000092019302F0C4FE114B8FB2E41B1C806B
:10434000B078FFF774FE0F4CA0707078FFF76FFE27
:10435000E0703078FFF76BFE2071E878FFF767FEBA
:10436000009B6071A371A878FFF761FEE0713800CF
:10437000FFF75DFE20720198FEF7E0FCFEBDC0462F
:10438000CC060010F405001010B50223FFF7CAFF99
:1043900010BD431E984110B5420101210020FEF7D7
:1043A00071FC10BD70B5040001200D00FFF7F1FF96
:1043B000200000F085F8072102F06CFF20000A00C1
:1043C0002900FFF7E1FF96204000FFF71DF90020CC
:1043D000FFF7DFFF70BD000073B50400FFF776FE46
:1043E000002801D1002076BD1D4D6E780A20FFF710
:1043F0000BF9FFF76BFE0028F4D06B78B342F5D0D1
:10440000FEF78CFC0028EDD001A96846FFF7FAFE04
:10441000684600F055F8050001A800F031F8114B8E
:1044200004199C420DD90122E3171343ED18694684
:10443000280000F077F80C4AE31713400B4A9B184A
:10444000E418200001A900F025F82800072102F057
:1044500021FF68460A0001A9FFF796FFC3E7C0469F
:10446000CE0600107F51010000A3020080AEFEFFC7
:1044700007231840014B8000C0587047849B000000
:104480003C23020000785178584340184343907809
:104490001818704770B50C003C21050002F0FAFEB8
:1044A0002800A1703C2102F00FFE3C2102F0F2FE38
:1044B0006170E1212800090102F006FE207070BD44
:1044C00070B5962283780688050000205201B61840
:1044D000010002229A424141761A022B00D80C3088
:1044E000C0189923033858436E240521023002F086
:1044F000EBFD6421FF3474430419B01024184942C1
:10450000300002F0E1FDC82124184900300002F01B
:10451000DBFD034B2018EC78C018001970BDC046B5
:10452000D382FFFFF8B5214B050080000E00C018B4
:104530001F4902F0C9FD032703007B43D817384009
:10454000C01880101B4B2D18AD00ED1828001A491B
:1045500002F0A0FECC173C4064180237A4107C4344
:1045600002342000992102F095FE0800390002F083
:10457000ABFD0130F0709921200002F0A5FD0C2167
:10458000023002F087FE0131C8B20E21B070081A65
:10459000023902F099FD08490400280002F094FD58
:1045A000064BC01824183480F8BDC046652F04009F
:1045B000B13A02004F150000B505000094EDFFFF71
:1045C000012210B511001000FEF720FE0122022189
:1045D0001000FEF71BFE012100220800FEF7CAFDB5
:1045E000002202210120FEF7C5FD0120FFF78EF910
:1045F00010BD000070B50D00072101240600174B07
:1046000020001A688A431A601A6822431A60144B01
:104610001A688A431A601A68210022431A6022002D
:10462000FEF7A8FD220002212000FEF7A3FD0D4B9E
:104630003100186802F048FD01002000FFF786F9FC
:104640002000FFF773F9084E20003560FFF74EF9A0
:104650003368002BFCD1FFF7B3FF70BD7C400440F2
:1046600080400440B80400102C0600100300F8201D
:104670000A00C000890101405005800E0143F82066
:104680000002024011430A22514330B5CC101A19DE
:104690001000EB3055780078EA32684012781B5DE4
:1046A0000002104358400723194008418005800D3F
:1046B00030BD7047C023010010B55B01984201DB9B
:1046C000024BC1180248FFF7D1FF10BD00F8FFFFF1
:1046D000BA9A00000723020010B50F245943074B74
:1046E0009C31C9180E320B78234003700B780131CE
:1046F0001B09437002309042F5D110BDD80600105E
:1047000007230200594310B5064B9C31C9180E32DD
:10471000437804781B01234302300B70013182423D
:10472000F6D110BDD806001070B5B64D1726EB6E49
:1047300086B05A1E93416E443370B34BEA58D0068C
:10474000400F0138062808D802F016FC4431043620
:104750003C3F42000D23002404E06B6E16339B00A7
:104760005C59230050111F283BD802F019FC35007A
:104770003F00440048004E00560059005F006300AF
:1047800069007800830090009F00AC00B700C4006F
:10479000D100DF00EC00FD00FB000A011101160151
:1047A00023012E01330137013D01410145016B6EAB
:1047B00016339B00EB58CEE7AC6DEB6D9C42D1DD20
:1047C0000D23CFE702231C00CCE70C230324C9E709
:1047D0000D23F8E70223BEE7191B0131281902F067
:1047E0005FFD01203378EB6606B070BD191B87486A
:1047F00001312018F3E7191B85480131F9E7220040
:104800008249280001F0C5FAEBE71A1B7F48013204
:1048100029192018FFF70FFBE3E722007C49F0E796
:104820007A491A1B7A4801326118F2E72200784966
:104830007648E7E776491A1B013261182819E9E73B
:10484000296E0A22002900D1063200932300029229
:104850006E4A01962900280001F0A5FAC1E7296EE9
:104860000A22002900D1063202920093684A2300EE
:104870000196EFE70122296E32700932002900D13A
:10488000063202920093002223000196E2E7296E8D
:104890000A22002900D106320093230002925B4ACB
:1048A00001962900280001F0A9FA9AE70122296E51
:1048B00032700932002900D10632029200930022A0
:1048C00023000196EDE7296E0A22002900D1063265
:1048D000029200934E4A23000196E2E7296E0A22D3
:1048E000002900D106324A480292009302002300B8
:1048F00001960100B0E7296E0A22002900D1063294
:104900004348029200930200230029000196A3E786
:104910000122296E32700932002900D1063202923A
:104920000093002223003A480196E2E7296E0A220A
:10493000002900D10632364802920093020023007B
:1049400029000196AFE70122296E32700932002951
:1049500000D106322E48029200930022230001006B
:104960000196A0E701223270296E0A22002900D1A7
:10497000063227480292009302002300002101968C
:1049800091E7220000212148009601F099FA28E7DA
:10499000220000211E480096F7E7296E0A2200290E
:1049A00000D10632009323000292194A0196290091
:1049B000002078E7296E0A22002900D106320292EF
:1049C0000093124A23000196F1E72200002100968D
:1049D0002800DAE722000E490096F9E71A002100C4
:1049E000280001F084FAFCE61A0021000748F8E7E5
:1049F0001A0021000648F4E71A002100280001F0FF
:104A000087FAEEE6D8060010C4070000E60600109C
:104A1000F4060010064B10B519001A1DD46F0831AA
:104A2000CC67D96FD1679A6F9867DA6710BDC046B7
:104A3000D8060010064BDA6F986F9A671A1DD16F6F
:104A400008335967D96FD1670022DA677047C046CB
:104A5000D8060010F8B5134D2F008C373B68581C52
:104A6000FFF728FEF923DB00E8500123AA6E0400BB
:104A700003409A4213D10C4BEE58830703D4386895
:104A80000230FFF7C7FFFF202B000122A401000224
:104A90000440B6108C3334431C60044BEA500220AF
:104AA000F8BDC046D8060010C4070000AC070000DF
:104AB0000D4B0E490120CA5810B5D3059B0E940525
:104AC0000ED5403B8C6E92100240944206D10A00F3
:104AD0008C321468E3181360054BC850012010BDD8
:104AE000002BEFD10300EDE7C4070000D80600104B
:104AF000AC07000010B5084B5A1CD07F9A1CD27F1F
:104B000000011202104303331A7FDB7F10431B03A3
:104B10001843FFF77FFF10BDD806001010B5FFF750
:104B200089FF0F240323044A01002140D15401339B
:104B30000011072BF8D110BDF406001010B5FFF7D7
:104B400079FF044B01211A008C321060024A9950FF
:104B500010BDC046D8060010AC07000010B5064CCA
:104B6000A36E002B07D0FFF765FF230001228C33D3
:104B70001860024BE25010BDD8060010AC070000D0
:104B800010B5064CA36E002B07D1FFF753FF23008F
:104B900001228C331860024BE25010BDD806001081
:104BA000AC0700000121054B054A10B5D150054B5B
:104BB0001B68002B00D0984710BDC046BC07000002
:104BC000D8060010AC0E00100020144B144A70B52B
:104BD000985004329A5882421AD0F622D20099583C
:104BE000814214DD012909D1F721C9005C588442B2
:104BF00004D058500A210B4D99505C51F621C90040
:104C00005A58032A01DD0120D866013A5A5070BD76
:104C1000054B1B68002BFAD09847F8E7D806001020
:104C2000BC070000B4070000AC0E0010F822094BCE
:104C3000D2009A58002A04D0F622D2009A58002AAC
:104C400007DD0F21044A9A58013311401211997758
:104C5000DA777047D8060010B4070000044A537F83
:104C6000917F1B0109020B43117F0B435367704770
:104C7000D80600100B00093B30B5012B0BD80023E0
:104C8000074AD55CC45CA54206D0064A064B0839E3
:104C9000D0580143D15030BD01330E2BF1D1FAE78A
:104CA000F4060010D8060010A407000010B508296B
:104CB0000FD0192908D1082342781A4205D00022C2
:104CC00002704370FFF71CFD10BD0F230370083BFB
:104CD000F7E70200030000240E321C7001339342F8
:104CE000FBD1EFE730B5114B85B05C6F002802D0E7
:104CF0000F22944304430E4D5C67FF2C05DD0E210B
:104D0000280002F0CDFA05B030BD21006846FFF75B
:104D1000E1FC21006846FFF7C9FF00236A46D25C28
:104D2000EA5401330E2BF9D1EDE7C046D806001046
:104D3000F40600101FB50F22104B5C6F9443044320
:104D40005C67082C18D0FF2C16DC21006846FFF7A2
:104D5000C1FC21006846FFF78DFF00230849684623
:104D6000CA5CC25401330E2BF9D12100FFF79EFF1C
:104D700021006846FFF7C4FC1FBDC046D8060010DE
:104D8000F40600101FB50E4C616F082917D0FF29DB
:104D900015DC6846FFF79EFC616F6846FFF76AFF07
:104DA000002308496846CA5CC25401330E2BF9D16E
:104DB000616FFFF77BFF6846616FFFF7A1FC1FBDC6
:104DC000D8060010F406001010B50D4C631CD87FF7
:104DD000A31CDB7F00011B021843E37F1843E31C85
:104DE000DB7F1B031843FFF765FC0F220300134012
:104DF00023770311134000126377A07710BDC046DC
:104E0000D8060010024A536E16339B00D0507047EC
:104E1000D806001004494A6E1632920053581B1AE5
:104E20005A425341CB667047D8060010054A536E6C
:104E300016339B009958013901D4995070470D21C0
:104E4000FBE7C046D8060010064A536E16339B0097
:104E50009958481C0D2901D098507047002199504D
:104E6000FBE7C046D80600100F4B5A6E1632920070
:104E7000D05819180A7F0C2804DC497F09010A431D
:104E80005A657047F520094912015958800081423E
:104E900005D007480140B7208000814202D1596DFA
:104EA0000911ECE7197FEAE7D8060010CC070000EB
:104EB000FFFEFFFF224B30B55A6E16329200D258D9
:104EC0000C2A05D1F5211F4889001858884204D0C2
:104ED000FA21C900595800290DD00F20596D9A1890
:104EE00008400C1150771477FF220901114021432B
:104EF0001877596530BD0F25586D041105400C2AEF
:104F000003DC9B181D775C77F4E70E4A9958F5226D
:104F10009200914205D00C4A1140B7229200914272
:104F200008D11A00FF212932157002010A402243DC
:104F30005A65DFE71A00293214701D77DAE7C04698
:104F4000D8060010CC070000FFFEFFFF0F21254B05
:104F500070B55A6E586D16329200D2580140001149
:104F60000C2A05D1F524204DA4005D59A54204D09A
:104F7000FA24E4001C59002C0CD0551C5D192C7F20
:104F80009A18167F240134435C651C7F2C771077B8
:104F900019770CE0C9B20C2A0ADC551C5D192C7F6C
:104FA0009A18167F2401344328775C65117770BD09
:104FB0001D00F5260C4A29359C582A78B6001201A6
:104FC000B44205D0094E3440B726B600B44204D1ED
:104FD00002435A6529331970E9E71C7F2870224380
:104FE0005A65D5E7D8060010CC070000FFFEFFFF8A
:104FF00010B50E2202490348FEF71DFF10BDC04642
:10500000F40600101007001010B50E2202490348E4
:10501000FEF711FF10BDC04610070010F406001087
:1050200010B50D2300220249024800F0B2FE10BD67
:1050300010070010F406001010B50E2202490348B4
:10504000FEF7F9FE10BDC046F4060010020700107E
:1050500010B50E2202490348FEF7EDFE10BDC04612
:1050600002070010F406001010B50D2300220249BB
:10507000024800F08EFE10BD02070010F40600107A
:10508000024B181846300278DA667047D8060010CE
:10509000044B002219009A6408314C33CA871A80E5
:1050A0007047C046D8060010C21C431E002010B531
:1050B00004499A4200D110BD8C5C40002043013A63
:1050C000F7E7C0461E07001030B50124054A0B1D46
:1050D000994200D130BD05002540555440100131A2
:1050E000F6E7C0461E07001070B50020FFF7DCFF92
:1050F0000500084C0021207FFFF7E6FF25770420FC
:10510000FFF7D2FF05000421607FFFF7DDFF657721
:1051100070BDC046D806001010B50020FFF7C4FFD0
:10512000034C20770420FFF7BFFF607710BDC04617
:10513000D806001010B5054C0021207FFFF7C4FFF2
:105140000421607FFFF7C0FF10BDC046D8060010E5
:1051500010B50A4C23008C3318680130FFF7AAFA07
:10516000F923DB000F22E0500300134023770311E3
:10517000134000126377A07710BDC046D806001018
:1051800010B50E21054802F08BF80E21044802F0FC
:1051900087F80E21034802F083F810BDD8060010EE
:1051A000E6060010F40600100022054B197F18785F
:1051B00001320143197701330E2AF7D17047C046F7
:1051C000D80600100022054B187F197801320140E3
:1051D000197701330E2AF7D17047C046D806001060
:1051E0001FB500230A4A6C461118097F0130195572
:1051F0000D2800DD002001330E2BF4D10023054AD9
:105200006946C95CD15401330E2BF9D11FBDC0468C
:10521000D8060010F4060010074A10B5536E163376
:105220009B0099584C1E51189C500877002C01DAAD
:105230000D21995010BDC046D8060010034B002226
:105240001900983394310A601A607047D80600102C
:105250000122034B943319684A401A607047C046D4
:10526000D8060010074B002219008C310A6001217A
:105270001A67054A99501A009432126851424A41FD
:10528000DA667047D8060010AC07000070B5874B8F
:10529000874DEC58874BA210A41119570F231340C8
:1052A000581E0E283DD801F067FE0810171E223C3C
:1052B000283C3C2E3C3C3C323600002931DB0022AD
:1052C000691846310A70180070BD002929DB0123D6
:1052D000691846310B70F6E7002922DB0800FFF75A
:1052E000CFFE0123EFE72000FFF796FFF9E7002943
:1052F00017DB0800FFF78EFDF3E7002911DB08003C
:10530000FFF780FDEDE72000FFF714FDE9E720003F
:10531000FFF7E8FCE5E7002903DB0800FFF760FF83
:10532000DFE7982A00D19CE063DC382A00D186E0D0
:105330003DDC1C2A00D179E029DC162A70D021DC62
:105340000123002ABFD0023B0C2ABCD1012398358F
:105350002B60B8E7D63A1000222A15D801F00CFECF
:105360009014931414149614141414141414141480
:1053700099149C1414149F14141414A2ACAF14B2F6
:10538000B5B8BB00182A4ED001235B429BE72C2AFC
:1053900052D007DC262A4CD0282AF5D100236B6690
:1053A000013390E7362AEFD1FFF7D0FD99E7662A5F
:1053B0004ED00FDC562A48D007DC3C2A42D04C2A7B
:1053C000E2D1FFF7C5FE02237DE75C2ADCD1FFF7BF
:1053D00091FB86E7762A41D006DC682A3BD06C2A0E
:1053E000D2D1FFF79BFB7CE7882ACDD1FFF71EFCCB
:1053F00077E7F82AC8DCD52AACDCBC2A3AD008DC2E
:10540000A82A31D0B82A32D09C2ABDD1FFF726FC79
:1054100067E7C82A31D0CC2AB6D1FFF7D5FC60E7C0
:10542000FFF722FD5DE7FFF71DFF5AE7FFF7E0FDFD
:1054300057E7FFF73FFD54E7FFF7E6FD51E701238C
:105440006B6640E7FFF7ECFD4BE7FFF7F5FD48E73C
:10545000FFF7FEFD45E7FFF793FE42E7FFF704FE87
:105460003FE700232B669BE701232B662BE7FFF723
:10547000E5FE36E7FFF786FC33E7FFF7E9FE30E7A6
:10548000FFF758FE2DE7FFF769FB2AE7FFF78CFED1
:1054900027E7FFF741FE24E7FFF772FB21E7FFF75D
:1054A00091FE1EE7FFF7F4FD1BE7C046C4070000AE
:1054B000D8060010A4D70000FFF774FB11E7FFF730
:1054C00083FB0EE7FFF7B2FC0BE7FFF70DFE08E7E3
:1054D000FFF7BAFC05E7FFF731FB02E770B51D4C9B
:1054E0001D4D1E4B6259E25023008C331868FFF7A4
:1054F000E1F8E36E6051A3660023194DE366635142
:105500000333184002281FD0984220D0012818D019
:10551000FFF7BCFE00280CDD6359002B04D12200EC
:105520008C3213681B1813602200903213681B180A
:105530001360FA22D200A358002B01D0013BA350E4
:1055400070BDFFF787FAE5E7FFF7EEF8E2E7FFF750
:10555000AFFADFE7D8060010C4070000CC07000050
:10556000AC0700000122034BDA66034A9A830F223C
:105570009A777047D80600100F0F000070B5F42519
:10558000074CED0066592000064901F089FE66517E
:10559000FFF7E8FF0123044A6366A35470BDC046C9
:1055A000D8060010D40700009C07000070470000D8
:1055B00030B50D4D049C28600C4801600C490A6010
:1055C0000C4A13600C4B039A1A600C4B0C4A1C607B
:1055D000F423DB00D4500B4B0B4A1A600B4B0C4AE4
:1055E00013600C4A136030BDB40E0010CC0E0010D6
:1055F000E80E0010D40E0010F00E00104400001051
:10560000D8060010AC0E001079570000AD55000010
:10561000BC0E0010EC0E0010014B18607047C04625
:10562000C80E0010084B10B51968084A002906D1A9
:10563000074C24682160106001221A6010BD1168B7
:105640008842F8DA0800F6E7C00E0010C40E001019
:10565000C80E0010034B1B68002B01D1024A1360D7
:105660007047C046B80E0010C00E001070B51A4D3D
:105670002B0098331B68002B0DD0184B1C6801239E
:105680001C40F523DB00EB58A34208D1144BEB5828
:10569000002B10D170BD2B0094331C68F1E7002C57
:1056A0000BD1002BF6D00F4B1B68002B0FD0210025
:1056B000200098470BE0002CECD00A4B084E1B68EA
:1056C000002B02D02000A95998470023AB51F523A5
:1056D000DB00EC50DEE7C046D8060010B00E00102C
:1056E000A4070000B40E0010054B10B51B68002B7A
:1056F00004D00449044A01208958984710BDC04687
:10570000B40E0010D8060010A40700000023F821F2
:10571000054AC9001370054A5350054953500431D6
:105720005350044A13707047D10E0010D806001071
:10573000B4070000D80E0010084B1860084B196021
:1057400000280AD001230021064A1370064A11706E
:10575000064A07498850074A13707047DC0E00104C
:10576000E00E0010D10E0010D00E0010B4070000A3
:10577000D8060010D80E00102C4B73B51A682C4BAD
:105780001168186881421AD00021009101911268B5
:105790001A60284B1B688B4202D0684601A99847C3
:1057A000254900980C68019A244BA04202D11C683C
:1057B000944202D00125224C257008601A60214CC9
:1057C000214BE358002B10D000231D49CB56002B52
:1057D0000AD000221D4B9A56012A05D100220A70D8
:1057E0001B490A7002321A7073BD134B174D1868AB
:1057F000002807D00023EB56002B03D10F4B19686C
:10580000FFF79AFF0023EB56114E022B08D100231D
:10581000104A3370A3502B700023F356E366E3E77E
:10582000002BF9D00A20FFF7FDFEF5E7D40E00109B
:105830004C000010CC0E0010DC0E0010E00E00102A
:10584000D00E0010D8060010BC070000D80E0010C3
:10585000D10E0010B4070000F82370B5054CDB0032
:10586000E358002B05D1E56E034AA350FFF784FFF0
:10587000E56670BDD8060010BC070000084A094B59
:1058800011681B6810B5CB1A03D41360FFF7EEFE46
:1058900010BDFA235B001360034A13680133F4E779
:1058A00048000010F00E0010B00E00100122034B53
:1058B0001A60034BF432FF321A607047B00E0010CA
:1058C0004800001073B5040000250026134B009615
:1058D0001B680196B34218D101350220FAF72AFD60
:1058E0000F4B1A680F4B11681868814208D0126874
:1058F0001A60FFF7C3FF002C02D0013C002C02D03D
:10590000042DE2D10124200076BD684601A9984704
:10591000009B002BE0D03500DFE7C046CC0E001026
:10592000D40E0010E40E0010F7B50D000E21040097
:10593000019201F0B5FC184B03260A279D4211DDA8
:1059400009236373083B2373F7BD2800390001F076
:10595000A1FC2800A155390001F0B6FB0136050075
:105960000D2E01D0002DF0D1019BA11CF21A033A9B
:1059700022700D22A319921B013B8B4208D10F23E9
:1059800000229E1B731E032EDEDD1E00E254F9E78B
:1059900018789854F0E7C046FFC99A3B0378002B6B
:1059A00001D10133FF334078002801D10130FF30AD
:1059B000181A70479B23F0B5224E5B00F45C85B04B
:1059C0000D000390002C01D10134FF343023FF334C
:1059D000F35C002B32D002933823FF33F25C373B69
:1059E00007279C4201D0083717401748FFF7D6FF1A
:1059F0000721C91B01918021029B4900E31A0C1B5E
:105A0000421C009411490398FEF70AFA002341242E
:105A10002B702800FEF752FA2F1830007530FF3037
:105A2000001BFFF7BBFF22000300094938000134C7
:105A3000FEF7F6F9462CECD105B0F0BD80235B00F3
:105A4000C9E7C046D80600100C080010B4D7000003
:105A5000C1D70000F0B5784B784C0500E050043316
:105A6000E150230094331B680E0093B0002B1BD130
:105A7000182817D1C32907D0F723DB00E358332BAD
:105A800010D100F00FF90DE06D4B1B680F2B09D101
:105A900016220E216B4800F067F9674BE35801931B
:105AA000182BE9D0FFF75EFD00239D4200D00A339A
:105AB000F62231002800D200A350FFF73DFE624BD2
:105AC00025001B6800261A68604B8C351A60FFF7AA
:105AD000C1FD012323671D3301935D4B1B68002B20
:105AE00014D05C4F3B68002B10D01B68002B54D0A7
:105AF0003A681368013B1360574A1368002B05DDB1
:105B0000013B1360002B01D1FFF7A4FDFFF7E6FC7A
:105B1000002807DA22002B68903201332B601368CB
:105B2000013313604D4B4E4F9E420CD04023320048
:105B30009A434C4B9A4206D04B4B9E4203D0533370
:105B4000FF339E4211D1E359484A93420AD01A00CA
:105B50002020474982438A4204D040229343454A49
:105B6000934202D10A20FFF75DFD2B68424AE659B5
:105B700093423BD016DC414A93421CD0404A9342A8
:105B80001CD0019B002B40DD013B0193236F002BB8
:105B9000A3D1FFF76BFD13B0F0BD3A4B1B689847DC
:105BA0003B68A2E7384A934219D0384A9342E8D179
:105BB000FBF7AEFAE5E7FBF751FAE2E7FBF7BAFAD3
:105BC000FFF792FDFAF760FC314B204A18601A4B40
:105BD000E0501368013B13602E4B2B60D1E7FAF7BE
:105BE000ADFBFFF763FEFFF77FFDCAE72A4F3B6877
:105BF000002BC6D00AA902A8FFF7DCFE3B680AA961
:105C000002A898472B682733E7E7244B1B6898477F
:105C10001E200D4B01901A68214B116818688142B3
:105C2000B4D012681A60FFF717FEFFF727FE154B76
:105C30001B689847AAE7C046B4070000D8060010C2
:105C40004400001010070010D40E00104C0000108B
:105C5000C00E0010C80E0010C40E00106E0200002E
:105C6000C4070000260200007A020000FB030000C7
:105C7000CB030000A30300003E27000048080000FB
:105C8000790D0000BC0E00105C2800008533000078
:105C9000DC0E00107E0D0000E80E0010EC0E00106F
:105CA000E40E0010F8B52A4D00202B681C68FFF7A1
:105CB00009FE2B681A68A242FCD01F68FFF752FC4D
:105CC000F6230A22234CDB00E2501823224A012645
:105CD000A350F7231522DB00E2500833E6502300DF
:105CE000002290332D371A60FF37FFF73BFC266701
:105CF0002B681B68BB421ED12300F8260127F60043
:105D00009033002118201D68A751FFF7A3FE134B05
:105D10002800196801F0D8F9042201001048FFF7A3
:105D200003FE18230C4A2800A350F7230022DB00AF
:105D3000A751E250F8BDFFF7D1FB2A68094B116863
:105D400018688142D4D012681A60FFF797FDCFE738
:105D5000D40E0010D8060010B4070000F00E00109A
:105D600010070010E40E0010F0B50125002A00DC39
:105D7000F0BD03784C1E2B40002C01DA013AF5E708
:105D8000065DDB0077083B4303553300013C2B40A5
:105D9000F2E730B59A4200DD30BD845C8D5C8554FD
:105DA0008C540132F6E7F0B5060007A8057806988E
:105DB00001240078002A1DD0059CA34204DD0123A4
:105DC0001840069B1870F0BDD75CCC5CBC466444A0
:105DD00024180020A54201DC641B0130F454013377
:105DE000EAE7CA5C12180020954201DC2000521B31
:105DF000F2540133059A9342F3DDE0E7F7B50AACBC
:105E00002478089F0194099C2478002839D00F2514
:105E1000002933D0002A1ED1019E0F32013E1640C8
:105E2000BB421ADCCA5C121B0024551C01D1320093
:105E30000134C2540133F3E7CD5C2E00D55C751BF1
:105E40002D1B0024A54204DA019C65190F2425406E
:105E50000E3CC5540133BB42EEDD01231C40099BBF
:105E60001C70F7BDD15C49420C1B00218C4203D051
:105E70000199091901242940C1540133BB42F1DDC4
:105E8000EBE7002919D0002A0ED1BB42E5DCCA5C41
:105E90000133141B013462425441F6E7C85CD55CFF
:105EA0000133401B041BE40FBB42F7DDD5E7D15C97
:105EB000013349420C1B611E8C41BB42F7DDCCE72C
:105EC00070B50125049C257000290BD19A420BDC8A
:105ED000815C00290AD10132F8E7865C8D5CAE4214
:105EE00004D101329A42F8DD0023237070BD0B000B
:105EF00030B5441C934207DB00242300914200DCB0
:105F0000531A4018C45430BDE55CC5540133F1E761
:105F1000130030B5441E8B4207DC002423008A4264
:105F200000DB8B1A8018C45430BDE55CC554013BBE
:105F3000F1E70000F0B5114A01241378C15C5378F1
:105F40000B405A1E93410E499B010B600D4B0022E2
:105F50001F0001254A6012371A785E78825C16426B
:105F600002D04A682A434A6002336D00BB42F3D133
:105F7000013404310B2CEAD10020F0BD9201001055
:105F800088100010DE000010122230B505254A43AB
:105F9000324C01311319A25C5C78825C6943144273
:105FA00004D05F242E4A5218947054709A78DC788A
:105FB000825C144204D07C24294A52185332147053
:105FC0001A795C79825C144204D07C24244A5218E9
:105FD000A33214709A79DC79825C144207D0204A8B
:105FE0005F2452181500A132A2352C7014701A7A51
:105FF0005C7A825C144204D07C24194A5218A03284
:1060000014709A7ADC7A825C144204D07C24144A9C
:106010005218503214701A7B5C7B825C144207D099
:106020000F4A5F2452181500513252352C701470EB
:106030009A7BDC7B825C144204D02E24084A5218DE
:10604000A43214701A7C5B7C825C134204D0044B33
:1060500059182723F4310B70002030BDDE000010EA
:10606000F80E0010F7B5040000262D4D2F00393F23
:106070004F2220213800FDF7FFFE002E02D07C23A6
:106080003B702B7000210136A9755035052EEDD1DE
:10609000244B2D221800383002701800373002705F
:1060A000A1209A705A70400032321A544220FF30B8
:1060B0001A54053019541C4908784978205C01426B
:1060C00004D01900523353310A701A700027390076
:1060D00020000137FFF758FF0A2FF8D10025134E93
:1060E0000197134BAA00D15833787278E35C114FB3
:1060F0001A420CD03800013501F0FCF80236092DA7
:10610000EFD138000C4901F0F5F80520FEBD08007C
:10611000FDF7D4FE019B0949181A0918EAE7C046A1
:10612000310F0010F80E001092010010CC0000108A
:106130007400001038100010C9D70000BC00001017
:10614000014B18707047C046F70E00100020034B3B
:10615000185642425041C0B218707047F60E0010F7
:10616000014B40B218707047F50E00100020014B33
:1061700018567047F50E001070B50C00C3050FD50A
:10618000CCB2D5B2A01DE91DC9B2C0B2FCF79CFAD1
:10619000290005340831C9B2E0B2FCF795FA70BDA8
:1061A0000306FCD506320634D1B202230122E0B246
:1061B000FCF79EFAF3E7012370B506000C0015000A
:1061C000184206D0D118E0180322C9B2C0B2FCF7B9
:1061D0008FFA02231E4206D0E918201D0122C9B2FF
:1061E000C0B2FCF785FA730707D5691D201D02238D
:1061F0000122C9B2C0B2FCF77BFA330707D5E91D0B
:10620000601C01230322C9B2C0B2FCF771FAF30685
:1062100006D5691D02230122C9B2E0B2FCF768FA73
:10622000B30606D5A91C02230122C9B2E0B2FCF7CD
:106230005FFA730607D5291D013401230322C9B271
:10624000E0B2FCF755FA70BD064B07201B785BB235
:10625000002B06D1044B01381B785BB2002B00D118
:1062600018007047F50E0010F60E00101C4B10B50C
:106270001900DE314A8808881A49120402430020B6
:106280008A4222D1E3335A781C7899781202DB785B
:1062900014430904144A21431B060B43934214D1AF
:1062A000FFF7D2FF1149124C0978020049B2236866
:1062B000104800290AD0023323600F210E4BFCF74F
:1062C00099FA2368023B0120236010BD0333236049
:1062D00009210A4BFCF78EFA2368033BF3E7C0461B
:1062E000D80600103D001D1111444C80F50E001021
:1062F00038000010D1D700004898000058980000DE
:10630000F0B5A24B89B01C680394022C03DD231F57
:106310005A425A410392FFF797FF9D4B06001B78A4
:106320005BB25A1E93415B420293052C4CD0994BB1
:106330000193062C04D0984B0193984B042C47D022
:106340000022974B05921B785BB2934205D007233E
:106350000393944B0193012305930023924C0093E4
:106360000C3C00228E4B9A560823002A00D104339D
:10637000009A0127002A01D017005F43834B1B6856
:10638000022B11DD00227F2007AB5A70E368184012
:106390004E281FDC212800D1CEE05DDC783213428C
:1063A0004ED01C2800D1CDE00123039A072A00D942
:1063B000DBE0100000F0F4FD0D017F010802D900C0
:1063C000D900D900D900000101235B420293774B29
:1063D0000193B5E74F383028E6D800F0D7FD6F00BD
:1063E000AD00E5FFE5FFE5FFB600E5FFE5FFE5FFF2
:1063F000E5FFE5FFE5FF6C00B000E5FF9E00E5FF6F
:10640000E5FFE5FFB300E5FFE5FFE5FF7200E5FF0F
:10641000E5FFE5FFE5FFE5FFE5FF7500E5FF81002E
:10642000E5FFA400E5FFAA00A700E5FFA70095008F
:10643000E5FFA100E5FFE5FF98007800E5FF7E009D
:106440000728B1D800F0A2FD1400B0FF8400B0FF0F
:10645000B0FFB0FF22004600232876D03838082845
:10646000A2D800F07FFD2557A1A1A1A1A14B4E000C
:10647000202207AB1A70019B3200390007A8FCF7F5
:10648000B9F9059B002B66D000238EE7312207ABBC
:106490001A70009B022BEEDD7F2362681A40542A9B
:1064A00006D0009A032AE6DD22681340542BE2D17D
:1064B0004C2207ABDEE7322207ABDBE7332207AB28
:1064C000D8E7342207ABD5E7352207ABD2E736222F
:1064D00007ABCFE7372207ABCCE7382207ABC9E7DA
:1064E000392307AA1370009B062BC4DD7F23A16804
:1064F0000B40232BBFD124331370BCE7302207ABF2
:10650000B8E72D2207ABB5E7412207ABB2E742223D
:1065100007ABAFE7432207ABACE7442207ABA9E7E1
:10652000452207ABA6E7462207ABA3E7482207AB05
:10653000A0E7502207AB9DE7522207AB9AE74F2214
:1065400007AB97E7552207AB94E74E2207AB91E7DD
:10655000492207AB8EE7E368DA050FD5029B1448A2
:106560009A19019BF91DFCF745F9009B043401338E
:1065700000930B2B00D0F4E609B0F0BD1B06F4D558
:106580003200019B0B48F91DEDE7C046C800001022
:10659000F60E001030980000589800005098000047
:1065A000F50E001048980000881000103898000080
:1065B000DED70000477A0000002B04D032003900FB
:1065C000E068FFF7F8FD32003900E068FFF7D4FD1E
:1065D000CBE70123E2681A4205D0B81C0522F1B2CC
:1065E000C0B2FCF785F8E3689B0707D5711CF81D5E
:1065F00003230122C9B2C0B2FCF77AF80423E2688F
:106600001A4206D0711DF81D0122C9B2C0B2FCF7B2
:106610006FF80822E368134208D03100B81C093132
:106620000123C9B2C0B2033AFCF762F8E368DB06A3
:1066300007D5711D781C04230122C9B2C0B2FCF732
:1066400057F8E3689B0607D5711C781C03230122C9
:10665000C9B2C0B2FCF74CF8E3685B0607D5311D40
:10666000B81C01230522C9B2C0B2FCF741F8E368A7
:10667000DA0513D5029BFFB2F518EDB229003800F8
:106680000A310930C9B2C0B2FCF71EF83B00093527
:106690000A33E9B2D8B2FCF717F866E71B0600D454
:1066A00063E731000123022209310937C9B2F8B288
:1066B000FCF71EF859E70122E368134212D0FDB23D
:1066C000F1B20495A81C0D001300C0B20432FCF70F
:1066D0000FF86B1CD9B2049B0322DD1CE8B2012326
:1066E000FCF706F80222E368134206D0711CB81DBD
:1066F0000323C9B2C0B2FBF7FBFF0423E2681A42CE
:1067000006D0711DB81D0222C9B2C0B2FBF7F0FF5E
:106710000822E368134212D0FDB2F1B2A81C09317D
:106720000123C9B2C0B2033AFBF7E2FFF1B208316C
:10673000033501230322C9B2E8B2FBF7D9FFE368AE
:10674000DB0607D5711D781C04230222C9B2C0B232
:10675000FBF7CEFFE3689B0607D5711C781C03236B
:106760000222C9B2C0B2FBF7C3FFE3685B0612D5D1
:10677000FDB2F3B2191DA81C01230522C9B2C0B293
:10678000FBF7B6FFF3B20533D9B203220123033579
:10679000E8B2FBF7ADFFE368DA055FD5029BFFB215
:1067A000F518EDB229003800022308310A301A002A
:1067B000C9B2C0B2FBF79CFF3B0009350933E9B20F
:1067C000D8B202231A0073E7E368DB0706D5781C0A
:1067D00002230722F1B2C0B2FBF78AFF0222E3686C
:1067E000134205D0B81D0623F1B2C0B2FBF780FFFB
:1067F000E3685B0707D5311DB81D06230222C9B225
:10680000C0B2FBF775FF0822E368134207D0B11846
:10681000781C0223C9B2C0B2013AFBF769FFE368F2
:10682000DB0607D5311D781C06230222C9B2C0B28F
:10683000FBF75EFFE3689B0606D5781C0623022261
:10684000F1B2C0B2FBF754FFE3685B06A3D5311D7C
:10685000781C02230722C9B2C0B29AE71B0600D4F3
:1068600083E6310009370831C9B2F8B2A9E7C0465A
:10687000F7B52C4A2C4B12781B6852B22B4C019066
:10688000002A27D0002B06D001228021284B29483E
:106890005242FBF7AFFF012700257F42264BEB5CFE
:1068A000012B12DC019922788A5C617811420CD0AC
:1068B000224AA9008858224AA95C08228900002B94
:1068C00000D13A001A4BFBF795FF01350234092D30
:1068D000E4D1F7BD1B4A0927127852B2002A01D031
:1068E00002277F42002B05D03A000021104B1148AF
:1068F000FBF780FF0025019A2378D35C62781A4267
:106900000AD0114B1148E95CAB009C4666463A0040
:10691000074B3058FBF76EFF01350234092DEAD1E1
:10692000D7E7C046F50E0010B0040010CC000010F0
:1069300040980000F875000037D8000050000010A3
:106940002ED80000F60E001040D80000980000106D
:1069500070B500F005FA00280CD0114B06241B7806
:1069600003265BB2002B09D002233200002118005D
:10697000FBF7BEFE70BD01340F2CFBD031002000B0
:1069800000F088FC2000CDB2310000F09DFB290012
:10699000C0B2FBF799FE092CEDD10234EEE7C046F8
:1069A000F50E001070B50D000400FFF7C3FAFBF7F9
:1069B000EBFDFFF75BFC002806D1002D01D0FFF7AF
:1069C0009FFC2000FFF754FF094B1B78002B0ED0D3
:1069D0002000FFF747FB0024502529006143054BA9
:1069E0000548C9180134FDF710FA052CF5D170BD22
:1069F00095020010F80E0010ED86000010B588B06A
:106A00000400092101A8FDF765FE12200A2168444F
:106A1000FDF760FE210001A8FFF7C4FF08B010BD1C
:106A200010B5124B1B785BB2002B14D1002813D089
:106A3000FBF775FD0120FFF7E1FFFBF7DDFD00230C
:106A40000B4AD356002B06DD013BDBB21370002B43
:106A500001D1FEF75BFE10BDFBF769FD054B1B780E
:106A6000002BF8D00448FDF7D0F9F4E7F70E00103A
:106A7000F40E001095020010E0D7000010B5FBF7EF
:106A800099FD10BD70B50D0004000721002D0BD03D
:106A9000FDF714FA062156234143591ACB43DB175D
:106AA0001940012D00DD491001222000024B524205
:106AB000FBF7A0FE70BDC04648980000F0B585B059
:106AC000050000F063F98023002849D101932B7C55
:106AD00002AA0093002353712B78092B08D1243389
:106AE000137101220121464B524203A8FBF782FE9B
:106AF0000126012476422B1B1B7CE7000F2B73D051
:106B0000082C2FD16A78002A2CD02D22002B00D1FE
:106B10000D3A02A90A71012C04D12A78012A01D167
:106B200037330B71374B1B68022B4EDC02AB1879E5
:106B30002038252849D800F01FFA444848484848DA
:106B400048484848484848384848364618282A2C73
:106B50002E303234484848484848483A3C3E404243
:106B60005B00B3E730221A43D3E75B2032003900E1
:106B7000FFF721FB009B092B36D8180000F0FCF929
:106B80003C34342C34342C34342C4F20EEE7662043
:106B9000ECE76D20EAE77D20E8E70720E6E77F20C5
:106BA000E4E76F20E2E73F20E0E74020DEE77720E0
:106BB000DCE77C20DAE73920D8E75E20D6E77920C9
:106BC000D4E70020D2E70620D0E7320039000C4B92
:106BD00003A8FBF70FFECDE7C02032003900019B70
:106BE00040005840FFF7C8FA009B0134013B009376
:106BF0000B2C80D105B0F0BD320039000198F1E7CF
:106C000048980000C8000010002210B5094B9A56A1
:106C1000094B002A04D007221100FBF7EBFD10BD41
:106C20000021064A51560622002900D1053A0C21BE
:106C3000F3E7C046F50E001048980000F60E00106D
:106C400010B50400FBF7A0FC0020FFF7D7FE2000E2
:106C5000FFF7DAFF10BD10B5FFF7D6FF10BD00003B
:106C6000002370B5134A144C0D00A3500432A350F6
:106C7000083AA35022008C3210600122E36622679A
:106C8000236F002B04D026008C363368AB4203D12F
:106C9000FEF7E8FA002070BDFEF720FC0028EFDACE
:106CA000220033689032013333601368013313607C
:106CB000E6E7C046B4070000D8060010F0B5224C45
:106CC000A3B015000E0001902100782204A8FDF762
:106CD000B2F81E4F0722390002A8FDF7ACF80123D5
:106CE00031000E221A4823666366FDF7A4F80E22CF
:106CF00000211848FDF7C0F801980021431E984173
:106D0000154B40421840154BA167C018FFF7A8FF6C
:106D1000230045331B7821002B7023004E331B7852
:106D2000E81C5A1E93410E226B70FDF784F804A9EB
:106D300078222000FDF77FF80722380002A9FDF72E
:106D40007AF823B0F0BDC046D806001090070010B6
:106D5000100700101E070010882C00008A02000097
:106D6000014B4A3318787047D80600100200103AD9
:106D70000300B82A05D80448C0181038007840B27B
:106D8000704701204042FBE794010010D320024BE2
:106D90001856C00F7047C046D8060010014B463346
:106DA00018787047D8060010044BD33318780F2397
:106DB00018400F38434258417047C046D80600106B
:106DC000024B986D0338434258417047D806001073
:106DD000014B493318787047D8060010014B4F33E8
:106DE00018787047D8060010084B01201A004A3264
:106DF0001278002A07D09A6D042A03D0B833188875
:106E00000011C0B270474042FCE7C046D8060010EF
:106E100070B504000E49FDF759F82000FDF74EF853
:106E20000C4B0F211A00B932157806002A000A40CF
:106E30000D4202D02F320130A255B8331B781B0906
:106E400002D02F33235401300023235470BDC04699
:106E500049D80000D8060010034B1B18C03B187817
:106E6000024BC0187047C046E4DC000014DD00008F
:106E700070B504000D002878002801D1207070BD85
:106E8000BF2803D8207001340135F4E7FFF7E4FF91
:106E9000060001002000FDF719F83000FDF70EF89C
:106EA0002418F1E70268030010B50B488A4212DC8F
:106EB0005C688C420FDB3F20891A8A1101409818C8
:106EC000047C05488C4206DD9868DB6892009B587C
:106ED00080585B5CC01810BDF3980000C24310B529
:106EE000C3B212070AD1A02B08DD1B11054A0A3BC9
:106EF0009B0001129858FFF7D5FF10BD19000248FA
:106F0000F9E7C04648E60000D0DC000010B50400F8
:106F10000800FFF7E3FF01002000FFF7A9FF10BD05
:106F2000FEE7FEE710B50A4A0A4B0B498B4207D32E
:106F300000210A4B0A4A934207D3FAF737FFFEE7CC
:106F40001078013218700133F0E719700133F2E75D
:106F500060E60000000000104D020010500200101A
:106F6000B410001002B4714649084900095649009E
:106F70008E4402BC7047C04602B4714649084900BD
:106F8000095C49008E4402BC7047C04603B4714698
:106F9000490840004900095E49008E4403BC70471F
:106FA00003B47146490840004900095A49008E441B
:106FB00003BC7047002243088B4274D303098B4201
:106FC0005FD3030A8B4244D3030B8B4228D3030CB9
:106FD0008B420DD3FF22090212BA030C8B4202D35B
:106FE0001212090265D0030B8B4219D300E0090A83
:106FF000C30B8B4201D3CB03C01A5241830B8B428C
:1070000001D38B03C01A5241430B8B4201D34B0374
:10701000C01A5241030B8B4201D30B03C01A5241D9
:10702000C30A8B4201D3CB02C01A5241830A8B425E
:1070300001D38B02C01A5241430A8B4201D34B0247
:10704000C01A5241030A8B4201D30B02C01A5241AB
:10705000CDD2C3098B4201D3CB01C01A524183095F
:107060008B4201D38B01C01A524143098B4201D399
:107070004B01C01A524103098B4201D30B01C01AC4
:107080005241C3088B4201D3CB00C01A524183083E
:107090008B4201D38B00C01A524143088B4201D36B
:1070A0004B00C01A5241411A00D2014652411046CB
:1070B0007047FFE701B5002000F0F0F802BDC046C0
:1070C0000029F7D076E7704703460B437FD40022B0
:1070D00043088B4274D303098B425FD3030A8B426C
:1070E00044D3030B8B4228D3030C8B420DD3FF22D6
:1070F000090212BA030C8B4202D31212090265D0A4
:10710000030B8B4219D300E0090AC30B8B4201D356
:10711000CB03C01A5241830B8B4201D38B03C01A9D
:107120005241430B8B4201D34B03C01A5241030B14
:107130008B4201D30B03C01A5241C30A8B4201D3C5
:10714000CB02C01A5241830A8B4201D38B02C01A70
:107150005241430A8B4201D34B02C01A5241030AE7
:107160008B4201D30B02C01A5241CDD2C3098B42CC
:1071700001D3CB01C01A524183098B4201D38B0149
:10718000C01A524143098B4201D34B01C01A5241EC
:1071900003098B4201D30B01C01A5241C3088B4231
:1071A00001D3CB00C01A524183088B4201D38B001C
:1071B000C01A524143088B4201D34B00C01A5241BE
:1071C000411A00D201465241104670475DE0CA0F95
:1071D00000D04942031000D34042534000229C4655
:1071E00003098B422DD3030A8B4212D3FC2289015F
:1071F00012BA030A8B420CD3890192118B4208D335
:10720000890192118B4204D389013AD0921100E096
:107210008909C3098B4201D3CB01C01A52418309AA
:107220008B4201D38B01C01A524143098B4201D3D7
:107230004B01C01A524103098B4201D30B01C01A02
:107240005241C3088B4201D3CB00C01A524183087C
:107250008B4201D38B00C01A5241D9D243088B42D2
:1072600001D34B00C01A5241411A00D20146634675
:1072700052415B10104601D34042002B00D54942D9
:10728000704763465B1000D3404201B5002000F018
:1072900005F802BD0029F8D016E770477047C046D0
:1072A00010B50A000021FCF7E7FD10BD30B5032A38
:1072B0000CD903000B439B0719D103680C68A34248
:1072C00015D1043A04300431032AF6D8551E002A99
:1072D0000BD0002303E05A1C9D4206D01300C25C71
:1072E000CC5CA242F7D0101B00E0002030BD551E40
:1072F000EFE7C04670B50400830716D102680E4B55
:107300000E4DD31893432B420FD142680A4B0430E1
:10731000D31893432B4208D14268074B0430D3184B
:1073200093432B42F1D000E001300378002BFBD1D6
:10733000FCF7CCFD200070BDFFFEFEFE808080804B
:107340005B4025303278253032785D0D0A00444D9F
:1073500031355F4D31420025732025730D0A0053EE
:10736000455249414C20434F4E534F4C45007265A6
:10737000616479000D0A4279652E2E2E0D0A004EA9
:107380004F00203F00563334002573202573202002
:1073900025694D485A00202025692E25303369562D
:1073A0000020257352544320005245534554205425
:1073B0004F2041424F525400524541445920464FBC
:1073C0005220464C415348494E47004C43443A25CD
:1073D000303269202D2025690050524553532045F5
:1073E0004E54455220544F2053415645005357495F
:1073F00053534D4943524F532028432920323031B3
:10740000302D323032350025633120484F5552003F
:107410002D005254432052454144204641494C00DE
:107420005F007E005052474D20544F50004E554C47
:107430004C00537461727420626F6F746C6F61647E
:1074400065723F00454E544552206966204F4B20DF
:10745000656C73652061626F72740053657475703A
:107460003A0050726573732061206B6579004C653A
:107470006176696E67207365747570206D656E75D1
:107480000089004B657920257800556E7573656419
:10749000206B6579008B008A002573202D3E202506
:1074A000730031202573203D00583C3E5920666F03
:1074B0007220636F6E7374616E747300583C3E5932
:1074C00020666F7220636F6E76657273696F6E737C
:1074D000004D657472696320746F20496D70657228
:1074E00069616C00436F6E7665727420666F7277A7
:1074F000617264206F7200496D70657269616C2001
:10750000746F204D657472696300436F6E766572A7
:1075100074206261636B77617264206F72006661D0
:1075200063746F7220746F20737461636B005075A5
:10753000736820636F6E7374616E74206F72206362
:107540006F6E762E004C656176696E6720636F6E94
:107550007374616E7473206D656E7500556E75730E
:107560006564206B6579202578005B4031383030C8
:107570005D0D0A005B40303030305D0D0A007475DF
:10758000726E6564206F6E003C52455345543E0D4B
:107590000A00436F6E7374616E747300436F6E768E
:1075A000657273696F6E73006B7068006D70680050
:1075B0006D2F730066742F73006B6E6F74004670CE
:1075C00046006D6D00696E006D69006674006B6D3C
:1075D000006E6D006B67006F7A00746F6E28696DC6
:1075E000702900746F6E2875732900746F6E286D92
:1075F0006574726963290050610070736900617479
:107600006D00746F7272004A006674206C627300C1
:107610006B5720680062747500636D9100696E910C
:1076200000667491006B6D91006D699100616372E9
:1076300065009C43009C460067616C2875732900B7
:1076400067616C28696D702900636DA000696EA088
:10765000006674A0005370656564206F66206C69D5
:1076600067687400506C616E636B20636F6E737437
:10767000616E74004A20730052656475636564200E
:10768000506C616E636B20636F6E73742E00426F7B
:107690006C747A6D616E6E20636F6E7374616E745C
:1076A000004A2F4B0041766F676164726F20636FF1
:1076B0006E7374616E7400312F6D6F6C004D6F6C62
:1076C00061722067617320636F6E7374616E740002
:1076D0004A2F6D6F6C2F4B00466172616461792097
:1076E000636F6E7374616E7400432F6D6F6C004D29
:1076F0006F6C2E766F6C2E20696465616C206761FB
:107700007320535450006DA02F6D6F6C0041746F47
:107710006D6963206D61737320636F6E7374616E46
:107720007400426F687220726164697573004772F9
:10773000617669746174696F6E616C20636F6E73DA
:1077400074616E74006DA02F6B672F73910041639D
:1077500063656C657261742E206F66206772617656
:10776000697479006D2F739100456C656D656E7459
:10777000617279206368617267650056616375752F
:107780006D207065726D69747469766974790046EC
:107790002F6D0056616375756D207065726D656142
:1077A00062696C697479004E2F41910046696E657B
:1077B0002D73747275637475726520636F6E737464
:1077C0002E005279646265726720636F6E73746114
:1077D0006E7400312F6D00436F6E64756374616E5B
:1077E0006365207175616E74756D004D61672E2043
:1077F000666C7578207175616E74756D00576200E6
:10780000426F6872206D61676E65746F6E004A2FFB
:107810005400456C656374726F6E206D6173730004
:107820004E657574726F6E206D6173730050726F68
:10783000746F6E206D61737300417374726F6E6F3D
:107840006D6963616C20756E6974004C696768745A
:107850002D796561720050617273656300536F6CBE
:107860006172206D6173730053746566616E2D42A1
:107870006F6C747A6D616E6E20636F6E73740057F7
:107880002F6D912F4BA1005769656E20776176654A
:107890006C656E67746820636F6E73742E006D2064
:1078A0004B004A757069746572206D617373004591
:1078B00061727468206D6173730045617274682031
:1078C0006D65616E20726164697573004D6F6F6ED6
:1078D000206D617373004100446973706C6179209D
:1078E000646174652F74696D650042656E63686DCF
:1078F00061726B0053657269616C20636F6E736FA8
:107900006C6500537461727420626F6F746C6F6188
:107910006465720053797374656D20696E666F00DB
:10792000434853004C434420636F6E747261737418
:1079300000454558004C434420636F6E7472617378
:10794000742072657365740053544F005254432081
:107950002D3120686F75720052434C005254432001
:107960002B3120686F7572003100312D6C696E65A6
:1079700020646973706C6179003200322D6C696E1D
:107980006520646973706C61790037004379636CBA
:107990006520666F6E74003900546F67676C6520F0
:1079A000435055207370656564008F004B657962A4
:1079B0006F6172642074657374008E0053656C6629
:1079C000207465737400506F7765722072657365FB
:1079D00074002B00456E646C65737320746573745A
:1079E00000546F67676C6520646F742F636F6D6DF3
:1079F00061005353540041646A7573742064617468
:107A0000652F74696D650047544F00546F67676C4C
:107A10006520616E6E756E636961746F7220706F40
:107A2000730052434C2B200052434C2B202E00520B
:107A3000434C2D200052434C2D202E0052434C2A03
:107A4000200052434C2A202E0052434C2F2000523B
:107A5000434C2F202E0053544F2B200053544F2BB8
:107A6000202E0053544F2D200053544F2D202E0014
:107A700053544F2A200053544F2A202E0053544F62
:107A80002F200053544F2F202E00534F4C5645208B
:107A900000534F4C5645202E009596200095962079
:107AA0002E00783C3E2000783C3E202E004453457A
:107AB0002000445345202E00495347200049534796
:107AC000202E004C424C202E0047544F202E0047C1
:107AD0005342202E005346200043462000463F20BC
:107AE0000046495820005343492000454E47200096
:107AF00053544F204D415452495820004C424C2081
:107B00000047544F2000475342200052434C20006E
:107B100053544F200052434C202E0053544F202EDC
:107B20000052434C204D4154524958200052455375
:107B3000554C54200052434C2044494D20005243A0
:107B40004C2067200053544F206720004859502094
:107B500000485950932000544553542000330036B8
:107B60000038002869290097002A002F00434C5252
:107B70005F5052474D00496E76616C6964206D61BB
:107B800074682F446976206279203000496D7072E4
:107B90006F706572204D6174726978206F70732EFA
:107BA00000496D70726F7065722097206F70732E30
:107BB000004261642052656720232F4D6174726911
:107BC0007820656C656D00426164204C696E6520AB
:107BD000232F4C6162656C2063616C6C005375628D
:107BE00072206C6576656C20746F6F2064656570BB
:107BF00000496D70726F70657220666C6167206EEF
:107C0000756D626572005265637572736976652081
:107C1000536F6C7665206F72209500536F6C76659C
:107C20002063616E27742066696E6420726F6F74C2
:107C300000496E76616C69642073656C662D7465AD
:107C4000737400496E73756666696369656E742046
:107C50006D656D6F727900496D70726F706572201D
:107C60004D6174726978206172670000767B000054
:107C70008C7B0000A17B0000B17B0000C77B000073
:107C8000DD7B0000F17B0000067C00001B7C000017
:107C9000317C0000437C0000577C0000CA00CB0010
:107CA000CC00CD00CE00C300FFFFFFFFFFFFFD00B3
:107CB000FFFFFDFFC700C800C900D7FFFFFFFFFFA0
:107CC000FFFFFC00FFFFFCFFC400C500FFFFC10079
:107CD000FFFFFFFFFFFFFB00FFFFFFFFFFFFFAFFBC
:107CE000FBFFFFFFFFFFFFFFFE00FA002A002B0053
:107CF0002C002D002E0005FF08FF07FF06FF1DFFCB
:107D0000FEFFF1FFF5FFFFFFDEFFF6FF19FF17FF94
:107D100015FF1BFFFFFFDD00EEFFA500FFFFA10029
:107D2000D100D200D300DB00FFFFFFFFFFFFA30065
:107D3000FFFFFFFFD000A000DE00DA00BA00BB00AA
:107D4000BC00BD00BE00B300E700E800E900ED00A4
:107D5000FFFFF0FFB700B800B900B6000BFF0AFF45
:107D600009FFEC00FFFFB200B400B500A200B100B3
:107D7000E100E200E3000F00FFFFFFFFFFFFEB0069
:107D8000FFFFFFFFE000B000EE00EA00001100007E
:107D900055760000B075000008005824799902005B
:107DA0000012000064760000747600006609157009
:107DB0006062060000130000787600007476000010
:107DC0006679817145050100001400008E7600007F
:107DD000A17600007709004906380100001500006F
:107DE000A5760000B7760000230076402102060049
:107DF00000160000BD760000D076000000806162B1
:107E00004431080000170000D8760000E976000031
:107E1000042021338564090000180000EF7600007B
:107E20000677000096499596132402000019000079
:107E30000D770000D47500007399063905660100BE
:107E40000010000022770000D577000089591072D9
:107E500017290500002100002E770000457700005B
:107E60008909000043670600002200004E770000E9
:107E700064770000000000506680090000230000C5
:107E80006977000033760000814963762160010044
:107E9000002400007B7700008F770000889981879D
:107EA000418508000025000093770000A7770000B7
:107EB000941906376625010000260000AC77000003
:107EC000F3980000974956527329070000270000D5
:107ED000C2770000D37700000770157373090100A3
:107EE00000280000D7770000227900009599729150
:107EF0008074070000290000EB770000FD77000088
:107F00008589843378060200002000000078000094
:107F10000E78000076690610402709000031000045
:107F200012780000D475000069497183931009002C
:107F30000032000020780000D4750000731950272B
:107F400049670100003300002D780000D47500005F
:107F5000736992212667010000370000397800001C
:107F6000D577000011707078594901000038000081
:107F70004B780000D57700001530473007460900E0
:107F80000039000056780000D577000016105877A9
:107F900056080300003000005D780000D475000032
:107FA00030000075849801000044000068780000EB
:107FB0007F78000092994174036705000045000036
:107FC000877800009E7800009759957177890200A4
:107FD00000470000A2780000D475000027000030A0
:107FE0008189010000480000AF780000D4750000CE
:107FF000240000002297050000490000BA78000024
:10800000D577000006000000103706000040000091
:10801000CC780000D4750000220000002034070056
:1080200000FF0000F3980000F3980000000000003B
:1080300000000000927500009C7500008C7D00001F
:108040004480000002110000A8750000AC7500001B
:10805000000000409360010001120000B0750000B4
:10806000B475000000000040082803000113000060
:10807000B9750000AC750000000000800715010014
:1080800001140000B9750000A87500000000000090
:108090002085010002150000BE750000AC750000CF
:1080A000030000008068020002160000C275000094
:1080B000C575000001000000005402000117000017
:1080C000C8750000CB750000030000000028050003
:1080D00001180000D5770000CB75000000000040BB
:1080E0000828030002190000CE750000C8750000C2
:1080F000000000409360010001100000D1750000F5
:10810000C875000000000080071501000121000073
:10811000D47500000C76000000000020462002000C
:1081200002220000D5750000D77500000100005044
:108130004983020001230000DA7500000C7600007C
:10814000030000000024020001240000E375000089
:108150000C76000003000000000002000125000072
:10816000EB7500000C7600000300002046200200A2
:1081700001260000F7750000FA75000096090080DE
:108180000345010001270000F7750000FE7500009F
:10819000940900009286090001280000F77500008C
:1081A0000276000097090020065007000129000010
:1081B000FA75000002760000010000901417050017
:1081C00001200000FE7500000276000002000000A1
:1081D000006007000131000007760000097600000A
:1081E0009909002056370700013200001076000080
:1081F000097600000600000052650200013300000D
:1082000009760000157600009709007050280100DB
:1082100002370000197600001D7600000000000003
:1082200060450600023800001A7600002176000042
:108230009809000003290900023900002576000092
:1082400029760000000000909958020001300000DB
:108250002D760000297600009709000025560100C0
:108260000144000032760000357600000000000076
:1082700000800100015500003276000035760000D4
:1082800001000000002003000145000032760000DC
:10829000A07800000000000000000100015500006F
:1082A00032760000A0780000020000001573020082
:1082B00002470000E2740000387600000000001061
:1082C0005478030002480000E27400004076000089
:1082D000000000906054040001490000497600004D
:1082E0004D76000098090070231006000140000040
:1082F0004A7600005176000001000070145303001C
:1083000000FF0000F3980000F39800000000000058
:1083100000000000E4FFE3FFE2FFE1FFE0FF05FFF4
:10832000E7FFE6FFE5FFD8FFFFFFFFFFF5FFDDFFFB
:10833000DEFFF6FFEAFFE9FFE8FFD9FFFFFFFFFFDF
:10834000FFFFFFFFFFFF5DFFEDFFECFFEBFFDAFF3D
:10835000FFFFFFFFFFFFFFFFFFFFFFFFEEFFDFFF5E
:10836000DCFFDBFFC001071C10DF01071C10DF4131
:10837000071C10DF61071C10DFE1071E10C041075A
:108380001C10C001071C301F000000001F2000004F
:10839000001F6000000020030820A0007000000003
:1083A00020020820A00101010101000000000000DE
:1083B00000000000000100010001000100000000B9
:1083C00000000000000100010001000100000100A8
:1083D0000100010001000100000000000000000099
:1083E0000000000000000000010202050400000778
:1083F00007090908080A0A00030003000300030034
:108400000000000000000000030003000300030060
:108410000001000100020003000300000000000052
:10842000000000060606060606000700FC7A0000AB
:10843000017B0000067B00000B7B0000107B00002E
:10844000157B00001B7B0000217B00002D7B0000C2
:10845000397B0000357B00003E7B0000457B00003F
:108460004C7B0000517B0000577B00008A7B0000A2
:1084700068790000797900005D7B00008773000057
:10848000057400005F7B00008A790000617B0000BA
:1084900097790000D678000055730000337600000D
:1084A000F8D700006C730000477A0000799B000049
:1084B000637B0000677B0000D2790000107400002D
:1084C000697B00006B7B000031790000F3980000AD
:1084D000F39800006D7B0000227A0000287A0000EB
:1084E0002F7A0000357A00003C7A0000427A0000C2
:1084F000497A00004F7A0000F3980000F3980000DA
:10850000F3980000F3980000F3980000F39800003F
:10851000F3980000F3980000567A00005C7A00009F
:10852000637A0000697A0000707A0000767A0000B1
:108530007D7A0000837A0000F39800008A7A0000B8
:10854000917A0000997A00009D7A0000A27A0000DA
:10855000A77A0000AD7A0000B27A0000B87A000075
:10856000BD7A0000F3980000F3980000F398000033
:10857000F3980000F3980000C37A0000C97A000065
:10858000CF7A0000D57A0000D97A0000DD7A0000A9
:10859000E17A0000E67A0000EB7A0000257B00001B
:1085A000F07A000011000000D6780000D8780000B2
:1085B0001200000055730000EA780000130000006C
:1085C00033760000F478000014000000F8D70000B3
:1085D00003790000150000006C730000147900009E
:1085E0001600000020790000247900002600000019
:1085F000317900003579000044000000487900001E
:108600004C79000045000000587900005C790000BA
:1086100037000000687900006A7900003800000027
:10862000797900007B790000170000008A7900004A
:108630008C790000190000009779000099790000FA
:1086400010000000AA790000AC79000020000000B2
:10865000BA790000BC7900003000000010740000FE
:10866000C679000040000000D2790000D4790000F3
:1086700048000000477A0000E17900002100000076
:10868000F2790000F679000022000000077A00006D
:108690000B7A0000FF000000F3980000F398000040
:1086A000426164206E756D6265722E0D0A00424152
:1086B000543A2025696D560D0A000D0A253032788E
:1086C00020200057616974696E6720666F722064AC
:1086D0006174612E2E2E0D0A00426164206D6F645C
:1086E000656C0D0A004F4B00526561642025730DC7
:1086F0000A004641494C4544006F6666004C4344BD
:108700002064656275672025730D0A004B42442082
:108710006F75747075742025730D0A00436F6E7346
:108720006F6C652074696D656F7574207365742056
:10873000746F202569206D696E757465730D0A006C
:1087400074776F006F6E650053617920626F6F748C
:108750006C6F61646572202573206D6F7265207483
:10876000696D652573202E2E2E0D0A004C61756EE5
:108770006368696E6720626F6F746C6F61646572A5
:10878000202E2E2E0D0A00000000005C000C000CB4
:108790007C287C7C447C241048285408000C003839
:1087A0004400443800201008103810804000101099
:1087B00010004000201008384438007C0064544801
:1087C0004454281C107C4C542438542004740C2825
:1087D000542808543800500080500010284428289D
:1087E00028442810045408384C5C7814787C5428A9
:1087F0003844447C44387C54447C14043844347CED
:10880000107C007C0020403C7C106C7C40407C084C
:108810007C7C047C7C447C7C14083844787C146820
:10882000485424047C047C407C3C403C7C207C6C90
:10883000106C1C601C64544C7C4400081020447C68
:108840000008040880808004080078447878447820
:1088500078447878447878447878141448543C0004
:108860000503050000BE0405000E000E050528FEE8
:1088700028FE2805054854FE54240505462610C840
:10888000C405056C92AA44A00305000A060405006D
:10889000384482040500824438050528107C1028DD
:1088A000050510107C1010030500A06005051010D0
:1088B000101010030500C0C00505804020100805F9
:1088C000057CA2928A7C04050084FE800505C4A272
:1088D00092928C0505449292926C0505302824FEF4
:1088E0002005054E8A8A8A72050578949292600561
:1088F0000502E2120A0605056C9292926C05050CBF
:108900009292523C0305006C6C030500AC6C0405AC
:108910001028448205052828282828040582442890
:108920001005050402A2120C05056492F2827C0572
:1089300005FC121212FC0505FE9292926C05057C54
:10894000828282440505FE828244380505FE9292A9
:1089500092820505FE1212120205057C8282A2E4B3
:108960000505FE101010FE04050082FE820505605C
:108970008080807E0505FE102844820505FE8080EB
:1089800080800505FE041804FE0505FE081020FE83
:1089900005057C8282827C0505FE1212120C0505FB
:1089A0007C82A242BC0505FE1232528C05054C9217
:1089B00092926405050202FE020205057E80808017
:1089C0007E05050E30C0300E0505FE403040FE0528
:1089D00005C6281028C605050608F008060505C2C4
:1089E000A2928A86040500FE8282050508102040B6
:1089F000800405008282FE050508040204080505BE
:108A00008080808080040500020408050540A8A835
:108A1000A8F00505FE909090600405708888880590
:108A20000560909090FE050570A8A8A830050588FF
:108A300088FC8A8A050510A8A8A8780505FE1010EC
:108A400010E005058888FA8080040500888A78058A
:108A500005FE20205088050502027E80800505F86D
:108A6000083008F00505F8080808F0050570888842
:108A700088700505F828282810050510282828F8EA
:108A80000505F810080808050590A8A8A8480505D8
:108A900008087E8888050578808040F805051860FC
:108AA000806018050538C030C03805058850205052
:108AB00088050518A0A0A078050588C8A89888048E
:108AC0000500106C8203050000FE040500826C1096
:108AD0000505201010201000050505905060A0909D
:108AE000050590A04020100505945464A494050544
:108AF00094A44424140505905462A490050590A400
:108B00004224100505A0B0A8A4A20505A2A4A8B0FF
:108B1000A005052868382C280505103854101005C4
:108B200005101054381005050804FE04080505203A
:108B300040FE40200305003030050544281028443D
:108B400005051010541010040500243E20030532C2
:108B50002A240505120A0C14120505080808003E0F
:108B600005052040FE0202050540807C0204030545
:108B70002AC42A050582C6AA92C60505887808F87F
:108B8000880505609090701005057C9292927C0596
:108B90000580C0A090F804050C12120C0405008892
:108BA000FA8004057C54544405058000800080034D
:108BB00005222A14040518143E10000500000406BE
:108BC00003000000007F0107040000070000000709
:108BD0000B064400FF0144004400FF014409058CDA
:108BE000009200FF019200620C0686004600200001
:108BF0001000880184010C06EE00110111012E0104
:108C0000C000600105030000000007090500000026
:108C100000010182007C080400007C008200010148
:108C20000905100054003800540010090510001008
:108C3000007C0010001006030000800580030B0676
:108C4000100010001000100010001006030000803B
:108C500001800109050000C00030000C00030B0674
:108C6000FE000101010101010101FE0C06000004EA
:108C7000010201FF01000100010C068201410121F6
:108C800001210111010E010B0682000101110111E8
:108C9000011101EE0B063000280024002200FF0124
:108CA000200B068F000901090109010901F10B06DA
:108CB000FC001201110111011101E00B060100017C
:108CC00000E10111000900070B06EE00110111017E
:108CD00011011101EE0B060E00110111011101919C
:108CE000007E060300009801980106030000980525
:108CF00098030A05100028004400820001010B06B9
:108D000028002800280028002800280905010182E1
:108D10000044002800100905020001006101110053
:108D20000E0B06FE000101190125012901BE0C06EA
:108D3000FE011100110011001100FE010B06FF01E0
:108D40001101110111011101EE0B06FE00010101DB
:108D50000101010101820B06FF0101010101010175
:108D60000101FE0C06FF01110111011101110101A8
:108D7000010B06FF011100110011001100010B068B
:108D8000FE000101010111011101F20C06FF0110A9
:108D900000100010001000FF010A0501010101FF91
:108DA00001010101010B068000000100010001002A
:108DB00001FF0C06FF0110002800440082000101A1
:108DC0000C06FF01000100010001000100010C067A
:108DD000FF010400180018000400FF010C06FF0149
:108DE0000400080010002000FF010B06FE00010136
:108DF000010101010101FE0B06FF0111001100112B
:108E00000011000E0C06FE0001010101410181006C
:108E10007E010C06FF0111003100510091000E018E
:108E20000B068E001101110111011101E20905016A
:108E3000000100FF010100010B06FF00000100011D
:108E400000010001FF0B061F00600080018001602F
:108E5000001F0C06FF014000300030004000FF0101
:108E60000C06C3012400180018002400C3010905E2
:108E700007000800F0010800070C06C101210111DC
:108E80000109010501030100040603000000007F41
:108E9000010704000007000000070B064400FF0163
:108EA00044004400FF014409058C009200FF019238
:108EB00000620C0686004600200010008801840134
:108EC0000C06EE00110111012E01C0006001050326
:108ED0000000000007090500000000010182007C7D
:108EE000080400007C008200010109051000540004
:108EF00038005400100905100010007C001000100C
:108F000006030000800580030B061000100010000F
:108F10001000100010060300008001800109050008
:108F200000C00030000C00030B06FE0021011101FF
:108F300009010501FE0C06000004010201FF010009
:108F40000100010C06820141012101210111010EE4
:108F5000010B0682000101110111011101EE0B0646
:108F60003000280024002200FF01200B068F00099A
:108F700001090109010901F10B06FC0012011101AF
:108F800011011101E00B0601000100E101110009CE
:108F900000070B06EE001101110111011101EE0B8A
:108FA000060E0011011101110191007E060300005F
:108FB0009801980106030000980598030A0510001F
:108FC00028004400820001010B0628002800280028
:108FD000280028002809050101820044002800100B
:108FE000090502000100610111000E0B06FE0001DF
:108FF00001190125012901BE0C06FE011100110015
:1090000011001100FE010B06FF01110111011101F8
:109010001101EE0B06FE00010101010101010182B7
:109020000B06FF010101010101010101FE0C06FF18
:1090300001110111011101110101010B06FF0111C3
:1090400000110011001100010B06FE0001010101D9
:1090500011011101F20C06FF0110001000100010A8
:1090600000FF010A0501010101FF01010101010BDE
:109070000680000001000100010001FF0C06FF0155
:10908000100028004400820001010C06FF010001CD
:1090900000010001000100010C06FF01040018009E
:1090A00018000400FF010C06FF0104000800100076
:1090B0002000FF010B06FE00010101010101010179
:1090C000FE0B06FF0111001100110011000E0C062D
:1090D000FE0001010101410181007E010C06FF013A
:1090E00011003100510091000E010B068E0011019C
:1090F000110111011101E2090501000100FF010147
:1091000000010B06FF000001000100010001FF0B40
:10911000061F0060008001800160001F0C06FF0137
:109120004000300030004000FF010C06C301240065
:10913000180018002400C301090507000800F00109
:109140000800070C06C101210111010901050103F5
:10915000010007080400000000BF01BF010905006D
:109160000007000700070007130A00002000E400C2
:10917000FC003F00E700FC003F002700040F080050
:10918000000C011E01FF03FF032201E201C2190DC1
:1091900000000E001F0011019101FF007E00FC0085
:1091A000FE0113011101F001E0140A0000EE00FFBE
:1091B0000111011101BF01EE00E0013001100105B4
:1091C0000300000F000F0A050000F800FE03070768
:1091D00001040B060000000001040707FE03F80F5E
:1091E00008000000000A000E001F001F000E000A09
:1091F00011090000100010001000FE00FE00100019
:10920000100010080400000004800780030D070010
:1092100000100010001000100010001008040000E2
:109220000000800180010D07000C000FC003F0005A
:109230003C000F00030F080000FE00FF01010101C8
:10924000010101FF01FE10080000000002010201FF
:10925000FF01FF0100010001100800008601C701A5
:109260006101210131011F010E010F080000820080
:109270008301110111011101FF01EE1109000030FC
:109280000038002C002600FF01FF012000200F08FD
:10929000000080009F011F0111011101F101E10F88
:1092A000080000FC00FE010B0109010901F901F0B1
:1092B0000F08000001000100C101F1013D000F0095
:1092C000030F080000EE00FF01110111011101FF61
:1092D00001EE0F0800001E003F0121012101A10144
:1092E000FF007E0804000000008C018C01080400CF
:1092F0000000048C078C031209000020007000504D
:1093000000D80088008C0104010401110900004804
:10931000004800480048004800480048004811093B
:109320000000040104018C018800D8005000700086
:10933000200D07000002000300B101B9010F000673
:10934000190D0000F800FC010603FB06FD050505EC
:109350000505FD05FF050601FC01F8120900008066
:1093600001F0017C004F004F007C00F00180010FF4
:10937000080000FF01FF01110111011F01FE01E0C2
:10938000110900007C00FE008301010101010101BF
:1093900083018211090000FF01FF010101010101A8
:1093A000018301FE007C10080000FF01FF01110194
:1093B00011011101110111010F080000FF01FF014E
:1093C000110011001100110001120900007C00FEC3
:1093D000008301010121012101E301E201120900E1
:1093E00000FF01FF011000100010001000FF01FF3E
:1093F000010A0500000101FF01FF0101010B060048
:1094000001000101010101FF01FF10080000FF013F
:10941000FF0138006C00C600830101011008000044
:10942000FF01FF0100010001000100010001160B16
:109430000000FF01FF010F003C00F000F0003C00C5
:109440000F00FF01FF0112090000FF01FF010F00E3
:109450001C007000E001FF01FF01130A00007C0006
:10946000FE0083010101010101018301FE007C0F67
:10947000080000FF01FF012100210021003F001E24
:10948000140A00007C00FE008301010101010103B8
:109490008307FE047C0412090000FF01FF01210084
:1094A00021007100DF008E010001110900008E0013
:1094B0009F011101110111011101F301E2110900D4
:1094C00000010001000100FF01FF01010001000196
:1094D000110900007F00FF008001000100018001F0
:1094E000FF007F1109000007001F007800E001E085
:1094F0000178001F0007190D00000F007F00F00128
:10950000E0017C001F001F007C00E001F0017F00F3
:109510000F120900008301C7016C00380038006C8D
:1095200000C701830111090000010007001E00F8B7
:1095300001F8011E00070001120900008101C101AC
:109540006101310119010D01070103010004040249
:1095500000007F0109050000070000000000070B64
:10956000064400FF0144004400FF01440B060000D4
:109570008C001201FF032201C40D07820045002563
:1095800000920048014401820C060000E600190127
:109590002601C000200107040000000001000208AD
:1095A0000400000000FE01010208040000000001A8
:1095B00002FE010B060000880050002000500088C9
:1095C0000B06000020002000F80020002006030009
:1095D00000000400020B06000020002000200020F4
:1095E00000200603000000000001090500008001C2
:1095F00060001800060B060000FE000101010101D9
:1096000001FE0804000002000200FF010C06000039
:1096100082014101210111010E010B0600008200AF
:10962000010111011101EE0B060000600058004617
:1096300000FF01400B0600009F000901090109011C
:10964000F10B060000FE00110111011101E20B06F1
:1096500000000100C10131000D00030B060000EE07
:1096600000110111011101EE0B0600008E00110125
:1096700011011101FE0804000000008C018C01089A
:109680000400000000000208010A0500002000504C
:1096900000880004010B06000050005000500050EC
:1096A000005009050000040188005000200B06004E
:1096B0000002000100610111000E0D077800860113
:1096C00032014902390242027C0E07800170004CCF
:1096D0000043004C00700080010B060000FF0111E8
:1096E0000111011101EE0B06FE0001010101010152
:1096F0000101820B06FF0101010101010182007CD1
:109700000C060000FF0111011101110101010B06FE
:109710000000FF01110011001100010C06FE000104
:1097200001010111019100F2010C06FF011000106E
:109730000010001000FF010804000000000000FFFE
:10974000010704C00000010001FF0E070000FF0137
:10975000180024004200810000010C060000FF01F7
:1097600000010001000100010E07FF010C003000A4
:10977000C00030000C00FF010C06FF0106001800BD
:109780002000C000FF010B06FE00010101010101E4
:109790000101FE0B06FF0111001100110011000E66
:1097A0000C06FE000101010141018101FE020C06CF
:1097B000FF011100110011002900C6010B06000075
:1097C0008E00110111011101E20B060000010001E0
:1097D00000FF010100010B06FF0000010001000174
:1097E0000001FF0D0703001C006000800160001CE9
:1097F00000030D071F00600080017C0080016000F5
:109800001F0E078301440028001000280044008335
:10981000010D07030004000800F001080004000324
:109820000E07810141012101110109010501030117
:109830000D0C205A519100000D0C205A4C9500003F
:109840000307206787870000050820A25F880000C3
:10985000060B205A878E0000060B205ABD8B000095
:109860002024282C383C4044484C1811101338311F
:10987000303378717073C8C1C0C388818083848499
:109880008782C5C4C7C275747772353437321514F0
:10989000171200070008000A01000207020802016F
:1098A00000030109030402040205030500064669DA
:1098B000726D776172652025735F5633340D0A002F
:1098C000252D3130732025732573000D0A547970CE
:1098D0006520273C636F6D6D616E643E203F2720DD
:1098E000666F7220706172616D730D0A0025730DD1
:1098F0000A0D0A00564F5941474552203E3E20006E
:1099000025630048656C70004E6F20706172616D58
:1099100073004B6579207072657373003C6B6579D9
:10992000313E203C6B6579323E202E2E2E00447550
:109930006D70206D656D6F7279004C6F6164206D84
:10994000656D6F727900637400436F6E736F6C6541
:109950002074696D656F7574003C6D696E75746512
:10996000733E00496E766F6B6520426F6F746C6F4B
:109970006164657200536179207468726565207452
:10998000696D6573004765742074696D6500536582
:10999000742074696D65003C595959594D4D4444C2
:1099A0003E203C48484D4D53533E00746400557072
:1099B000646174652074696D65003C6F66667365EB
:1099C000745F696E5F6D696E757465733E006B627E
:1099D00000546F67676C65206B6579626F617264B4
:1099E000206F757470757420746F20636F6E736F61
:1099F0006C6500546F67676C6520646973706C6197
:109A000079206F757470757420746F20636F6E7336
:109A10006F6C65005265616420626174746572796F
:109A200020766F6C7461676500000000837300002E
:109A300000000000592F0000039900000899000061
:109A4000EF7B0000FF000000B5220000129900002B
:109A50001C9900007676000000000000DD20000068
:109A60002E99000008990000E27400000000000038
:109A7000812100003A9900000899000046990000F1
:109A80000100000065230000499900005999000079
:109A90000979000000000000A12300006399000084
:109AA00075990000479900000000000001200000A7
:109AB00085990000089900009975000002000000D7
:109AC000612000008E99000097990000AB9900007A
:109AD000010000009D200000AE990000BA9900002E
:109AE000CE9900000000000039230000D199000049
:109AF00008990000A8790000000000000D23000074
:109B0000F399000008990000FE77000000000000B3
:109B1000ED1F0000149A0000089900000D0A413A58
:109B20002000202025633A20000D0A533A20000D22
:109B30000A4D3A20002020473A20253032780D0A7D
:109B4000006661696C00253034692D253032692D3D
:109B50002530326920253032693A253032693A257C
:109B6000303269202573004D4F4E00545545005743
:109B7000454400544855004652490053415400534F
:109B8000554E0000679B00006B9B00006F9B000020
:109B9000739B0000779B00007B9B00007F9B000075
:109BA000F3980000CF95131213577369A459BD00A1
:109BB000C5AC92BEFD80B5CE9F98745A1E1C87A07E
:109BC0008C309B1D161C0EA57CE0CEBEDC6938D8FF
:109BD0007077392B6403889871818141E509226A85
:109BE000F3EBF2823B00B59CC522ABA062C018C16A
:109BF000B9317F644E00C0402ECA888B22B3D80290
:109C0000F5A8650D7244D4821A3F628921E1575B41
:109C1000803C152DC8571EC6383C49ED72020130F4
:109C2000A05E1A45943196EC6CBEB90861B8DC9B15
:109C30004ECB9F4F4BA4DF92D13A63006F7D02D091
:109C400009FADEB755AAEF5A2D23A220A75A06EA31
:109C50004554B8591586C41CCCF53753455208995C
:109C6000AC4A234D5B4595E889BBD54EA5CC432531
:109C7000F9AC4F1A235B63BB72C863758706F38C1C
:109C80001C0DCA1A3B8C2F3438767F194E858E09ED
:109C9000ABB1DD534BEB695D9E7584CC05E7E11AF2
:109CA00000E92ACCD5A85F3AEED0BFC29DE5576443
:109CB0008CA13C508CBA69810939FAE40FF17453D4
:109CC00008C0A8E583D1C4CAC3E67C3FD14013D500
:109CD0004CBF6F00B89B322583EA98FCA6D75B0681
:109CE000F94481B1664D634323195762EA54A2DEF9
:109CF000414BE020739228CB7417C83526D150D839
:109D000032C2ED08972588E75D8021E527C831CF6D
:109D10006CE0B84E6155DC8C39B7BB9F8AF589BFC2
:109D2000CBA23CC22126D1CB3CB635DA12B33AFCE9
:109D30001FD7B44BAD91E57A01AF548E3700981C14
:109D400041962DE1F0B244052300D99F0BBB4100A1
:109D50008CE4C95B1544FF4CBBFF2A597DDC03CB67
:109D6000E390A6F061F9A604C2BE49BEC90B3AE968
:109D7000B35BD8F8C6EFD46D0F6227B409DED29B6F
:109D80001B316889C54C4EC3591410ED6AEADF983F
:109D900094ABC7DFA652D4FA43FEC980A933948B93
:109DA000609DC8BC73F7FE48CD9102C310CD8A6395
:109DB0000EEB0C8AA7615DD4D220B8514B0D72A274
:109DC0006214003FA5DB2A5846B5F4D5E3324B7543
:109DD00053B15A43F7C6A05C6ACC539EEE0ABFCC7F
:109DE000AEC76503BABDACD0F742471CAAD84DE751
:109DF00085D7118020DB9668D15B87142E1451859E
:109E00005C3029828917F705A919F07BDD1211133F
:109E10008D87DC28CE54AB52F0FB22E7AAC05E8FC0
:109E2000886A188675B766C604A4FB47878CCFE29C
:109E3000F92E36335550629D8D9AC9D57C4DE47C00
:109E4000F86C4E8829CA6EF4F6C0E78337A4D37243
:109E5000E14A6E3E57DE4387D7870B679CF702A81F
:109E6000C44FEABC1D07323FF6A8BAFCE803FE5611
:109E70003F0355BA1CD56BEADAD6006CF698B28C63
:109E8000B2AC1508AFB2B1196B119557EDF77B3332
:109E90001269659113D6372B8A82E51A3F4497AC35
:109EA00029244464A8D5BE368226677A30FEA14EA6
:109EB000B621A7ABC7FB16DF9972DB654D13B4283B
:109EC0005011E2E73DEEE3D981ECDCE5B37191EDB1
:109ED000CD6EFF91E7DE06B5197DC0FAA2B031A0C4
:109EE0005359A05FE03E8AE2F3F196E0AE564B9CF8
:109EF000CC4BC5592F21CDDED627FB5F595C06051B
:109F00004BE913073581F840C32EA1195A8C5C0127
:109F1000DF55105CFFDCDFCBEFD242EF876A997C24
:109F200056C9EA4A47856A0AE7E50D346BB84D8899
:109F30008FE9B6F086899D8FEB96C54A5AEC17D308
:109F400036F705D31BB71DF17C18D7091ADC0B4275
:109F50006E0615A688FC50E0764D0757DD0A5DC9F0
:109F600064095B24842D9FAEB2D682848351F2E8CB
:109F70007C916007F0A5E4C5B7ABD7C567970AE643
:109F8000F3268446031E57DE74490724D954021E63
:109F900081AEA3D638270CCEB3C839BDDDCB11AC0A
:109FA000EFB4385D889802F3259E9C21B1D763CD2C
:109FB000EB1A196E79648CA7E15158ADC6F4EC52D6
:109FC00075A521AE60B8FBADC2380683FA39D1F56C
:109FD0007BE77BC197C7B270B1EEC64BE3C37F6C22
:109FE000B83E554BEB93A9D0098FB89488053566D8
:109FF000EC9834E7AC21A2A4BA5D7EB8DE553800F7
:10A000008C74699040EF8779810C8B5936BB1B4665
:10A010002E03201397C1EEB94BB87460EF963BA4A2
:10A02000CB8BC0A647D5C10F6C1736F7D98494FEE9
:10A03000E6A951D07757D767EB8274120DB28988A1
:10A04000CCAF9655551BE5BC67BFED91909C3EF19A
:10A05000947D3C24820CFE50F2084EF960B496E4E4
:10A0600090434DCCA7075F24561AB3BFDD8A5338FF
:10A0700001D205C96A129EAEF52589AE00582AD5CF
:10A080008DD796B5397551F37536C45AA05A823FAB
:10A0900052199C61407E7D3829BD6784E6AF6B18FC
:10A0A00037A5692BE47CA00262B20266CDCA06A184
:10A0B000BCB8EAF49C96892918A44DCCFCD6B3060A
:10A0C000EB6CF1BAC37137857FADBC3E8E10F45492
:10A0D0005274096F18CB29ECD46C9A8B6032B4D9C6
:10A0E0007E4C590F662067F1070F7D67E3189A5978
:10A0F00076EA1A7670E4013C9B93F1736435F10CB7
:10A1000098BC59DBEC1525973DD80BC7E2C05A9592
:10A11000AD3FDC8734E47D3A2C8CE1C6F5426564C2
:10A1200055856D0274D6854A32034481CF95562CED
:10A13000058F8681C57FC173342259C577CC91EFD5
:10A140008D5C789A7C8463A7AE78800F6CE6C1360C
:10A15000141577FC28FAE8EF474A387804F9F397A2
:10A16000D28E5B9DCBAEF4E2CAC2BDF54BEA46325D
:10A17000AD787636E5A99974438B157B2AA4481AE5
:10A1800021E44E5BCFE2DC00840A9648370A636A1A
:10A19000080144917B87E80B5BC08FC651995048FA
:10A1A000F96DB9B261723EA5988A2BCDA8EAA7C312
:10A1B00035A4B20F7847171E0594590DACF91AB89B
:10A1C000AB579FFD9A7DE812A1F308BF02FF6544DB
:10A1D0009EC2B5322C675B27DD47FE9AD87A140AF7
:10A1E000B95F759FB1FE0003B8903CFEF4B6AB9921
:10A1F0006E0E2EAE3ADCA5E696E5A956FAC1952676
:10A20000640B80486043E6243F8545FFDE8CEA5EB0
:10A21000A7D73173E077C3A5ADAFEE01F56EC1FBF3
:10A22000D5DFD4E68B402629B6FFE8D4C3A35FF878
:10A2300058942C7B9312B8DAF50598654C1BBCCB6F
:10A24000D36B1E3CA5B60ED394DBB29F7159B9E611
:10A25000D8FF4FC1BCE6FC8287BBA94EE770E7BDC3
:10A2600009B4CBEA948B536A988ACAA6D692FA8626
:10A2700080BA6604A774BB640595348DC4437E4DD3
:10A280001BCACE8141E9FF5C0046DC2C1C9A561E9D
:10A29000F529C10C781B19B3C6B10FB175CC4E05A9
:10A2A00013133D80CE0DF865A0AA9909262370FEF0
:10A2B0002488BE662E4F8DCFA6C7F138E75F0A33DC
:10A2C000BB1C595E2D8BB89D152BF55A220F3C34C3
:10A2D000BB5119130953F7A590409E7CADD62E466D
:10A2E0005064CFAD15787F989F3226429D2E79031A
:10A2F000EA21F68724EF6B862AB5AC88A339E2649D
:10A30000521579CE0FF990E3D1032F2C78E9AE6482
:10A310003A1359210274FB4D674BF8A7AFF1569ED3
:10A32000C83A7114BC6D075A0E6B7729B77CC02DE3
:10A33000BB51CD5FD65D68CE7544AA744EA78DBD66
:10A34000D4842B9FA49D1B9DDE5C099E4205DE9C50
:10A3500053EF933F0A549282390E87661DD59F3082
:10A36000425FC2919718FFFD8742A5A420C5F1AABC
:10A37000939D37BE92287DACE1C756BBCABB377FE1
:10A38000DBBEB8EDADA3123101F356B264E68BE843
:10A39000FC6B1E481909356FB04725F72D283C5C2A
:10A3A000056F76C6F0CFC67E6087F0BFAED12E1F98
:10A3B000ACA5A4EAF3621A8E65774AD61EB402876A
:10A3C0006DC30012BEFE1FC3AADA44CECF9F94D83D
:10A3D000CD9AA06106E11D2E0A1B1AFAFAE159DD99
:10A3E0006A987F31FAB24B800382526BA4180578C9
:10A3F00091AE1AA7EFDAD4F99BDD115FBAE11638F6
:10A40000E73C8A73597FDE3C7A9107BAF34702FA38
:10A41000BF589D994BBDD6DE872C839001137E8556
:10A42000AEFB108824B3421499EF9C3572F9F5AB5A
:10A4300018AF9F6C881439A5E67859FE876D2847B8
:10A440001612F90A459608A772B661E4F222165D63
:10A450001FBE63BE610A60B4FAF9DDE527B5B5F445
:10A460004628617D50BAAA8D493FFB470FB4CB7A8D
:10A4700054F54640654927F70084CC682DC90D3B4B
:10A48000324D41A2F4E1D580DDC82E7FE7299CAF93
:10A49000A7F82DE2E6469C49CC93DFDC480AD8B504
:10A4A000D2CC8079E8D87F730E6F313886189D2220
:10A4B000DC0A53217457321313C3E9FABBD26090FC
:10A4C000D72ABF47246B33E095ED094E3699868035
:10A4D00047A1438213E1B7E9347995FD0FF17D8EF1
:10A4E00046B09790115C4FFAD2CD037C72994887A1
:10A4F00096879949C79C81798855C51A76DCF5C13C
:10A5000035FEB1D49B8C871B0481AD0AE7D94292FA
:10A5100031D0D4CC7CB2789CE217DE8E58F0EE2697
:10A520007194AF2F9AD31B2114A6392F5968A2BD5D
:10A53000247F135321D0E2BAB15869C79BBC5F6E28
:10A540007B1C437CC6DE6763A50C705AC8387770E5
:10A5500059F0483F1B54D147877E1A9950F5038420
:10A560004BC99548D40976856B0A79E1193354C3F0
:10A570009D9DE5C82F7A99D332FCB8A5D60E155902
:10A580000FA9C3CADFFC29AF31305D8CC499E63D09
:10A59000719BE5FD5256C6DE9E0ED283318E619DC3
:10A5A000019117C3B934BBD0FC854F25EC75FC1B5A
:10A5B0003B77AE8C583306719A78DC3ECC6290388B
:10A5C00001C6560B94C018EBE5484E6FA761CCD07E
:10A5D0000140520F0B5E22A98A775B26F589CEB720
:10A5E000FCFB6A9BE15EDE0D4D587FC55156855FD1
:10A5F00020DB7DAFF090A5E185BDA9FFDFE227F26A
:10A6000040E9A02BEA18EF79A21A70158433E9DE2D
:10A610001106482D5211AD860921147C19C7AF5A75
:10A620007AC3086F2AD9173CA2271789556769D5BD
:10A63000CB136539670EEBBCF47B8EB4E8304DFA72
:10A64000D165337B6A833175D6883F7B9104A21034
:10A6500033BC6269262213E4775B76197A6A266630
:10A66000C9564E62D8643E14CBE8CDA3C56B5D3CA1
:10A67000D50BD9285D9CA4AE2D9D549955DFD26889
:10A680001F567B9F28EE5B93F483EF11F549A8AC2E
:10A6900036A0BDAC32872A0D2228D377BD807BF34C
:10A6A000923E42C8BCDB44DA9C54C17FE98AFA80FE
:10A6B00092F8830841FC3F1F5612B10132CD1F6C46
:10A6C000F71392761165FB68BEFEBCCECE4446758C
:10A6D0007E614CF25CC76DBA81098E639E2BFF9937
:10A6E0001D01BF953969C10C2F2A43E9A7ECDA7522
:10A6F000FD7185ABF343B2EB9EAD3CCC4F2E8A543B
:10A70000050FE25011F630F8B72E7E8FC12FEA12F6
:10A71000F9CC4C961B860980F8C2E24155FA2DAF60
:10A72000D6145B4EA22FFAE4E2EB8DA6B1E6D4BDBF
:10A73000D996AE95A2D9A304EE9CB9D1D2ABFCD2E6
:10A74000150B95E3B65B78D5052600755CC0E12B4B
:10A750001A7B13A7AD13AA71B0F1B50AFFE8B4CC08
:10A76000FE1EC95A1C02F7DE13649CDEAF8F3BFE4F
:10A7700055E30B89478D5D482CA3389553E89ADA49
:10A7800091EFA62DEE73E714458AEF0E8147971BD4
:10A790007198DE122A94679B4AF329E8311B7933BA
:10A7A00033D3D2604BCDDE37E61D7482874D106EF9
:10A7B000E903FFFE8ADE8483069D6B1C4E3316D9A7
:10A7C00010346E09A9C152107D8EFBE07F203651F6
:10A7D00039E969037DE1E76902FAF51112AE857A7C
:10A7E00023F497BEB00D4CD6B636E78B6D98F92999
:10A7F000804D6FF51813CFD59394E24342368B1FEB
:10A8000047C5C822E7727ADA1FA415B83F5B8E3FAE
:10A8100056D408A1BC045B0DC4CBB202AC90D49C4E
:10A820002DC4C3B4A7650058FB0A3A82219B8DC092
:10A830007A542E80B9160C0C0759D742EB2BA4EB97
:10A840006877B64CD7B42EF24E2EFB52B7F87D0087
:10A85000B9601F357CD9E16BF20266329B4B4D9E8D
:10A860005434CCA528371F04315BABED46A37F7170
:10A87000971A1083C1B643C35655B19C4D921A65C1
:10A8800081D1D1BD4DBD071C8C5E1E99B0CBBA20C5
:10A890005858F65C10D53BB7E1C82C05015C18414F
:10A8A000AA0B62D12FD13431A7DB92B45EE863C822
:10A8B0005E004809DA33C553BAC662E58E89EA14E8
:10A8C000B181BEFF3DD71040E24AE2345DBA52B5D5
:10A8D0008D5AB60676C96F446511644D656C6BDDA3
:10A8E0007FBA8F4FA4F64985509D9DC9456FE5738A
:10A8F0003053EE3692B6090D9B37F7FC7501D38FB6
:10A90000D8830A63B386DE4B0098EBFC4769A32D1E
:10A9100038E9FF283B2273BDC15662E83FE1F1D51B
:10A92000093635503F19D4389FD0A976A5C0DFC06D
:10A93000A9B3E4D24A5316E254E33D38C8D17F4369
:10A94000CF439207224AC0B94D1EED3AEDD42A27D3
:10A950006236855A6CA504A4FBD6B18CF20966F860
:10A960003BE334D72398899E30D96C11E0F1D47D34
:10A97000055B2A27F3197AC1AA505395FCC89F1783
:10A980001BFBE313EA00A9E6B12CA0551ED2BD467D
:10A99000277D231796A75029A1A0724C84C23B356E
:10A9A00069EF7C56D769343A661793830EF44B8F60
:10A9B000E9A07E63AAA49F0A93C5BC740036CEF9B1
:10A9C000F27775B9A0A32B5F485DB621A6D0858428
:10A9D0004F912361AC4B565F38F32EDCE003D13C42
:10A9E00090FC6B053C2E887B625DD0A03237D2F79D
:10A9F00017657E44E12BBF85A75BE6FD51872C835D
:10AA00004B8E7E46976D68309E9B1D8EC810659953
:10AA10005A33ACEB48749BEA8F80A0C0BF6B53D213
:10AA20003625C47BF217842EA7DF5E1B73A7800533
:10AA30003F722D08B33AADC0C66153F747B868B549
:10AA4000A82C5D79D3053FC3534F5503845C08D0D0
:10AA50003175E4D16291E27B0C61AFBBAE7AAD0996
:10AA6000B70D5FCCE804E3CA8C57BDFEC8B392D1E2
:10AA700030240DB56F1CCC0E2326E48109935BD2E4
:10AA80005E20616B76649AC26A936E436888800523
:10AA9000DA6A76FD73233E906D7813E6EEF5B14ADF
:10AAA000DBEAAD81ED0EE0E6BCE931B3942B26374D
:10AAB0007F0011130E2367D4159C8250BD6F5D86F5
:10AAC0009A4C242A28616D93A0BD09E552763EEB8D
:10AAD000D02DD648BE1D4BE31CBB6A7E9E84E23857
:10AAE0007E7B84DBC4B9CC8DB9602B0DBCC55CF614
:10AAF0009270679F43744E0D299F9831B17C5E9C84
:10AB000059E39E22645EABC1DFAF36289285E89A96
:10AB1000B862B7729E83B259E4BD3EB5E128B36F07
:10AB2000D359566357E7079889B38FE5FBA6AD3233
:10AB30009393C8D7542D3C6CC1D47F39D20A684056
:10AB40005A0A2335DEF9457081B59A0EFE946E3FA0
:10AB500052DA307F5CBC8213BDB9FCBF246A43DD8E
:10AB6000F00295671080099562D3D53507EF7A79A1
:10AB70009E6E8A50225DD8A4DB137BC6467E793355
:10AB8000CB0FEDFA38BA81293C01C5CABF979B8E1D
:10AB900058A181664FC15DA35747BE64B14B0851B0
:10ABA0007FC639996796326FFFDA9A1B51CCDA7AF1
:10ABB000E601BBCD09E0CA6AE52E6794E6B9BC0C94
:10ABC000237AA8C26C6EC0E0C2FAAC9263C197C986
:10ABD00064BD7C4C942F86C1D86E7207671BB88108
:10ABE000F4AA95D809BB63D75B5219228510221F9E
:10ABF0002F0A350796EAE349B0F2BC6987D906B552
:10AC0000B0C674FD08F4A258B50BDB81502F55AACD
:10AC1000593481E3BCC9FA16EF52825F78155E3E63
:10AC2000D230D159543B7FBFA0BC9C1A128F47B978
:10AC30007D48BDCB0494C594E95D48D6C3AF1AB432
:10AC400062198FF75018346DD6E72F91D629081D59
:10AC50003DD2713FD13C2E91EABB27E38C6A234859
:10AC6000F13D4F9038C6E6BA321BE422396A54D21D
:10AC7000AAD3898D8C56DB4F965B9B92537239F920
:10AC8000E5205BF8F3E870734CB3D1A690C47BD495
:10AC90002DD9D4AAA8DDF267D8122E0B3411A72023
:10ACA000CE9E356EC22A5F27246E33820D016DA7BA
:10ACB0002A4C7218A6BA9ACB87D5DCFD7C8D9E3CB7
:10ACC0008A90374575DF4E1A7073B9879CDCDEDDDC
:10ACD00009566FA457B6DC8501040F67E51186ABF2
:10ACE00001001ECAF1C891D900585D0C786DFA6F49
:10ACF000B0AC2553764B2217E1A04A632987B88070
:10AD0000C4F563DDD79B38119A728369E8B95E2870
:10AD1000B8EEEF184B5C065752DF3D288B4D17F20B
:10AD2000FFC0E3BCD5E6302E288C6ED6B630560276
:10AD30002C7FC66BEE35CAC5E579D9F5EDAF491A5A
:10AD4000EC877AD7E872B716504AF0C901003ADFAB
:10AD5000C6434B1AEF2C6CFB36FCBF7701585B5F88
:10AD60009376949490E249F3BBD245728435F7E828
:10AD7000E87446324F968E4F01DA0CFF74C2242ECF
:10AD800074AC3241166B350227B08C9A433EDBA778
:10AD9000C40D4503172026377BAB0DB80258AE3FD4
:10ADA00027DB073A8D5B4015E5BF9BA8928A769515
:10ADB000FDB346C8D07F4917F28B677E6E2CDFF556
:10ADC000725506F276EA651BE91B59301F86600B47
:10ADD0000DCC32C42E1280835C9FF2A499F5EB87D0
:10ADE0002710CFE0F8E76A98C882A2CB387DED59EA
:10ADF00034D0B9F19A665D66BF063F23DDCB6D4E58
:10AE00008AED716BC682A39C904DB48F3A29B62708
:10AE10008A8C2943A262B3169AA2EEFBDE7BC55D43
:10AE20008B8F305B5338E1AE5569A2AB0C91F35672
:10AE300099525A07F0F46EBA23DB55487B3B46AB78
:10AE4000E537161DF4EC499C2962174EA0BF502A25
:10AE50009600C364A7D4BC053BEEAA53C0F0B3D69A
:10AE600066C50D42807C345A65CE5FCC8780AAEAE5
:10AE7000BF052992F298257F832F26A2CC1463D692
:10AE8000241387E9CE293C0F4ABA27DB0E6E27A48C
:10AE900049AEE15F8AB8C329343564FFF61AB78436
:10AEA000016691519196EB9E5DAC45F6C65E3DB153
:10AEB0005E9F5D9C129C5F32EE877EF2D4C11EE5E0
:10AEC000644DBEAC954A9CDF4D77DE91A5FA4327D1
:10AED000E31D926E01412B417F7B02D0E8FA3AE1FB
:10AEE000AB9FFEE775CEEFFFB9A574CEC5ABCCA87E
:10AEF000A5B43FF29D291A383BD4ECBE32C959C3E0
:10AF00000991B6D856DAB06B098080E32789558954
:10AF1000832B7EF09169DB794AF7139AAEC682D80B
:10AF2000C00259A95176CC85835FE3373AF937518E
:10AF3000F78C1963A95CA12F722A15BDC125A39AAC
:10AF40000CF50D50B1F9D0FA3BFD8CB23B4E753C7F
:10AF50008C0D2F6BB97A628449C523B522DEBC689B
:10AF60002358B1A3760FA3D8C35AAD3FABC7C6F9D8
:10AF7000C60A36F948E52ABDB4265EAEE75EB87962
:10AF80003A38E8253EFFA60ADEEB44CAC58E7D208E
:10AF900096273FEE1C2E073C1B66BD80BE9EA7DF9A
:10AFA000643764871B1371FA0E491CEDB9DAE3B0FC
:10AFB0002C60EC4966A064F01D0B9C0E9672F8069E
:10AFC000BF527716B52D600049D1A22810657A4A84
:10AFD00066BF41FF9CC464491987EF080777069C48
:10AFE000E74AF2FC8222732D89C945C5D3082A5B42
:10AFF0008806BF19C443E19819A8B8AAEBDBE79308
:10B0000030E4F7D98BFFC4D48CE18A131D1AAB311D
:10B010005C55482C06B9715F62B4F3BF52FB4258CD
:10B02000C5CEEB2391D2FF85A31ECB23EF965AFF0B
:10B030008B7203FFD30243AFFD7FC25D4EC9107810
:10B040003EF9CED0D3558650BD50DB32B5D500B1D8
:10B050009C1BC4A015D1ADD5CA98311D02C9310DB4
:10B06000E9B4E01F60237FBDEBF8D0311E4BFFCA6F
:10B07000F246EA5AFDCAD04FFFF7813CCF8C3FF928
:10B08000FF81D9F2C67ECC5D827138630289285D6A
:10B0900011BFD6DD904EDCD484C95C8D6F52107A1E
:10B0A000CF48BCA550E20659399FF77B43254EC6D1
:10B0B000F799BE6841D0ECCB4A870B990267F5E659
:10B0C00050071D96F9DDA7D7C31438D62B0486A6E2
:10B0D0008DCCFF483EE6E3061F87180EBFCACC653D
:10B0E000F39E8ACB189168C57BD3700572BE8B83A3
:10B0F0002BC2746560DB9901EEF5AA4E2FB048C9EA
:10B10000D9A4B6C3C03D421BE558CCE44DBB9AC799
:10B11000ABE3B5180FEE3EF20F279F625DAEEB9DDD
:10B12000005F18FB914D030935D250634FD1547322
:10B13000BCF1BF50C2CB37C60E7C12985977F4EAE7
:10B14000C977B79C08AB017E7DF5A961048C42C923
:10B15000BE45D5DA318497CFF0CA3B4EDA57FCDFD3
:10B16000C497FEA687104F1CFDFABCFDCD3C4D05D3
:10B1700082E5A56B56FF43A81E3EEE8717FA348280
:10B180001C10406BF8F58BDC2BD6BB8B7DB36ADAD9
:10B19000E48B3EC138E4444137FE8787F946257584
:10B1A000C1BD6CA1FDA7F5C7C42001211AAEA8AD91
:10B1B000B299C7F87BEEC2771B5283220E2A939D69
:10B1C000D3BF688E374CAA34086F3F1D20C09C8ABD
:10B1D00074B5FAC82CA5F6A9FD2D2B80C9C64EABB7
:10B1E00029BEFDE6124A2B9709711A9D8239508FAC
:10B1F000246B3E6BADC2B5BF24C78AC9339A00EA3F
:10B200002EA22D661E6C0D16609E27B14140101EA9
:10B210000B311148031B2D507380576A77C519ED08
:10B2200005A52684967BDE658A53BF1220DBF213C8
:10B23000AEB871FD103EAC323BBBB348E17449E59A
:10B240009DC08B20D0CB0D53CFD365FAF83D9C6DBC
:10B25000174CD9072FFC94412DAA3AABE8AB739158
:10B26000EB45EFEEDEF7F43D1F6A2C9189A7EFD393
:10B2700005BC3B802B63FFA89F7644EB9D0896CCD2
:10B280006AE725E01F8E3D6C653503A868D829CD97
:10B2900025E54AAFC2F10B6A2AA03FF4D474BBEB98
:10B2A000D267F992AB05AA6AE25ED407298C3E7395
:10B2B0009AD52D756075D24BA158AE2F4C8A5999ED
:10B2C000D42F643E10F04F50BDC819F508E8B238CD
:10B2D0009621936B568C98CE43CD976DBA2B8DA348
:10B2E000DB215A95D1B6953AF6E6BFCFA5FE17FDFC
:10B2F0001E46E6C7AA63A8EF242AFF0DE183A8969D
:10B3000021A0861504041F841115032B099295684A
:10B310001E01AACF91BA8FD077DA08884F8BCC1450
:10B3200041952ED5C3CA69CCE7A69DD9DFA4C672C4
:10B330000A433C3CFB7BF726AC6CAE21009F24D932
:10B3400043912D8BF9A6B893A245EF7355090AE8EE
:10B35000CF053A70421892E6CF005F4C1B16682D5D
:10B3600097288A683E43F2CC6C6066042B5FD1B2AA
:10B37000835987FB8B6380D2578F27C07E7ECA910B
:10B38000DFC0B219EF8B67A0806AB4415B8EB5173E
:10B39000DE7AA456F24614CD3F772E9A95F27B7250
:10B3A0009CAB575FC177B401644168EA4C1C76AC32
:10B3B0008D59AEE21C5EC76B8D25D9C3BD1D8E15A0
:10B3C0007DF0B62B3ADD3BB37EE0DE2C1615690628
:10B3D000946BD89731CC8E98D6A4874710116120F2
:10B3E0004BBF35EBEF734D23FC103625BDD097BC1A
:10B3F0002F75378F78A78452BE9A2E7A8B6D4A4A62
:10B400003753F6C94860AD04E72C3526B8CEADD227
:10B4100005C412D515307487E833024666621018E9
:10B42000DD6712656C35560BA7300A8FD2BB1AA2A6
:10B43000B64346346231E531CEEBA5B98212A11094
:10B440009E5EB88F24576B974EDE917D8E9B35564E
:10B45000107C6BFC03A5AC42A7CB83DB1A92450F93
:10B4600020D7AF41AF2B6F28B4D0DAD185A25709CE
:10B47000F7AFBBD0B0FB4A650E9EE26A1D6F962403
:10B480008C1D3FB6433289112E56537D11A184ABDA
:10B490001CB843DB3BA60F1D5874ADDBCCF62F1058
:10B4A000FF6E9E2B9D6B5FD34C5509153030CC073A
:10B4B000D336D1BEE17DD02DF14794B61691112936
:10B4C0000EB3E89E59CAAE71C3E837E6952BED7E00
:10B4D0005DB3281B9325FF27BC3C2C6E57DE4088AC
:10B4E000B46B4B0F3505F26C78280B93C40843C03E
:10B4F0001406E936C50C76BB1D1FA724BC1C75B30A
:10B50000DB15F34C8AAEE5EBC35AD46245DF04DEAB
:10B51000D348C94408CB1ED5F8D5896048C169B065
:10B52000F621FE28A4AEFD1160A51342804FEF5115
:10B53000636767C4FF85FF5B4D8446DC0FEE3170A7
:10B540009D84ABAD78F214AC6EA3106C7B53891163
:10B550008EBC970CA8FC27410F48F58E8F264E5ABB
:10B56000CFECE0BDB3D310895520DFD78FB642BFF3
:10B5700026C19776C5AFE847C5470FA8A1BD564776
:10B580006770A8736281FC0DAC03997D3DC81F678D
:10B59000C3634D5F553E3E630BA9E75763E707F76B
:10B5A0007826A7939B538E0E9F6907B2DCAD2D09B9
:10B5B0001B0817DBB3A5F689A83B5DBDE6FE9A34F0
:10B5C000892A570FEF6717DEC1FC5557BABA342ADC
:10B5D000528D5DB258D5A89852A89B164881D6FCCA
:10B5E00046BA0EE7F789FF1C7B76D5667BBFB1961E
:10B5F000EA5520CE6C50BA37EA9EDA5DFDE50A6A5C
:10B60000C6396C0909F94797F23A4A26002AA50F6C
:10B61000EE5158E126657EADDA504C29BE0C7630ED
:10B62000C7AA384B5ED087A63BB7F380D2505802EA
:10B63000E8A9E2B015ABBC1A97BDA23D0A23CE061D
:10B64000FFD5DC311E611D37A01BCBF5E4835BF811
:10B65000B65ECE9B3EB8EEA1E2785A67B892949F50
:10B660006C2620368DA8FEEA13F3D2C8D5728387E4
:10B67000E2348919C666D1081A23A5122CC746E6FA
:10B680008707BD06A75752E0177283CC21D475E80F
:10B690008DCA962EBFF0C9A2C324DF3D933D7D8E97
:10B6A000149C06030B9CF6481B55AF25190CEE6342
:10B6B000539EC13DA853D22B76F254F1497C5B7264
:10B6C000D621233CE00AC9A3F89B76EF69D36B51DE
:10B6D000462EF3FFEE5E7AF8FDAEB634123B72589A
:10B6E000612F8CB8502679BD0450273758E26A1F65
:10B6F000CFBC7C822BE2F88CA5BF9066D745FA437D
:10B70000FA5CB1BBEBCBB0B57B16109CCAA9405418
:10B7100080D3833088D082665916C09912A55B7396
:10B72000DC1D0434ACFC0330E5DB7B20E184CA0E75
:10B73000DDB4E3C064185A9835A8BB609AFDC433E1
:10B74000BBD008C33E3DE08EE597D236A5D68DEC42
:10B75000B6267FC2AFAB651ED1BEC67BD1F2D8592B
:10B76000AF61DBA4F6ECA1C7452E81BC3F02BB8FC5
:10B7700092EB1604AD747294DAA88D2B5CDEF15B4B
:10B78000678D3BF9E75C357EB3D1169191ED742757
:10B79000EE59F1EE4E2B099CF5A26A9E8705B96E13
:10B7A000DD26B530C0FF61C4DB7759A44CDC745989
:10B7B0005697110F6D11E8D0A15549EDE05BFD865C
:10B7C00041994BBDCC54D52A59134CAE11AB9FBDFA
:10B7D000013C8D18577A65A184F5C679C6D89022A8
:10B7E000CD5B4FCC209B25D5B86BF05CFFF82A4E83
:10B7F000A3F56FAA93234641A1D0D36FF3B513FBF2
:10B80000FC17DA0DAEA2623D4EED927DC2B1372437
:10B81000E040E7EC98C05640FC43E45053EB022272
:10B82000BA5CC76B1289D4BEE373BFD11F1CA9DCFD
:10B830006C9D4BB3348EFC4617C5A6264882ADBE20
:10B8400021BFD05F31709E16D17EC1B7996691330A
:10B8500066FF85095EA07C6331F4FC511B0F379AAB
:10B860001293C9FCA0414884431B87B4399F0757F2
:10B87000325464702EC5F7E2ECCEE65CC508B40B1A
:10B88000AFB56991FB1ADE15064EC926E9ABC87241
:10B89000F84C5F001AA3B5DE7557D98CE16D4E07E1
:10B8A00096214ACB1AFD61B8ED1C5D64ADA1663AE4
:10B8B000152157870CC693A3B456BABE1023F1F7CF
:10B8C000A514DCBDB61102563E72CE467B83987B32
:10B8D000AF9668827B5828680841B0F5259E8D7127
:10B8E000872090F1C97EB315D656718B63FAABC130
:10B8F000054DA0F3FC83043C108EB0C001E86B152D
:10B90000EF21EC67AAB8ED6A296C42B64D2051319F
:10B91000BB11F82FFE30910749A36FB8070DDC6DFE
:10B92000485D912B46A0983E9C3121BFF2BDF1337A
:10B930008E5655387C64675C95DE71EF3F5EA6A835
:10B94000026AD5E0934A7B0E80BB42E261DF484D3C
:10B95000886045CCF75EA7D8B7748AE4E6ED8F7FA0
:10B9600043A09CFDD698411ED25AA6D4A58F42086A
:10B970000D1BC07407F3E005545DEC4C69E6FBE772
:10B980002E905515CD64CA8DA84D77DD720E112EFF
:10B99000B258089A0E784D2500F51B605B942D086F
:10B9A000F643BAAE661365611249A7F60DE79BA48C
:10B9B000865E1EF6CE44729F9E769E95742437C88E
:10B9C0002F783DC635F953C4ED948A13927DD9186A
:10B9D000D7696E09E79D251BF3B176F56220CDAAE4
:10B9E0002704D3A11A446F68F45601A3F3D1BD8094
:10B9F00074D19C47C75388115F599ED6BC317E30A5
:10BA0000131E2A8E86E3B71E06E9D41FE39766A5A8
:10BA10001C39A4313080DEA175DF7251F3087E6DD0
:10BA20004E7F1591F5F8DF65A22C2697936C90F464
:10BA3000A1AD65AB8CEA40355861DD76014E68FEFC
:10BA4000694AA0C8CAC0B08CF36163A2A6EDB7EF83
:10BA5000F4DA00DA3AD4A17727F90F13E29C26A88A
:10BA6000B8C6ED0A2BC0F6760B2537A27D90286E5E
:10BA7000ACFDB80C4F89EFEF985D6518E81A78199E
:10BA80001D81E67158987A5079CC65E3D800253548
:10BA9000132658894CC2E8E3B9C5A3BB5B70524476
:10BAA0002392A2062A4426EC73A83A0841F680FAAB
:10BAB00057D4A1A41BA82DC1B8BED391BFA985910D
:10BAC000AFF2E163FECEC6F4169203AC1123054B30
:10BAD00049FA36677FAD12ADBE8E70C761069633E8
:10BAE0001A03507625005E522670E31E25ADF647F8
:10BAF0003B96A96CA51FEBB8E2C2903D86376890D3
:10BB00009DDD7838B395E378BFC6684E958174A6FD
:10BB100061F596E8AC84DD6C11778A559E489C04EB
:10BB20004EAC5A6C41C639CA5BE26DD940EFDFE8D2
:10BB300039C4794AD980A4D3A7F1803F4BE2773545
:10BB400031BEEAB963C1C480725B0A81357AADC582
:10BB5000FE544B2566AE9A30EACCBF05311ECD921D
:10BB6000FF4908CF64DF18F8F536B78F87F6372E10
:10BB7000924AFDD26B7F3BE76F660600BCF5833AC5
:10BB8000ED879779348E9E1C9A4920939C2D6AE804
:10BB9000A2A8C981BD04054DA79A81C0809C1B390C
:10BBA00044A00D8592100F883258E3A9715B3F4F76
:10BBB000D5992F56098A4C145B53870290B168BD02
:10BBC000976EB5D7CEC5A20FB1232873926D36E616
:10BBD000C0204CB8AC1E64AFD9076F81A470889A9E
:10BBE00077BFC0FA602FB93BBC5096D92E86AB55B3
:10BBF000E068F77EB2839A3D7C1660DC9A2B058E56
:10BC000007C861E70B100EA85C0772D1CBAE42EA01
:10BC1000010A99D37D0AF80D55EF17241F2DA0B303
:10BC20006457BCDEBFFE6967D8CF0BBFA237E331D4
:10BC3000C604CC9070403959EA71ABFC5879213E6A
:10BC40001D86E469BA4167463C99D29E172F80D57C
:10BC5000D256DDF6BD403702D72A587605D1246A80
:10BC6000BE81443662AE7CFEEC5EA95D3CF6395383
:10BC7000DF7C0A62638620688949E4BAC7A356EC70
:10BC80005EA5A1D7E3D5579635A946A4916F1212A8
:10BC90004BC0136F61B0586AC54CF8B7234C8D1078
:10BCA000FAFC9A57001238B2091B961FD550D5D509
:10BCB000E20F701A0103D4FB2CCFA05E8CA34FBA05
:10BCC000A426C6BB0E80A53986A4577D8ACDB59320
:10BCD000B9B303DC8ED86A0ADA95F272898E80D203
:10BCE000C232C0EE8B7305A77DCD8B57F253067A17
:10BCF000F73550D7E25865BE4C63588AAD3F2D6E7C
:10BD00007D6CD0FBC98A8F6FAADD7827141156DCB1
:10BD10008B0092994BCBB761E4B40606CB80F8F464
:10BD2000A2BE1A6A2F28655AA19E9E8EEB89854075
:10BD300023FEC607E31BA89F701E7BE9D077FFE8B0
:10BD400011A64F69D2EFADE8359E580446B7558726
:10BD5000D81ECC2E6865DC195AB0D23D0D5C601B34
:10BD600052E0976095BAC6A77866A60ECEBF673434
:10BD7000B71E9A38B664DB716B90D4673A27595175
:10BD8000597ADAC8EDC8AA8196B430F73E4FD26628
:10BD9000F536EBFC18A789DB5D56A14F94CB16ED69
:10BDA00064CF9ACEB0E0B6774BB4003E02C3D31D49
:10BDB0003DE20FE7D7F9D6F4896EF44301FE33BCB8
:10BDC000E312E61DCAE3959EC096C036AF6613E641
:10BDD00062DBCDCD4ADBFADF42575936ECE1E65162
:10BDE0006BB2CB8A948CE39F22E96C22D03A4AC989
:10BDF00021FF48D78289F47B5FF06170EA1B78FBF2
:10BE0000FA20EEAAA7F769C3827482AF2846A7205A
:10BE1000B5BE1B13DD0AA3D51C62B1CABC4ED31933
:10BE2000ACBDCE68B4F1B60E4F981079A9FB10C323
:10BE300023CF758CFE14D68FD1A4A2A06AA8735903
:10BE4000A1A018A4BC1FFBB9C7A55CA110185DAACE
:10BE50009E935F6C2E1AD2B6470FB3D4D1B4335031
:10BE60001539F814E079193767D5D47996406118F7
:10BE7000CC3988050274A70D4A65C8D16ECF04E796
:10BE800048D7C75D684B7C29CDC3DC9F0A5CDD5F6A
:10BE90008AD74C3B434EF0332D0DC53B9DEDF889C1
:10BEA0009493AE40854B80B6D04112B2C93E4283D6
:10BEB000269FE3BF23B6274D0D96F0D8CC45D3DEA1
:10BEC000FECFEC434FB775607C93E2F2E0D6B587C6
:10BED000F3B0A227ED8B79EF41CD0DBED3D5869976
:10BEE000441B99D859480A97DBED9B7AC7A89B4F0A
:10BEF00030AFAD6E02131D40A9A0750C596FA86F2D
:10BF0000B19CA15A6554290D33A2AE75E625F5E022
:10BF1000E839839811F330BBC4CE9E40C9BE3613B6
:10BF2000CA870B0F2E75CEA872520998D8AFB7C129
:10BF3000FE1A3BA4EB5C0644C5BD0E4B1C54781C9A
:10BF4000FFC7C434DE4E84FF5BED6D28C8366059F0
:10BF5000983F4588F5381C7625D99D829B454EB47F
:10BF6000A31D59E12C4F2F2CB7C5662F694109C776
:10BF70007D65B14C068454A406E7E3AEB46A332F62
:10BF8000B0D3631DED7B9DACF2DD8808F02994B33E
:10BF90005974F1B950624C36600B3253E81EAF53FE
:10BFA000F6B5EDD68055DB59575C71CB70990DAE67
:10BFB0006F06C2613242F3F772FB72F36E1D2D20E1
:10BFC000205E595917E895210D1A2D5BDDDE5D477E
:10BFD000A2AEEFEC9CEB66243CD6D24D886E2D755C
:10BFE000C648349B08F9DD3C601AB03DCEEA2654C1
:10BFF0006845A0A796D4C96431C0BE31FD13A970AD
:10C00000B8043ED89D4485024610778C3C77AFFB40
:10C01000978AEA1E833928F1B586D68BAAF698C48A
:10C020006787871572EFFCC379E9E033476B8FF1BF
:10C03000F454B901E1992A1D4FD94CC35F9A2C746D
:10C04000876A0659DD769A26AED32B1506BFC7142C
:10C05000F72AA09536A98E199006D07BFD24D79794
:10C060008A947A2760EF258BD8FF9C775B9EEE6BD6
:10C0700001787976DCB0CAED9E765D06338C455A40
:10C080008D0DE14863926A4C4C4A15258CF704618A
:10C090005E11CE2F67CDBB9D459E7D9CEB42A64396
:10C0A000B7852CD7B6F069AD292E0DA66AF9D1E275
:10C0B000A99C2F18934A79CADBE4CB164D69C73384
:10C0C0004824DD4605C0BB3AC28FD5A812B16ED058
:10C0D0005C53240519A94DFD28E80C8FA885F7D4D9
:10C0E000585610514ED1EC512148390C71C661544B
:10C0F000A120B694728318879D18878A762492A00F
:10C1000013F379984F26E40648ABF60ABC4442CEB6
:10C110008663942DE60B6B68CBFCD64E391FFD3D34
:10C12000EA2960FB56C2BDF1B445758A472B5566B6
:10C130001BE5785B134175A94FAD6D0BDA1DB46F2C
:10C14000C62ED805D14592B53F94B4946F8527A5E6
:10C15000A645FBBE96E3335BEFAF2C40397498A540
:10C160009F2C5CC304FEF09E5C4A65F8D2B5B9D43E
:10C1700096ABC261329C0EE114ED9E00FC0D5C8911
:10C1800023812757F810E860EF03718D601F36EFA9
:10C190006EBDE1A8EBA2367121E2A29C6134714E22
:10C1A0007D7457EA4047A568C5BC21DCE4C21FD0B6
:10C1B000879ACC1E312DABF324F3C123E63D9A4A76
:10C1C00021322810CB0398A3A1B9B19D5B83DFC1B5
:10C1D0006D19B2C0C90E7E85E96C6578B77553805C
:10C1E0005099D538453F5FBC8B4416F3F54C4869F0
:10C1F000FBE8D30E594384E79EA0846677F2B26FC2
:10C20000064A91C428724991C6164E91133951FFBE
:10C2100026C8BC45F83E126027C29B4B57559BC5AC
:10C2200023A96CEC170F2418DAAF34EFCC4995979B
:10C2300093A5B7A4B71D793B216B93451CCD14C5BD
:10C240001195E8DBAE9537959361BA6CA8C800D715
:10C25000B0BED8C972B65ABDBEF8385BCF6AF1001D
:10C260007EF925ED30907E057E71573E657B21304D
:10C27000EAA8E98FC99F697ED897EF39F252C920A1
:10C280007D28656FF2AC6644410D40749BD094CF1D
:10C290009ED655DEE5DA5CF99B62EE72CDCF28437F
:10C2A000DBCBC5B77FB346BAE94A3D42C93723E580
:10C2B000DA62AAB9BF7C8997B90CDE0BBFEA4D8A56
:10C2C0006BDACDA510FDFF2A2274DB91492F3DAF1B
:10C2D000769F0F6630F7D107BB0FE1E8F07E9549F6
:10C2E000980965C2266F8A04D9AFCD724686226E40
:10C2F000D731CC1B5E4819E548EFCC88576AB49E0D
:10C30000FD8E2DC2C3B25E516349A72E24F44E07A1
:10C31000A510F82734FEE4598F970286C9AA53D492
:10C320003A531079107873A87DF12E95BD5248DFED
:10C330008D5B78039D0AE8C8618167B081CB750881
:10C34000CB5CE948871BCBEFB907D67431C334AD5A
:10C3500049914E7199C66E707F01DA29F1AD41CBDA
:10C36000BA193BA6D7F8717BC5D8F620FA91F07DB3
:10C370007266CD41A07A579414C6A0D6FD3E63CF15
:10C3800078475BA05B69A52CA747FFB324ACE6CD3B
:10C39000E292E88E75BCA3B53AC2221386B923E0B7
:10C3A0001955B20CD04B7E224874E1B287150B05AB
:10C3B000FAF9CC8788FE6FB3CDDD4B1251E8D0116E
:10C3C000D7BB0B432EE39618A7CA9B95A34A436499
:10C3D000A0D82DEE87CAA814F0760089CCFA1B38B5
:10C3E0007F078ADAC79FCC66899167054624FE14C9
:10C3F0007791AE43FB6D72E0868CE870522C8A0711
:10C400009618AC7751896E91F5C5ABC7339F3797B6
:10C41000FD8364B1AE883222F26C85BC646F7D1AF4
:10C42000F6EE834372A0A6DF3982752C0DC98D32DA
:10C430002BD4FD8B179A0D2B64AD4B5D2EE124F6AA
:10C440009742FB17B868B2A8D985527FBEB0EB0AF5
:10C45000C771EE2220AEF99F68E43DAC87AF13FAB6
:10C46000CEADB82AAEB92990A3166CE98B285D62CF
:10C47000AF0A1D6C91DB1CAD7722EFAAE95F0B4779
:10C48000DA155E8EFFA3E67F32C8E577E6FAD87B41
:10C4900096E06D6301F1943BA8432191DC503E2767
:10C4A0006C208E7D38F2DB60B64AD71D48ADB527CB
:10C4B000A517AAFC83A7A8BAD96CA440916761EF1D
:10C4C000E6858F2702ABE46E1ABC508ACF9CCCB2B3
:10C4D000DC8658205449FD0550532419674B53AB53
:10C4E0008BDB85B8A6309B285256D978B263BA1236
:10C4F0000F90B9CB9203FC32408CB3875B29376A2B
:10C50000A30BE22C453715D5C4C9FB616B07948F8B
:10C51000BC07BDE73E4826291FB586706D59B83B5C
:10C52000AD11AD67FD4AB69D654971C890B81993C4
:10C53000FD6AC8718A3E59FE95A82F174E1C46BE4B
:10C54000CB96606A056FB658BDD68F25FD90B6753F
:10C55000049F0D3AE074B283BE622B528CFDC3D6A9
:10C56000303C7603C983D1FE0BC3535B648ABB1D89
:10C57000EBFCDDD8A90F3A5AE66B1FAD5DE29CB724
:10C58000A50FAAFC40D139543ABB9F4110E052E1BB
:10C59000DAB3546C51B2D886C50167A081A4FEAD50
:10C5A0000193780FA16F4E01856CF59A2B9F70A0B7
:10C5B000DECACE3ADEC981A6D82E5468BAB4135961
:10C5C000BF9D53D820EFBD23551730FB47058FF68D
:10C5D00074EA7B9A7908BF44FBA487F8999D11C33C
:10C5E00058330CAA5947F6D3D9CAC11BB4E2FDD6B9
:10C5F00064BE984D172B99C194ED395FF38BD049E8
:10C6000018278E27843E83BBF9F18F36496C79F564
:10C61000338464F758177AE44DC881E91157ADF8AF
:10C62000C0C61495C1968131E44285567B14392DDC
:10C630007669B1D0B6E57A6A0C54C6AE823401810F
:10C64000BEA8E291F941871DB0D9D72DDEBB52ECCF
:10C650003F861F4F18E643B3528D3C4CDDC975151C
:10C660007A2A6A5FF85703A2199E43166A77BA2A94
:10C67000E29FA3AD51A2176D54FB3315F5F1EF7393
:10C68000E141195DD04E0B47A42E0EC0A5351B8C81
:10C69000D91489E8381002F9202ADDD52666DCCDC8
:10C6A000B653DABF53786B359C96B211F7946A9FF4
:10C6B00066A897A6B8309D1DE128729BF508834EA9
:10C6C000924568B167EB9C0C16BFC0F10F6DBAA420
:10C6D00092D7958CB01B1B01C6A6D9BFB30B2FEA0E
:10C6E0009659349E3BF0EA2D3D47BE7F3E33629122
:10C6F0000DFB0DF0CB63EDACAB628CDF8467633E6A
:10C70000EB7D6A4809387292A9D6264FF6143B5041
:10C710005938E5BA7946719D5733EF00216AD095B3
:10C72000C1930C13B691B5528D991E1ECCB763837D
:10C73000221691626498673D2281E08D37DF6AA7F7
:10C74000A2CAB28F37435868B6D677848E9E7514C6
:10C75000A73A1E4DEAAED2B643C60486C2584DFE75
:10C76000CC6633866F94FC40FCCDF855E15ACA0F75
:10C77000E4BD72FA5DDB2E2E309CD82E86DD21F4CE
:10C78000153E9C4A0BB95A201D7FB4CDE75EB756C3
:10C790006575244D2E1E53ACBB24E8A69677971CD6
:10C7A000A58446689401CE9B13F3D4841121D8F854
:10C7B000208C0198F408086C42C2531E99C03C3783
:10C7C000F93B8A32863FB96C95FB0BF10D526381C0
:10C7D0002C21E5E67CF51133CE952774A1941B0E30
:10C7E000F3816620066C09C7A1F3FD7BCE484DF0AE
:10C7F000698AC6DD05D521B0F0541FF8516E7EE47C
:10C80000B09FC47023F92607D7F32193EA2C85C97A
:10C81000582885826EC1DC943990201F561E17540B
:10C82000E8A723B2D03921843AC82792FC3D1548A5
:10C8300048E85642989422DAD3F7495CFF1FFFA0DC
:10C8400043BF87DEE11EF38BDBED304C5300D1326A
:10C85000C5D4FC0A8CF8E15BDB097C51F7FC11F7CD
:10C8600045E2E0526C604CF536E4D3B64E83E47991
:10C8700077BCA19354C7E8B0E739829BCA433F42D3
:10C880004019BE27ACDE23E605B11A4D12ADD7180C
:10C890006AEB6D38D99E736752F966956D50269F85
:10C8A00072ACF5AA33E492F15A41B497057301C50D
:10C8B0005C69D91B785108C52D91DFE3EDCAC4141A
:10C8C000860816D0CBF0B8B24901CD4EC1E044661F
:10C8D00027637921E9686AE84934903CD64C02FB29
:10C8E0002F395B2471A008EAF9BD50C0A4E6C087C7
:10C8F0004B66F49D81CF6A0A7002D48988E4266D64
:10C90000612231F69AD0B93AE74623239174F94C63
:10C910002538CA3A2535CD4D4727CDFE18557E3AE4
:10C92000998FE7F2CDF30F07AF35DB5161D0E534D6
:10C930008BA7EAFF18824B027BF341CE9C9E0558E1
:10C940003B53BD913572167803D5DF29CBE5E888D6
:10C950004826FC37E8D3F2EAE9F8087FA6C9A42AFA
:10C96000668BEE8201185BAD6F4D6AC6D1B79E181B
:10C9700039A605A0880A0F8D169BD4421D2BE6BC54
:10C9800058A73696921B5D3C61E6C22C8F52CF822F
:10C9900008937C65F8B7C7D6BFD6F08DC97FAB7F4B
:10C9A00055446EDF676078E16024E68C176CBA7FCF
:10C9B0001F68F5C1767FAED8C46F9992E84479328A
:10C9C0003F89BCFAD33B4A68EA2B298BBF6F3A9C5C
:10C9D000C9C3C9BC7E11BB851BAD355C17598B1B08
:10C9E00051C5CD1B180A820520D708B326313C89D2
:10C9F000043BAB9C6FAD0E37C4CF18BBC39C55DA5C
:10CA000003B89F1ECC755EFBBEBE00CC43428FF9BF
:10CA10001E47DFA6DC7F8F9AB7AF03D7EA9EB0AF81
:10CA2000EF72D5278376AC6683C7C5C95C126A12DC
:10CA30008C3AB6FEBF5AC664D1BEBA6776EDFEBF69
:10CA4000183AE174A0108855383E62183E84B8D96F
:10CA500052559F8FA3716C91DC283D61B8774E5F72
:10CA6000EB55FF93104432CBA5765C6A8307BF3742
:10CA700053356D75C4B45230543DA9A148E491D5E5
:10CA8000DE6681AC904DCBC2946C6D50BDD8BCFAC3
:10CA90009925A2B74E131D6236DFDDA9F97D8FBA45
:10CAA000FD9ED5D45B6BCF34BB3B3471606AF12BF8
:10CAB0007C36E4F66DEAA3CEE833506729AEFA98E7
:10CAC00043F93B2D1E46E5A1C25ADF19C990C9B1F1
:10CAD000F9610FB908572510C4339D72A1BE5136B4
:10CAE0000B1023132395C11368FDB6392F04E19A67
:10CAF00049D2023E2F7A62EC6F1C8E7C4365DF3296
:10CB00006064B12808C7E67CB12B712C77C52CFF77
:10CB10005544E5DB93912DD7DA32B2603B2C44E1EA
:10CB2000AD10D0B9E66C7440D5C304FEC47B73600D
:10CB300000D679EA587619A72549508697E11B4017
:10CB4000D52904E93FDBE987BC82DF822F82DE51F1
:10CB5000050035E41B7796B16E3053CBDBCA4A3DF6
:10CB6000107C244FFF0F601510C230BA03BC082B95
:10CB70004BCB3E462360B5D9CAD8138D3898545252
:10CB80001ADC23FC116C00798A49509EE24CBACE23
:10CB9000012D4B09F49276D0A8EAFE4C6210427C3B
:10CBA0002A835138544A674E78D35A2CEBFF8AE9CE
:10CBB0008078574EF6436159692875A31B9F293227
:10CBC0008E7641184D0FA0B7C92547109D3419CC5A
:10CBD0002503F448958B2E8B7DC228828702083569
:10CBE0009FFE36D1AFF678CEB0D2AE6CD9402A7760
:10CBF0006F3C0DBBF297F366CCD17BF301D0577A33
:10CC0000694F993861DC4A174579CD5310B2A8E0D5
:10CC10006C94C0A914CC48D174DAE9D0DFC3C73A08
:10CC200014B42B55E8442ACA8A5931AD17178F9B83
:10CC300094DE1ABA0B1AB6E447B98FF31D252A36CB
:10CC400020FFAEB298DE5AD8B82F5A84244E744CC6
:10CC5000ED94DFB56B4043F7846DCFD302C4146EFF
:10CC600035B3807743B0D9165264E8B4A5BD47EF19
:10CC70000AF8E76220515F56760E05BE58716DD1F5
:10CC80004BC1B16F7246FED632B31D97577C7340CD
:10CC90007770DA810F4DE93F186A13D6AFA59DACC6
:10CCA000C5990D2D5CF268091E058A3B52BE4C05E4
:10CCB00021184C25971492B717DFDDD5645DCA1093
:10CCC0001776791E7BE9208B8C6D1F7E071814B4B4
:10CCD000C58D1422BCD8E266789AFF6504297019C4
:10CCE0004C08BA1778E33473D4F1D232F4EC59EB30
:10CCF000E45F25ED73FF503D23E2F00F04A2EC96B4
:10CD0000D1197DDAB9E2DCBD998079FB21C996C4DD
:10CD100023D905ECDE13298B1A8113CB7596ABBF93
:10CD2000B8771BD94AF113C58539B3C43C0A8303CC
:10CD3000555573CD31991CAE2017DDA8DB22E8D9FB
:10CD4000A3EC419A07E9898F9CD3ADAB0CE57AA39C
:10CD500089195B64F8326F9D6E933299C96CBEF08D
:10CD60001BD71B123DDDDD5A6F49E940F76193ACDB
:10CD70003239D0B571077C45B049768886244D0795
:10CD80000607BC8C02FB1A04DC26E91C9F1FD46B2F
:10CD90000D118CB937240C6E800F3D678CADCA6ABB
:10CDA000FFB936DF0978841B757E53BB5A68D41BE4
:10CDB000E3079DA16FFDCFF5D2DC9540713D3C6549
:10CDC0006C25FDEB94592DA3F3F7C81B73DAB5AAB4
:10CDD0006034E0D134181A9F3A6007F3FDE576EF2E
:10CDE00031CD7F7479F3BECCD4594DB0B4C192F239
:10CDF000C4D97C98B5CAB3E886B59079A734E20A5D
:10CE0000198A8630354CA27417967C7B15F3BBF9D2
:10CE100014E959E125A576A4F3CB60E2AFC5658C92
:10CE20002B526C04C8F247FA8448795C19083AB767
:10CE3000C90FD5175F405F25CB6687B0601D1942CB
:10CE400075F3C186D03C04A1AE5CA315F8F444444C
:10CE5000385E2199994391305A5D028E5D5E4AD3C6
:10CE6000CD6B7910BB85AF8C0C000B23FE04C43650
:10CE7000CABD9BE6E4139D30BF4CE538D7FD3A3B75
:10CE8000059ED119153BF00C0062713A28CF07C0FE
:10CE90009E2576E269B5B96EF7F54B65BFD7BBCD78
:10CEA0009DF64A1D66D05608E07D79024197E195CE
:10CEB000A7A82F7B08CC7B746D774F9C15D9690D83
:10CEC000D5435A43A5B6AEBDB2EC56118FE26942C6
:10CED00004D410141B52440015E1422AF4D5E6761E
:10CEE000332185BBBEC375EBEB7BEABEF6EDD811F3
:10CEF000A270D05A04BC58C0016195A5D54B954786
:10CF0000B368EF98AF8EEF253A8CAF54B0880B7FA3
:10CF100002E6F31FDA0125F86ADC4CC30DDB125878
:10CF200037D4C8C1AE5E109157CE17554B95C0B7D8
:10CF3000744D8D6E663539B9A5E8909725B2456B6D
:10CF400045A4D011F2426E6D50CBD85F4E788AD492
:10CF5000DF9A26BAB521D7B5B4D36546AD95F5129B
:10CF6000A212CDCFE8E7C124F8B616A9FDB8270D67
:10CF7000FE94E6684E38B111BFE38155B589AA89A0
:10CF800093D676489F755DDDB5A399414DA2BE79D4
:10CF90005F0C185802B72BA67D6561AA71751DC577
:10CFA0007F7B111820022CF9FD5A7D1D3A00273B8A
:10CFB00083FB30B6D53CF3113F1BD8D5B02121E01F
:10CFC000FE58154E79C46F5BEBB135D358A3AE96BE
:10CFD000F48420774470A738DE4DAEB358AB1DBA49
:10CFE000BFC720A6153FD0789F5E10782820DE8D21
:10CFF00089BEA9876C1CF3709A6D8688AFBF0F231A
:10D000002A509F59410CBB7B97551C045CF6DBAE44
:10D010002C8B6F4024C9D311DF689F3AC7220E9131
:10D02000217DA6407EA5E4F81AEE101CD6322E4EC5
:10D030008D23019EED9A0D3BAC251A396414752A97
:10D040005CB5F936BC748473078939948FBF28EABC
:10D050009B9C09A690EC019EC00BF1FC870B5F0D19
:10D06000ED295BB346B51E4B0D132FA4D558BDDB80
:10D07000AD30160E174C9CBDB1AD2F4FD0530446AA
:10D08000FEBE48C1614B6147E65DD6719E9DA36BB4
:10D090004E84BD2A7E912D377F3F0964CCF654AB78
:10D0A000B4D88A19DC5A9553E26127E89D833A8601
:10D0B000CD6325B41EC5A9701F0BF225E6901C1880
:10D0C000EA37E0D5E2839AE6125786F328B9299623
:10D0D00093344216702F4EF4AEF3491DDB5BD4BE81
:10D0E000D4573A63EB18B98FFEC80588832BD30752
:10D0F000E4A7E7866C8F847EF248DFA3EB242FFE43
:10D100006F08F1F2DC46EFE6041E67F10BC845FE3E
:10D11000FC2CAF533B78802F3E92F94F9FB70BB258
:10D12000CE2C87A1E212643F9BDAB8BBB60E144C3A
:10D13000BF5F9EAFAE8FE5B3F1D21AE259F05561F1
:10D14000DEC64D05F5CAC983A42332103FD0E97F5E
:10D15000823BC89A1C12A5082B461136B21E4912F2
:10D160006C7EBB75A313D31F64134FDC56FED8BA75
:10D17000C265E95C13AE08E49B475031AF1C8C9C40
:10D18000AA20434FAAEEDF1EF94A30A6DA69BFA9EA
:10D1900087E5C6360386DE03642EF0AFC5A1C2095B
:10D1A00032783B11EDD90A5D113FFC5723A2F2D62C
:10D1B00077881C667BE2899F18322BF6F13FD8876F
:10D1C0008D83CF317D5E91907A7E165DE5CDA78609
:10D1D0007E7B2D32C70BBACD82025AD9B782198411
:10D1E000DA68838B92BBBAB1E8B339C9FEDCD0E907
:10D1F000576FD27BA091DD125261FACEAA6D0DDC81
:10D200003881396A3ABFE2A6D4CE3D4482D7A3B969
:10D210005D0FAE52586E8D3E645A1AF1B45F588E4F
:10D22000A1AC383B78C42316C8F14AB83175E6CBB7
:10D23000CEFD7E382226E3B02A78ABF7285EAD8F8C
:10D24000B680ED4B3A38C3DDC45750FF72F098BD3D
:10D250004BD1E750E178901D6426A18086813FB2D2
:10D26000CC87E08C26FDE22F54CD19A501E18AFC84
:10D27000C93C25EA559622A14CE84D0F7F3E8F0B05
:10D28000DEF5E5A07D00E72B6F69EE2548182C61DF
:10D29000622071B5D7EBD2227D37517A3436224ADB
:10D2A0001031AE216FEE626328E5FA8FF51AB4AF44
:10D2B00032964DC3A55FCAFE9FB2BA7812FEF70A36
:10D2C000BEDEDC8265D8D94EC286FC245FD75216FA
:10D2D000928A98024D39DB92EFD27CC3927AE56252
:10D2E000D30A9A644692A3A9823D4458D1542B9400
:10D2F0007AD2DA19B9FC49DA90E8ECDDBE3484D68A
:10D300002EAE27862E7FF22D1DAC4222FAA0765338
:10D31000E3E692D1283272566604F9F9483326437F
:10D32000B3CE2019FAC2F0FE688B39FC1E8A111B9D
:10D3300079711BF261FD81963F25528B236D5D96BD
:10D340000ADFCBAEBA056CCBAE1FAC00ECB35A040F
:10D35000234C0000FAB529D656F863F62E230012A6
:10D3600069E470A78D14E7581569CE699AA4A81DC1
:10D37000D0148BAB8D4F7D1098E9DFCAA53685DCC4
:10D380008E7ABCBA44F73FAFF74DCCC1836B3AF508
:10D39000E2CC221DB6777588B4F6C3AECCEAB9B834
:10D3A0001BE0B43ECA5092BF59027E7DAE5EE5DA04
:10D3B000FF66F4949E0221344972932489728E741C
:10D3C000936C9DB177F44A422B9532C3EBA741820F
:10D3D00001998937D8838521A115F789D827905CD1
:10D3E000131BA7E8D7FD6F055B72766F23D0847F90
:10D3F000F361ED0D0326E92F864142E8CDCD4FEFD5
:10D4000026B5701512B1D0D37D22BB91F891F3E807
:10D41000C6E1B047CE287FB29F0EC6ADC39E30B5E1
:10D420006F79FF8479B7B30FBF6CD2870FABE4BBC2
:10D43000AE22BE1F206029F98ED5E295181F06C5C1
:10D4400045D66570BB1BAED2EEE2A477FAAC3F16B0
:10D45000E36EE90FA379BEED33D46702427E5560D7
:10D4600023A6057ACCDDE546D54D9366C078C3F892
:10D47000633AF24370DD63AC3DDA5A4D0D0D9117FE
:10D4800097E8B0F6C2082AE0B2787B86F9609FA9D7
:10D49000F3E993CBE3FDFB3A95B85A841AC585832B
:10D4A0003C185FC1A1254E3E4E1D197D41D174B07F
:10D4B0005259CF51BF5BFA2F6308DC337954935D27
:10D4C00027516294C42B29A21E191DEA4710E91D99
:10D4D00054017C72B5FFE1D45B03C3A0E538A79E7D
:10D4E0002A38B19D9AEED7E6972A8FA5FFB9E25464
:10D4F000BFA7DED2DB0340201128F72E4CA7280758
:10D50000490EEE8D50157BA6F442B6058F4056812C
:10D51000E0979D4B4ADB9729FB24B379FA6275EEBD
:10D52000511884D54CE5E59A44CB90695B63F6B01D
:10D530006CDADDF48DE7A178913620D9D3E93BEBA5
:10D54000A2DD6B4DC0E5463059CFBF295F2D7CA5CC
:10D550006910745857DD690952E74F9CB223618303
:10D56000FF5CFCDDA2EFFCC9363A3B188BCBEBA687
:10D57000A969A478330F3B6810E094A957DCCFF970
:10D58000CAFB9C84F10210EE75AD93AE6DFD51B3F4
:10D59000C6A4832F2BC2C9E1ADB941A164323C546A
:10D5A000CD81D78BD114A5DC551070AD22F5D38475
:10D5B0002B037D935E76E70781BDFAD99E62DB5926
:10D5C0003A734B03D000D6BBB2B29EF8C6E2309E8F
:10D5D00074B6979C57AD6CC23A4584B9C1FB62D012
:10D5E0008D3DCD9CEB1A36B7D86F492DE88A901A3D
:10D5F000D3AF8551A611363096B8D5BF3C8FE99A86
:10D60000CDD9A8BD90DB1BA178D92DD4EA117A47DA
:10D61000683B56CBD4FC98F7841E6C5BC8C3C4C06F
:10D620006D4FA540FA4453925DCAF07C298100E415
:10D6300002B5A7CB7C6B785D260459F86338846CFF
:10D64000D7D18A2B4C8B6EAB47F584C08CB4A980A4
:10D65000C00ABF371C9E7B08E0B9D44CA31F0A6FD9
:10D6600048C006E0D02965DD1053EE5CD759DDB225
:10D67000B2CE2FF2EECEFD8677A503A9DCB712431A
:10D68000DED6350022B54DCABD5B77AE713F13DEE5
:10D69000BC4488CE6BB954CD61871C138957D55FC4
:10D6A00045E7A11A927FA5EC451CE603C80CF826B5
:10D6B0009713B8B2161825681AA2066582B7F99DA5
:10D6C000ADD519B95E3C580DD881DE859F492A73C6
:10D6D0005070E49C4913BFEA52D85200F3227533CC
:10D6E00068E9367DD8E50A58E3E498A5D82EADE47C
:10D6F00019988CDBB2B130A34F78D0CA96C46617A4
:10D70000439AE3A6D7632CE83C391C03A82606D825
:10D71000F35478A2D91C8F7063D3C6B8F80BDC9F82
:10D720007B76309D3B7A813E7D3676FE09F0800621
:10D73000F377B3D1A2D773C64AB8E91C367E51BF7E
:10D7400007AF8C1BBC909BD199FA541B0E5E93358E
:10D75000AAAD1753A23CD159CC6E1AA6A528440AEB
:10D7600042E5796885CF6A8E74631D5AAF6A983630
:10D77000DB8941A9E33993D9293AB8BC2EC2E62EF8
:10D78000C9FB12A4B2537CA73927101BD38C95492F
:10D79000075487DBE18DF062E919EB4A6C835A325A
:10D7A000FF0035A20304050A08060BFF0209070D56
:10D7B000010C00FF2025692025692025692D256998
:10D7C00000202025633A256900202020205F5F7C0F
:10D7D000004D454D4F525920434C454152002C00BD
:10D7E00044697370206F66660D0A005553455200F8
:10D7F000424547494E0052414400442E4D59005580
:10D80000534552202020006620200067202000423F
:10D810004547494E2020202020005241442020200E
:10D8200000442E4D592020200043202020001C17AA
:10D83000171717181D191B01000001010101000035
:10D84000081C242C4448586C74434853200000039F
:10D8500006090C0F1215181B1E2124272A022D3031
:10D860003336393C3F4245484B4E515457025A5D7E
:10D87000606366696C6F7275787B7E818402878ACB
:10D880008D909396999C9FA2A5A8ABAEB1D5300080
:10D89000D53100D53200D53300D53400D53500D58B
:10D8A0003600D53700D53800D53900D54100D542EE
:10D8B00000D54300D54400D54500D63000D6310010
:10D8C000D63200D63300D63400D63500D63600D650
:10D8D0003700D63800D63900D64100D64200D643AC
:10D8E00000D64400D64500D73000D73100D73200EB
:10D8F000D73300D73400D73500D73600D73700D715
:10D900003800D73900D74100D74200D74300D74469
:10D9100000D74500D83000D83100D83200D83300C5
:10D92000D83400D83500D83600D83700D83800D8D9
:10D930003900D84100D84200D84300D84400D84527
:10D9400000000306090C0F1215181B1E2124272A9C
:10D95000022D303336393C3F4245484B50555A5FD3
:10D960000264676A6D707376797C7F82878C91968A
:10D97000029BA3ABB3BBC3CBD3DBE3EBEFF3F7FB70
:10D98000DC3000DC3100DC3200DC3300DC3400DC75
:10D990003500DC3600DC3700DC3800DC3900DC41E7
:10D9A00000DC4200DC4300DC4400DC4500C4300005
:10D9B000C43100C43200C43300C43400C43500C4D0
:10D9C0003600C43700C43800C43900D8672041008D
:10D9D000D867204200D867204300D867204400D889
:10D9E00067204500C53000C53100C53200C5330091
:10D9F000C53400C53500C53600C53700C53800C57B
:10DA00003900DC67204100DC67204200DC672043EE
:10DA100000DC67204400DC67204500C7302C2078FC
:10DA2000883000C7312C20783E3000C7322C207857
:10DA30003C3000C7332C2078873000C7342C207846
:10DA4000863000C7352C20783D7900C7362C2078E9
:10DA5000887900C7372C20783E7900C7382C207889
:10DA60003C7900C7392C2078877900D8C14100D88B
:10DA7000C14200D8C14300D8C14400D8C14500000C
:10DA80000306090C0F1215181B1E2124272A022D2C
:10DA9000303336393C3F4245484B4E515457025A79
:10DAA0005E63676C6E767E8185898D919599029D06
:10DAB0009FA4A8ACAFB3B5B8BBBEC1C4C8CAD93067
:10DAC00000D9E900DA3000DAE900DB3000DBE900F8
:10DAD000D8E900D84900D64900D74900C24100C260
:10DAE0004200C24300C24400C24500D93100D949B6
:10DAF00000DA3100DA4900DB3100DB4900DCE90003
:10DB0000DC4900E5E900E54900E54100E54200E5C2
:10DB10004300E54400E54500852C720052414E2348
:10DB200000434C780046524143004900434C525F49
:10DB300052454700DC524553554C5400D89700D805
:10DB4000E5E900D8E54900D8E54100D8E54200D82C
:10DB5000E54300D8E54400D8E5450053004C535454
:10DB6000780052544E0041425300528B00524E44B2
:10DB7000009800EA9300EB9300EC93007891004C3E
:10DB80004E004C4F470025009B25000002080C105A
:10DB900013181C1E202225282C2F013336393F4410
:10DBA0004A50565E646A6F767A800185878A8D92C4
:10DBB00099A0A7ABAFB3B8BCC0C401C7C9CBCDCF88
:10DBC000D1D3D5D7D9DBDDDFE1E32E00454E544577
:10DBD0005200522F530043485300528C00783C3E71
:10DBE000790045455800EA00EB00EC0094780065A8
:10DBF000920031309200799200312F780078210024
:10DC00008A52008A482E4D53008A52414400485996
:10DC10005020EA0048595020EB0048595020EC00B1
:10DC2000D8524553554C5400D852414E2300DC5233
:10DC3000414E230050792C780052653C3E496D00DE
:10DC400050534500434C525F97004C2E522E008299
:10DC5000008A50008A48008A44454700485950933A
:10DC600020EA004859509320EB004859509320EC8B
:10DC70000044454700524144004752440043792C38
:10DC80007800494E5400783D300078867900972D11
:10DC900000300031003200330034003500360037E8
:10DCA00000380039002B002D002A002F00972B0090
:10DCB0004ED8000041D900007FDA00008BDB000065
:10DCC0008DD8000080D90000BEDA0000CADB000059
:10DCD00000000000FE000000C0DC0000B0DC00001E
:10DCE0003F3F3F3F00040C141B21272D33393F4594
:10DCF0004B51575D63696F757B81868B90959A9FB9
:10DD0000A4A9AEB3B8BDC2C7CCD1D6DBE0E5E9ED7E
:10DD1000F1F5F9FD959620004D41545249582000E7
:10DD2000524553554C542000534F4C5645200052F9
:10DD3000434C202E0053544F202E00555345522063
:10DD40000054455354200052434C2B2E0052434C58
:10DD50002D2E0052434C2A2E0052434C2F2E00539E
:10DD6000544F2B2E0053544F2D2E0053544F2A2E18
:10DD70000053544F2F2E00783C3E202E0044534534
:10DD8000202E00495347202E004C424C202E0047A5
:10DD90005342202E004C424C200047544F20004755
:10DDA0005342200052434C2000783C3E2000445314
:10DDB000452000495347200053544F200052434C04
:10DDC0002B0052434C2D0052434C2A0052434C2FFF
:10DDD0000053544F2B0053544F2D0053544F2A00DF
:10DDE00053544F2F0044494D2000464958200053BA
:10DDF00043492000454E4720002869290053494ED9
:10DE000000434F530054414E0053462000434620E8
:10DE100000463F2000000404040404040404040435
:10DE2000040404040405D86720E900DC6720E90045
:10DE300015DE000026DE00005D0000006D00000021
:10DE400034DE000030DE0000110000000004080C89
:10DE500010030303030303030303030314181C2029
:10DE600024C6D84100C6D84200C6D84300C6D8440C
:10DE700000C6D84500C6DC4100C6DC4200C6DC4313
:10DE800000C6DC4400C6DC450003030303030303B0
:10DE90000303030303000303030303030303030355
:10DEA000030303030304C6D8E900C6DCE90000004D
:10DEB0004CDE000089DE000061DE0000A6DE00000E
:10DEC0003A00000096000000B8DE0000B0DE00005E
:10DED00015110000000306090C0F1215181B1E2156
:10DEE00024272A022D303336393C3F42454802026E
:10DEF000024B4E025154575A5D606366696C6F72F3
:10DF000075787B027E8184878A8D90939699020230
:10DF1000029C9FDD3000DD3100DD3200DD3300DDAD
:10DF20003400DD3500DD3600DD3700DD3800DD3959
:10DF300000DD4100DD4200DD4300DD4400DD450041
:10DF4000C83000C83100C83200C83300C83400C827
:10DF50003500C83600C83700C83800C83900DDE9C8
:10DF600000DD4900DE3000DE3100DE3200DE33004D
:10DF7000DE3400DE3500DE3600DE3700DE3800DE5F
:10DF80003900DE4100DE4200DE4300DE4400DE45B3
:10DF900000C93000C93100C93200C93300C934009A
:10DFA000C93500C93600C93700C93800C93900DE93
:10DFB000E900DE4900DF3000DF3100DF3200DF330F
:10DFC00000DF3400DF3500DF3600DF3700DF3800E8
:10DFD000DF3900DF4100DF4200DF4300DF4400DFC4
:10DFE0004500CA3000CA3100CA3200CA3300CA3400
:10DFF00000CA3500CA3600CA3700CA3800CA39001C
:10E00000DFE900DF4900E03000E03100E03200E00D
:10E010003300E03400E03500E03600E03700E0385F
:10E0200000E03900E04100E04200E04300E044004D
:10E03000E04500CB3000CB3100CB3200CB3300CBFE
:10E040003400CB3500CB3600CB3700CB3800CB3992
:10E0500000E0E900E0490000D4DE0000D4DE00006A
:10E0600013DF0000B5DF000080000000FE000000AC
:10E0700060E0000058E000003F3F0000E13000E1B8
:10E080003100E13200E13300E13400E13500E136F6
:10E0900000E13700E13800E13900E14100E14200F0
:10E0A000E14300E14400E14500CC3000CC3100CC3C
:10E0B0003200CC3300CC3400CC3500CC3600CC3729
:10E0C00000CC3800CC3900E1E900E14900E2300041
:10E0D000E23100E23200E23300E23400E23500E2F5
:10E0E0003600E23700E23800E23900E24100E24265
:10E0F00000E24300E24400E24500CD3000CD3100B3
:10E10000CD3200CD3300CD3400CD3500CD3600CD3D
:10E110003700CD3800CD3900E2E900E24900E330B4
:10E1200000E33100E33200E33300E33400E3350081
:10E13000E33600E33700E33800E33900E34100E36E
:10E140004200E34300E34400E34500CE3000CE311B
:10E1500000CE3200CE3300CE3400CE3500CE3600B5
:10E16000CE3700CE3800CE3900E3E900E34900E4C1
:10E170003000E43100E43200E43300E43400E435FC
:10E1800000E43600E43700E43800E43900E44100FC
:10E19000E44200E44300E44400E44500CF3000CF13
:10E1A0003100CF3200CF3300CF3400CF3500CF362F
:10E1B00000CF3700CF3800CF3900E4E900E4490050
:10E1C0007CE000001EE1000080000000FE00000076
:10E1D000C0E1000058E000003F3F000000030609D6
:10E1E0000C0F1215181B1E2124272A022D31353938
:10E1F0003D4145494D5102020202020255585B5E03
:10E200006164676A6D707376797C7F0282868A8E1C
:10E2100092969A9EA2A6C33000C33100C33200C3B7
:10E220003300C33400C33500C33600C33700C338DE
:10E2300000C33900C34100C34200C34300C34400CC
:10E24000C34500C32E3000C32E3100C32E3200C39D
:10E250002E3300C32E3400C32E3500C32E3600C328
:10E260002E3700C32E3800C32E3900C03000C03115
:10E2700000C03200C03300C03400C03500C03600DA
:10E28000C03700C03800C03900C04100C04200C0E3
:10E290004300C04400C04500C02E3000C02E3100F5
:10E2A000C02E3200C02E3300C02E3400C02E3500E8
:10E2B000C02E3600C02E3700C02E3800C02E3900C8
:10E2C0000202000306090C0F1215181B1E2124025E
:10E2D000272A2D303336393C3F4202020202020225
:10E2E000020245484B4E5154575A5D6063666902BD
:10E2F0006C6F7275787B7E818487D93200D9330048
:10E30000D93400D93500D93600D93700D93800D9E9
:10E310003900D94100D94200D94300D94400D94538
:10E3200000D03000D03100D03200D03300D03400E3
:10E33000D03500D03600D03700D03800D03900DAE0
:10E340003200DA3300DA3400DA3500DA3600DA3750
:10E3500000DA3800DA3900DA4100DA4200DA430044
:10E36000DA4400DA4500D13000D13100D13200D199
:10E370003300D13400D13500D13600D13700D13847
:10E3800000D139000202000306090C0F1215181BF8
:10E390001E212402272A2D303336393C3F42DB32FE
:10E3A00000DB3300DB3400DB3500DB3600DB37001D
:10E3B000DB3800DB3900DB4100DB4200DB4300DB04
:10E3C0004400DB4500D23000D23100D23200D233DB
:10E3D00000D23400D23500D23600D23700D2380015
:10E3E000D2390000DCE10000C0E2000084E300005C
:10E3F00016E20000FAE200009EE3000010000000B8
:10E40000A9000000F0E30000E4E300003A3818003F
:10E41000000306090C0F1215181B02020202020269
:10E420001E22262A2E32363A3E4202020202020200
:10E4300046494C4F5255585B5E610202020202028D
:10E4400064676A6D707376797C7F0202020282D300
:10E450003000D33100D33200D33300D33400D3356E
:10E4600000D33600D33700D33800D33900D62E304E
:10E4700000D62E3100D62E3200D62E3300D62E34C2
:10E4800000D62E3500D62E3600D62E3700D62E38A2
:10E4900000D62E3900D43000D43100D43200D43329
:10E4A00000D43400D43500D43600D43700D438003A
:10E4B000D43900ED3000ED3100ED3200ED3300EDE8
:10E4C0003400ED3500ED3600ED3700ED3800ED3964
:10E4D00000ED4900000306090C0F1215181B02027B
:10E4E00002021E022124272A2D303336393C020233
:10E4F00002023F024245484B4E5154575A5D0202B8
:10E50000020260026366696C6F7275787B7E02023C
:10E51000020281EE3000EE3100EE3200EE3300EE0A
:10E520003400EE3500EE3600EE3700EE3800EE39FE
:10E5300000EE4900EF3000EF3100EF3200EF330022
:10E54000EF3400EF3500EF3600EF3700EF3800EF23
:10E550003900EF4900E63000E63100E63200E633EC
:10E5600000E63400E63500E63600E63700E638001F
:10E57000E63900E64900E73000E73100E73200E71E
:10E580003300E73400E73500E73600E73700E738C7
:10E5900000E73900E74900000306090C0F121518BF
:10E5A0001B020202021E022124272A2D3033363993
:10E5B0003C02020202020202020202020202020201
:10E5C000023F43474B4FE83000E83100E83200E8B3
:10E5D0003300E83400E83500E83600E83700E83872
:10E5E00000E83900E84900C13000C13100C1320003
:10E5F000C13300C13400C13500C13600C13700C18C
:10E600003800C13900DCC14100DCC14200DCC1433B
:10E6100000DCC14400DCC1450000000010E4000043
:10E62000D4E4000097E500004FE4000013E500008B
:10E63000C6E5000000000000AE00000028E6000073
:10E640001CE600003F3F2F0038DE0000C0DE000067
:10E6500068E00000C8E10000FCE3000034E60000D0
:10E6600001000000010000006483000069830000D5
:10E670006E830000738300007883000078830000BD
:10E680007D830000878300008C830000918300005D
:10E690009B8300000305000001000000FFFFFFFF57
:10E6A0004D0000000F000000F4010000FFFFFFFF1D
:10E6B000EBD70000FB860000D5750000F0D7000006
:10E6C000C9730000F6D70000FAD7000033760000C7
:10E6D000717B0000FFD7000007D800000BD80000B6
:10E6E0000FD80000C97300001AD8000021D800001C
:10E6F00029D80000717B0000EBD70000FB860000EA
:10E70000D5750000F0D70000C9730000F6D70000EF
:10E71000FAD7000033760000717B00002020202013
:10E72000202020202020000003000000040103011D
:10E730000201010411040F04170416011801050257
:10E74000050804080B080404050105040908090468
:10E750000608070206020402060106040701030870
:10E7600003040C080D020C0203020C010C040D0141
:10E770000D080D0408020808070802020704080132
:10E780000804090209010A080B020A0201080A0129
:10E790000A040B01020802041008110210021108F9
:10E7A00010011004110112021201130213081208C1
:10E7B0000F081204130113041402140115021508A2
:10E7C0001408170814041501150417021701190875
:10E7D0001A0219021602190119041A011608160460
:10E7E0001B021B081A0818021A041B011B04180834
:10E7F00018040B040A1409001D27FF131EFFFFFF56
:10E80000FFFFFFFFFFFFFFFFFFFFFFFFFFFFFFFF18
:10E81000FFFFFFFF0B1508011C26FF121FFFFFFF64
:10E82000FFFFFFFFFFFFFFFFFFFFFFFFFFFFFFFFF8
:10E83000FFFFFFFFFFFFFFFFFFFFFFFFFFFFFFFFE8
:10E84000FFFFFFFFFFFFFFFFFFFFFFFFFFFFFFFFD8
:10E85000FFFFFFFF0C1607021B25FF1120FFFFFF24
:10E86000FFFFFFFF0E18050419FFFF0F22FFFFFF38
:10E87000FFFFFFFFFFFFFFFFFFFFFFFFFFFFFFFFA8
:10E88000FFFFFFFFFFFFFFFFFFFFFFFFFFFFFFFF98
:10E89000FFFFFFFFFFFFFFFFFFFFFFFFFFFFFFFF88
:0DE8A000FFFFFFFF0D1706031A24FF1021D4
:00000001FF
